:020000040800F2
:1000000000100020813B0008F13C0008E1C4010819
:10001000F13C0008C1C40108A1C40108F13C00087A
:10002000F13C0008F13C0008F13C0008213D0008CB
:1000300081C40108F13C0008F13C0008213E0008A1
:10004000F13C000841950008F13C00088196000849
:10005000F13C0008F13C00080193000831930008CE
:100060006193000891930008C1930008318700084C
:1000700071870008B1870008F187000831880008FF
:1000800071880008B1880008E1900008519A0008C2
:10009000719A0008919A0008B19A0008F19300083B
:1000A00071B90008F1B80008F13C000811B9000866
:1000B00031B9000851B90008C1BC0008F1A100081D
:1000C00031A30008F13C0008F13C0008F13C0008B5
:1000D000F13C000851C1000871C1000891C100083D
:1000E0009194000881950008C1950008F13C000832
:1000F00051BD0008F13C000881BD0008F1880008EE
:10010000F13C0008F13C000841B70008F13C000850
:10011000F13C0008F13C0008F13C0008F13C00080B
:100120003189000871890008B1890008F189000847
:10013000318A0008F13C000801960008D19A0008B5
:10014000F19A0008119B0008319B000821AF0008BC
:10015000718A0008B18A0008F18A0008F13C0008A1
:10016000F13C0008F13C0008F13C0008F13C0008BB
:1001700041960008F13C0008F13C0008F13C000801
:10018000F13C0008F13C0008F13C0008F13C00089B
:10019000F13C0008F13C0008F13C0008F13C00088B
:0C01A000F13C0008F13C0008F13C0008B4
:1001AC0051020008D1020008F102000811030008F6
:1001BC005103000891030008C1030008E103000883
:1001CC00010400082104000861040008A1040008CF
:1001DC00C1040008610500087105000891050008BC
:1001EC00B1050008F10500081106000831060008E9
:1001FC0081060008E1060008110700083107000815
:10020C00B1070008D107000891080008B1080008E0
:10021C00D1080008210900084109000881090008DB
:10022C00D1090008710C0008C10C0008A10E0008CF
:0C023C007110000891100008F11000087B
:1002500070B543F29014C2F2000442F620612046C9
:10026000C2F2000126F0A4F943F29401201DC2F26B
:10027000000126F09DF942F6807104F10800C2F2F7
:10028000000126F095F943F28403C2F200032668C8
:100290006568A4681E6042F6207042F630211A4656
:1002A0005D609C60C2F20001C2F2000015F0F0FB3C
:1002B00043F27C00C2F2000026F052F943F28003C0
:1002C000C2F2000300221A705A709A7070BD00BF0B
:1002D00010B543F2A814C2F20004204615F040FD08
:1002E00004F11800BDE8104015F03ABDAFF30080EE
:1002F00008B544F25810C2F2000012F029F943F296
:10030000E010C2F20000BDE808400EF029BD00BFB9
:1003100038B544F2D01044F6F874C2F20004002557
:10032000C2F2000026F01CF9204629464FF48072E4
:10033000C4F8005102F0FCFE4023C4F80451C4F894
:100340000831C4F8045138BDAFF30080AFF300802A
:1003500038B545F2041045F21814C2F20004002525
:10036000C2F2000015F004FE204629464FF48072C8
:10037000C4F8005102F0DCFE4023C4F80451C4F874
:100380000831C4F8045138BDAFF30080AFF30080EA
:1003900010B545F22424C2F20004204615F0E8FD11
:1003A00004F1100015F0E4FD04F12000BDE8104058
:1003B00015F0DEBDAFF30080AFF30080AFF3008037
:1003C00045F298204BF6146145F2D422C2F20000A7
:1003D000C0F60201C2F2000241F2883325F0D0B922
:1003E00046F274604BF62471C2F20000C0F60201BE
:1003F00025F0DEB9AFF30080AFF30080AFF30080EB
:10040000044B002103F5DC7243F8581C5833934227
:10041000FAD17047D8670020AFF30080AFF30080B7
:10042000F8B546F678460024C2F20006402746F6A4
:100430002C45C2F2000521463A463046B46402F02B
:1004400077FE3A462846214634647464AC6402F070
:100450006FFE2C646C64F8BDAFF30080AFF30080D6
:10046000F8B546F610560024C2F20006402746F6BC
:10047000C445C2F2000521463A463046B46402F053
:1004800057FE3A462846214634647464AC6402F050
:100490004FFE2C646C64F8BDAFF30080AFF30080B6
:1004A00046F6645042F63031C2F20000C0F6030155
:1004B00025F07EB9AFF30080AFF30080AFF300808A
:1004C00046F67460C2F2000047F2B40110B4002294
:1004D000C2F200014FF0FF3481608161816281636B
:1004E000816481650260426002614261026242622F
:1004F000026342630264426402654265C460C4618F
:10050000C462C463C464C46500F1740300F5B270CE
:1005100043F80C1C43F8142C43F8102C43F8084CF7
:1005200043F8042C14338342F2D10A4B002203F126
:10053000F0044FF0FF3043F80C1C43F8142C43F840
:10054000102C03E905001433A342F4D15DF8044BE9
:10055000704700BFD86F0020AFF30080AFF300807A
:1005600047F2B800C2F2000015F06ABDAFF3008098
:1005700047F2FC304FF66811C2F20000C0F60201EB
:1005800025F016B9AFF30080AFF30080AFF3008021
:1005900047F2A0504FF6BC31C2F20000C0F6020193
:1005A00025F006B9AFF30080AFF30080AFF3008011
:1005B00038B50D4C04F50065204625F0B1F904F17D
:1005C0007C0004F5807425F0ABF9AC42F4D147F619
:1005D0009034C2F20004201D00214FF4006202F0AA
:1005E000A7FD0023236038BD9C7B0020AFF3008073
:1005F00048F220704FF65061C2F20000C0F60201CE
:1006000025F0D6B8AFF30080AFF30080AFF30080E1
:1006100049F2A00040F24C01C2F20000C0F6030112
:1006200025F0C6B8AFF30080AFF30080AFF30080D1
:1006300008B549F2CC5040F28C2149F2E4224FF443
:10064000FA73C0F60301C2F20002C2F2000025F004
:1006500097F849F2DC4041F2C471C2F20001C2F2E3
:10066000000019F0A5FF49F2F41041F26871C2F2DE
:100670000000C2F20001BDE8084019F099BF00BFB8
:1006800049F60C1040F2706138B5C0F60301C2F2B1
:10069000000015F05DFC49F6201549F68810C2F2FD
:1006A0000005C2F2000015F063FC49F6501428461C
:1006B00015F056FBC2F2000405F1180015F050FBCE
:1006C000204615F04DFB04F11800BDE8384015F048
:1006D00047BB00BFAFF30080AFF30080AFF30080F3
:1006E00008B549F6A85040F63401C2F20000C0F641
:1006F000030125F05DF849F69450C2F20000BDE810
:10070000084015F035BC00BFAFF30080AFF30080A8
:100710004AF2B80040F6B871C2F20000C0F6030118
:1007200025F046B8AFF30080AFF30080AFF3008050
:100730004EF6A46041F2B4214EF6F80208B5C2F2BA
:1007400000024FF4AF63C0F60301C2F2000025F0CF
:1007500017F84EF6E46041F2C021C0F60301C2F280
:10076000000025F025F84EF2F84041F2CC21C0F609
:100770000301C2F2000025F01BF84EF2E840C2F27D
:10078000000015F0F5FB4EF67060C2F2000015F0A7
:10079000EFFB4EF68060C2F2000015F0E9FB4EF66A
:1007A0009060C2F20000BDE8084015F0E1BB00BF58
:1007B00041F2001041F29461C2F20100C0F603015F
:1007C00024F0F6BFAFF30080AFF30080AFF30080FA
:1007D00010B541F21C2082B0C2F2010026F058FB95
:1007E0004CF2AE73C4F236330024009341F234204D
:1007F00047F6E12200232146CCF2D402C4F2A00342
:10080000C2F2010026F04CFB41F20C204DF6100222
:10081000002300944FF07C51C4F2B622C4F240038E
:10082000C2F2010026F03CFB0023C4F248330093DF
:1008300041F22420002321462246C4F2A003C2F242
:10084000010026F02DFB0023C4F28233009341F215
:100850001420002321464FF08242C4F2A003C2F2CA
:10086000010026F01DFB0023C4F2C823009341F2CF
:100870002C20002322464FF07C51C4F29003C2F298
:10088000010026F00DFB02B010BD00BFAFF30080E9
:1008900041F2E86042F6405141F20032C2F20100FA
:1008A000C0F60301C2F201024FF47A7324F068BF6C
:1008B00041F2487042F68051C2F20100C0F60301D5
:1008C00024F076BFAFF30080AFF30080AFF3008079
:1008D00038B541F6201042F6902141F6A805C0F641
:1008E0000301C2F20105C2F2010015F031FB41F62D
:1008F000E004284615F034FAC2F2010405F11800AC
:1009000015F02EFA204615F02BFA04F11800BDE878
:10091000384015F025BA00BFAFF30080AFF3008078
:1009200041F6704043F29811C2F20100C0F6030193
:1009300024F03EBFAFF30080AFF30080AFF3008040
:1009400042F2F03008B5C2F2010015F011FB42F29C
:100950009800C2F2010015F07BF841F68850C2F20F
:1009600001001BF025FB42F20440C2F20100BDE889
:10097000084012F085BB00BFAFF30080AFF30080EA
:1009800010B542F2307082B0C2F2010015F060F88A
:1009900042F21C70C2F2010015F0EAFA00244FF096
:1009A0007E5100220091C4F2B42442F20070002172
:1009B00013460194C4F22011C2F2010027F0C8FFCF
:1009C00002B010BDAFF30080AFF30080AFF3008042
:1009D0002DE9F04142F69864C2F20104002142F68A
:1009E000FC27C2F201070A46204642F6E06814F0EE
:1009F0004FFEC2F201082146384614F0D1FD42F6FE
:100A0000B435396840460722C2F2010514F050FEA1
:100A100043F2CC4239682846C0F6030242F62C6401
:100A2000C2F2010414F034FE43F2D4423968204685
:100A3000C0F6030242F64446C2F2010614F028FE54
:100A400043F2E04239683046C0F6030214F020FE5B
:100A500042F6785041460822C2F2010014F028FE06
:100A600042F6746041460922C2F2010014F020FEF1
:100A700042F6506029460A22C2F2010014F018FE24
:100A800042F60C3029460B22C2F2010014F010FE8F
:100A900042F68C4029460D22C2F2010014F008FEF5
:100AA00042F6902029460E22C2F2010014F000FE08
:100AB00042F60C5029461022C2F2010014F0F8FD53
:100AC00042F66C7029460C22C2F2010014F0F0FDCF
:100AD00042F6305029461422C2F2010014F0E8FD1B
:100AE00042F6487029461122C2F2010014F0E0FDDE
:100AF00042F6247029461222C2F2010014F0D8FDF9
:100B000042F6E45043F2E84240F2F1432146C0F697
:100B10000302C0F60203C2F2010014F0A9FD42F67E
:100B2000204043F2F44243F231232146C0F603024F
:100B3000C0F60203C2F2010014F09AFD42F608600A
:100B400043F2005243F2C123C0F602032146C0F62D
:100B50000302C2F2010014F08BFD42F66C3043F246
:100B60000C522146C0F60302C2F2010014F090FDBF
:100B700042F6903043F218522146C0F60302C2F208
:100B8000010014F085FD42F6483043F2245221461C
:100B9000C0F60302C2F2010014F07AFD42F6D8302A
:100BA00043F230522146C0F60302C2F2010014F0B3
:100BB0006FFD42F6684043F23C522146C0F6030204
:100BC000C2F2010014F064FD42F6D82043F24C5208
:100BD0002146C0F60302C2F2010014F059FD42F6AC
:100BE000B04043F25C522146C0F60302C2F201005B
:100BF00014F04EFD42F6D44043F26C522146C0F64A
:100C00000302C2F2010014F043FD42F65450314693
:100C10000122C2F2010014F04BFD42F6B42031462D
:100C20000222C2F2010014F043FD42F6BC603146DC
:100C30000322C2F2010014F03BFD42F6C0503146DF
:100C40000422C2F2010014F033FD42F6FC303146BA
:100C50000522C2F2010014F02BFD42F69C503146F1
:100C6000C2F201000622BDE8F04114F021BD00BF30
:100C700043F2B42043F2407108B5C0F60301C2F25A
:100C8000010024F095FD41F68810C1F2000014F037
:100C90008FF843F2B8300949C2F2010014F078FA33
:100CA00042F6B870C2F2010025F01AFC43F2B020FF
:100CB000C2F20100BDE8084025F052BC6864001093
:100CC0002DE9F00F48F24400C2F2010082B047F66D
:100CD0009872C2F201020168019047F6687347F604
:100CE0007470C2F201031160C2F2010040F68C413F
:100CF0000090C0F60301062047F6807AC2F2010A8E
:100D0000916050601A6043F64C32C0F6030248F21C
:100D10002C09C2F2010958609A60CAF8003040F20A
:100D200000030720C0F6030347F6F078C2F201087B
:100D3000CAF80830CAF80400C9F800A043F6503ACF
:100D4000C0F6030AC9F80400C9F808A0C8F8009062
:100D500048F2380C4FF00809C2F2010CC8F80490B0
:100D600043F65439C0F60309C8F80890CCF800805F
:100D700047F65C774FF00908C2F20107CCF804800F
:100D800043F65838C0F6030847F6A476C2F20106C7
:100D9000CCF80880C7F800C047F6FC754FF00A0C85
:100DA00043F65C38C2F20105C7F804C0C0F6030878
:100DB00048F2200443F6603CC2F20104C7F8088000
:100DC0003760C0F6030C0B2743F664387760C6F82B
:100DD00008C02E60C0F603080C2643F6B8476E60C4
:100DE000C5F808802560C0F603070325656043F653
:100DF000683CA7600098C0F6030C052704604760B4
:100E0000C0F808C048F2140B0198C2F2010B47F673
:100E10005071C2F20101C0F800B048F248020098D7
:100E200048F2080347F68C7A43F66C36C2F20103A7
:100E3000C2F2010AC2F20102C0F60306022443F61E
:100E4000703843F6743543F6783743F67C3CC0F689
:100E50000308C0F60305C0F60307C0F6030C4FF005
:100E6000040908604C600D200E248E600F2682E875
:100E70000202C2F808801A6058609D60CAF800300B
:100E8000CBF800A0CAF80440CAF80870CBF8046098
:100E9000CBF808C002B0BDE8F00F7047AFF3008098
:100EA00049F21C2044F23C1238B5C0F6030264211A
:100EB000C2F2010025F044FC49F2EC2041F61C523C
:100EC000C0F603026A21C2F2010025F039FC49F2A2
:100ED0001C5041F23012C0F603026B21C2F2010035
:100EE00025F02EFC49F2D42041F27412C0F6030220
:100EF0006D21C2F2010025F023FC49F2342042F6B4
:100F00003042C0F603026621C2F2010025F018FC4F
:100F100049F20C2043F68472C0F603026521C2F246
:100F2000010025F00DFC49F2045043F69462C0F62E
:100F300003026E21C2F2010025F002FC49F24020BA
:100F400043F68C72C0F603026821C2F2010025F05C
:100F5000F7FB48F2E41043F69C72C0F603026921E5
:100F6000C2F2010025F0ECFB48F6002043F6AC721B
:100F7000C0F603026721C2F2010025F0E1FB48F64A
:100F8000F41043F64C72C0F603026F21C2F2010066
:100F900025F0D6FB48F25800C2F2010049F2F824CD
:100FA00025F0EEFBC2F2010404F500752046103472
:100FB00025F0D6FBAC42F9D149F2F84049F2F821CC
:100FC000C2F20100C2F20101202248F2F41425F01D
:100FD00097FEC2F2010404F500652046103425F0A6
:100FE000BFFBAC42F9D149F2282048F2F411C2F219
:100FF0000100C2F20101802248F60C2425F080FE97
:10100000C2F2010404F500652046103425F0A8FB67
:10101000AC42F9D149F2E02048F60C21C2F20100BD
:10102000C2F2010180220F4C25F06AFE04F5E06552
:101030002046703414F00CFDAC42F9D149F24C203A
:10104000C2F2010048F2E40425F09AFBC2F2010466
:1010500004F580752046103414F08AFFAC42F9D1B3
:1010600038BD00BFA0C10010AFF30080AFF3008017
:1010700008B5054827F044FC4CF6A000C1F200007A
:1010800027F03EFC08BD00BFF0DA0010AFF300808F
:101090002DE9F04149F274570024C2F201074FF0E4
:1010A000400849F22856C2F2010621464246384617
:1010B00049F2C055C2F20105BC6402F039F821467C
:1010C000424630463C647C64B46402F031F84246E7
:1010D0002846214634647464AC6402F029F82C6418
:1010E0006C64BDE8F08100BFAFF30080AFF3008017
:1010F00049F20C6044F26031C2F20100C0F6030113
:1011000024F056BBAFF30080AFF30080AFF3008054
:1011100008B504F06DFC02F033FF1BF0A9F927F0CD
:101120008FFE002008BD00BFAFF30080AFF300804A
:1011300050EA010301D102207047D0F1010338BF0A
:101140000023B1F1004F08BF0028F4D021F0004186
:101150004FF6FF72A1F58010C7F6DF72904201D8FA
:1011600004207047B1F5801F01D203207047002092
:10117000C7F6F070814214BF002003F001007047F1
:10118000C1F30A5C2DE9F843ACF2FF33132B06469A
:101190000F4613DC002B40DB4FF6FF7CC0F20F0C38
:1011A0004CFA03F303EA010C5CEA000C1CD107F0D3
:1011B0000041C2E900676046BDE8F883332B1EDCBE
:1011C0004FF0FF33ACF2134C23FA0CFC1CEA000383
:1011D0001CD020EA0C060F460B46C2E900673246D7
:1011E00000F09AFABDE8F88321EA030700263B469F
:1011F000C2E90067324600F08FFABDE8F88307F0D5
:101200000041C2E900670020BDE8F88307F0004113
:10121000C2E900671846BDE8F88307F000494FF0BF
:101220000008C2E90089BDE8F88300BF00000000A3
:10123000F8B5C1F30A57A7F2FF360246132E0B4644
:101240000D468C4616DC002E31DB4FF6FF7CC0F2DB
:101250000F0C4CFA06FC0CEA010101430FD04FF4CD
:101260000023002143FA06F62E4426EA0C0C084619
:101270006146F8BD332E05DDB6F5806F23D01046EC
:101280001946F8BD4FF0FF30A7F21341C840104295
:10129000F5D0C7F5866701210237B940891828BF04
:1012A00003F1010C21EA000108466146F8BD01F096
:1012B000004C013602BF4CF07F5C00214CF4401C16
:1012C000D5D00021D3E700F029FAF8BD00000000D6
:1012D00070B58AB0054600F06BF841F20064C2F2C6
:1012E000000494F900300133064609D0284600F086
:1012F000EFF928B12846002101F0A6F9034610B104
:1013000030460AB070BD44F270322846C0F603027F
:101310000893019200F060FB2478CDE90401CDE947
:10132000020174BB4FF6FF734FF06042CCF2EF73D3
:10133000CDE906232846002101F05EF978B10223A9
:1013400000939C4229D0684600F0B2F928B3089B6C
:1013500043BBDDE9060100F05BFE0AB070BD022C64
:101360004FF00103009313D0684600F0A1F978B163
:1013700043F6E410C0F6030000F0A2F9CDE906013F
:10138000E5E700230022CFF6F073CDE90623D1E78D
:1013900001F06EFE21230360EAE701F069FE2223DB
:1013A0000360D4E701F064FE089B0360D1E700BF4F
:1013B00020F0004201462DE9F84F0346002A00F0D4
:1013C000B0800028C0F2D380B0F1FF4F80F2CB8014
:1013D000B0F5000FA8BF002706DA4FF098416FF074
:1013E000180700F075FF03464FF62030C3F31604CC
:1013F000C0F24A00DB1520447F3B00F400021F448A
:1014000082F07E504FF07E51204307EBD25700F020
:1014100053FE04F10F03C3F316030F2B054640F3ED
:1014200087804FF0804145F6304800F047FECFF608
:10143000CF78A044C4F5571404F5227444EA080890
:101440000146284600F0F8FF8146384600F0EAFEE3
:1014500049468346484600F03BFF0146824600F07D
:1014600037FF48F69701C3F61761064600F030FFD4
:1014700043F22531C3F63A6100F020FE314600F018
:1014800027FF44F62511C3F6926100F017FE31469E
:1014900000F01EFF4AF6AB21C3F62A7100F00EFEE3
:1014A000514600F015FF4DF24F01C3F61C61824614
:1014B000304600F00DFF48F62961C3F6636100F085
:1014C000FDFD314600F004FF4CF6CD41C3F6CC6182
:1014D00000F0F4FD314600F0FBFE0146504600F0FE
:1014E000EDFDB8F1000F064640F3AF804FF07C51A0
:1014F000284600F0EDFE294600F0EAFE0446002FE3
:1015000059D1314600F0DAFD494600F0E1FE0146CE
:10151000204600F0D1FD0146284600F0CDFDBDE893
:10152000F88F00214FF04C4000F086FFBDE8F88FA7
:10153000002101F061F808B3002F00F083803846E5
:1015400000F070FE4FF4E341C3F63171054600F040
:10155000BFFE4FF2D171C3F217710446284600F066
:10156000B7FE0146204600F0A9FDBDE8F88F00F067
:10157000A3FD002100F060FFBDE8F88F2946284652
:1015800000F0A6FE4AF6AB21C3F6AA61044628463F
:1015900000F09EFE01464FF07C5000F08DFD0146AC
:1015A000204600F095FE04466FBB2846214600F019
:1015B00083FDBDE8F88F4FF4E3415846C3F631711F
:1015C00000F086FE31460746204600F077FD49468A
:1015D00000F07EFE4FF2D171C3F2177106465846F5
:1015E00000F076FE0146304600F068FD01462046D8
:1015F00000F062FD294600F05FFD0146384600F02C
:101600005BFDBDE8F88F384600F00CFE4FF4E34177
:10161000C3F63171074600F05BFE4FF2D171C3F2A1
:1016200017710646384600F053FE0146204600F08A
:1016300043FD294600F040FD0146304600F03CFDE8
:10164000BDE8F88F0020BDE8F88F1FB34FF4E341E9
:101650005846C3F6317100F03BFE31460446284639
:1016600000F02AFD494600F033FE4FF2D171C3F27B
:1016700017710646584600F02BFE0146304600F032
:101680001BFD294600F018FD0146204600F014FD20
:10169000BDE8F88F0146284600F00EFD494600F0EF
:1016A00017FE0146284600F007FDBDE8F88F00BF91
:1016B0000020704700000000000000000000000053
:1016C00000210020C7F6F871704700BF000000003D
:1016D00030F0004001D102207047A0F50003B3F1C3
:1016E000FE4F01D2042070474FF6FE73421EC0F237
:1016F0007F039A4201D803207047B0F1FF4358425C
:101700005841704700000000000000000000000089
:1017100081F0004102E000BF83F0004330B54FEAA2
:1017200041044FEA430594EA050F08BF90EA020F0F
:101730001FBF54EA000C55EA020C7FEA645C7FEAA2
:10174000655C00F0E2804FEA5454D4EB5555B8BFC5
:101750006D420CDD2C4480EA020281EA030382EA36
:10176000000083EA010180EA020281EA0303362DC8
:1017700088BF30BD11F0004F4FEA01314FF4801C9B
:101780004CEA113102D0404261EB410113F0004FAD
:101790004FEA03334CEA133302D0524263EB430364
:1017A00094EA050F00F0A780A4F10104D5F1200E02
:1017B0000DDB02FA0EFC22FA05F2801841F100015D
:1017C00003FA0EF2801843FA05F359410EE0A5F131
:1017D00020050EF1200E012A03FA0EFC28BF4CF062
:1017E000020C43FA05F3C01851EBE37101F0004518
:1017F00007D54FF0000EDCF1000C7EEB00006EEB25
:101800000101B1F5801F1BD3B1F5001F0CD34908AE
:101810005FEA30004FEA3C0C04F101044FEA445205
:1018200012F5800F80F09A80BCF1004F08BF5FEA8C
:10183000500C50F1000041EB045141EA050130BD6C
:101840005FEA4C0C404141EB010111F4801FA4F10F
:101850000104E9D191F0000F04BF01460020B1FA64
:1018600081F308BF2033A3F10B03B3F120020CDA9C
:101870000C3208DD02F1140CC2F10C0201FA0CF07A
:1018800021FA02F10CE002F11402D8BFC2F1200CDF
:1018900001FA02F120FA0CFCDCBF41EA0C01904095
:1018A000E41AA2BF01EB0451294330BD6FEA0404DE
:1018B0001F3C1CDA0C340EDC04F11404C4F12002C9
:1018C00020FA04F001FA02F340EA030021FA04F3DB
:1018D00045EA030130BDC4F10C04C4F1200220FA32
:1018E00002F001FA04F340EA0300294630BD21FA70
:1018F00004F0294630BD94F0000F83F4801306BF36
:1019000081F480110134013D4EE77FEA645C18BF29
:101910007FEA655C29D094EA050F08BF90EA020FC0
:1019200005D054EA000C04BF1946104630BD91EAB8
:10193000030F1EBF0021002030BD5FEA545C05D1BB
:101940004000494128BF41F0004130BD14F58004FA
:101950003CBF01F5801130BD01F0004545F0FE416E
:1019600041F470014FF0000030BD7FEA645C1ABFA3
:10197000194610467FEA655C1CBF0B46024650EADA
:10198000013406BF52EA033591EA030F41F4002106
:1019900030BD00BF90F0000F04BF0021704730B58C
:1019A0004FF4806404F132044FF000054FF0000161
:1019B00050E700BF90F0000F04BF0021704730B522
:1019C0004FF4806404F1320410F0004548BF4042F7
:1019D0004FF000013EE700BF42004FEAE2014FEA4C
:1019E00031014FEA02701FBF12F07F4393F07F4F27
:1019F00081F06051704792F0000F14BF93F07F4F59
:101A0000704730B54FF4607401F0004521F000419B
:101A100020E700BF50EA010208BF704730B54FF021
:101A200000050AE050EA010208BF704730B511F026
:101A3000004502D5404261EB41014FF4806404F15E
:101A400032045FEA915C3FF4DCAE4FF003025FEAE0
:101A5000DC0C18BF03325FEADC0C18BF033202EB68
:101A6000DC02C2F1200300FA03FC20FA02F001FAC2
:101A700003FE40EA0E0021FA02F11444C1E600BF61
:101A800070B54FF0FF0C4CF4E06C1CEA11541DBF14
:101A90001CEA135594EA0C0F95EA0C0F00F0DEF8DF
:101AA0002C4481EA030621EA4C5123EA4C5350EAC4
:101AB000013518BF52EA033541F4801143F4801315
:101AC00038D0A0FB02CE4FF00005E1FB02E506F0A6
:101AD0000042E0FB03E54FF00006E1FB03569CF0FB
:101AE000000F18BF4EF0010EA4F1FF04B6F5007F01
:101AF00064F5407404D25FEA4E0E6D4146EB060673
:101B000042EAC62141EA55514FEAC52040EA5E50FB
:101B10004FEACE2EB4F1FD0C88BFBCF5E06F1ED8A5
:101B2000BEF1004F08BF5FEA500E50F1000041EBDC
:101B3000045170BD06F0004646EA010140EA020089
:101B400081EA0301B4EB5C04C2BFD4EB0C0541EAAB
:101B5000045170BD41F480114FF0000E013C00F3C0
:101B6000AB8014F1360FDEBF002001F0004170BDE4
:101B7000C4F10004203C35DA0C341BDC04F11404FD
:101B8000C4F1200500FA05F320FA04F001FA05F289
:101B900040EA020001F0004221F0004110EBD37056
:101BA00021FA04F642EB06015EEA430E08BF20EA82
:101BB000D37070BDC4F10C04C4F1200500FA04F325
:101BC00020FA05F001FA04F240EA020001F00041B7
:101BD00010EBD37041F100015EEA430E08BF20EA2A
:101BE000D37070BDC4F1200500FA05F24EEA020E72
:101BF00020FA04F301FA05F243EA020321FA04F0A1
:101C000001F0004121FA04F220EA020000EBD37057
:101C10005EEA430E08BF20EAD37070BD94F0000F57
:101C20000FD101F00046400041EB010111F4801F8B
:101C300008BF013CF7D041EA060195F0000F18BF3C
:101C4000704703F00046520043EB030313F4801F78
:101C500008BF013DF7D043EA0603704794EA0C0F32
:101C60000CEA135518BF95EA0C0F0CD050EA410648
:101C700018BF52EA4306D1D181EA030101F00041C5
:101C80004FF0000070BD50EA410606BF10461946ED
:101C900052EA430619D094EA0C0F02D150EA0136F9
:101CA00013D195EA0C0F05D152EA03361CBF10463A
:101CB00019460AD181EA030101F0004141F0FE41D9
:101CC00041F470014FF0000070BD41F0FE4141F45D
:101CD000780170BD70B54FF0FF0C4CF4E06C1CEA5D
:101CE00011541DBF1CEA135594EA0C0F95EA0C0F12
:101CF00000F0A7F8A4EB050481EA030E52EA0335CD
:101D00004FEA013100F088804FEA03334FF08055ED
:101D100045EA131343EA12634FEA022245EA11151A
:101D200045EA10654FEA00260EF000419D4208BFCB
:101D3000964244F1FD0404F5407402D25B084FEA78
:101D40003202B61A65EB03055B084FEA32024FF424
:101D500080104FF4002CB6EB020E75EB030E22BF81
:101D6000B61A754640EA0C005B084FEA3202B6EB41
:101D7000020E75EB030E22BFB61A754640EA5C00F0
:101D80005B084FEA3202B6EB020E75EB030E22BF80
:101D9000B61A754640EA9C005B084FEA3202B6EB81
:101DA000020E75EB030E22BFB61A754640EADC0040
:101DB00055EA060E18D04FEA051545EA16754FEAA2
:101DC00006164FEAC30343EA52734FEAC2025FEAC0
:101DD0001C1CC0D111F4801F0BD141EA00014FF04F
:101DE00000004FF0004CB6E711F4801F04BF014320
:101DF0000020B4F1FD0C88BFBCF5E06F3FF6AFAE3C
:101E0000B5EB030C04BFB6EB020C5FEA500C50F1CB
:101E1000000041EB045170BD0EF0004E4EEA11314E
:101E200014EB5C04C2BFD4EB0C0541EA045170BD55
:101E300041F480114FF0000E013C90E645EA060E99
:101E40008DE60CEA135594EA0C0F08BF95EA0C0FC7
:101E50003FF43BAF94EA0C0F0AD150EA01347FF40F
:101E600034AF95EA0C0F7FF425AF104619462CE7E6
:101E700095EA0C0F06D152EA03353FF4FDAE104649
:101E8000194622E750EA410618BF52EA43067FF49A
:101E9000C5AE50EA41047FF40DAF52EA43057FF42A
:101EA000EBAE12E7000000000000000000000000A0
:101EB0004FF0FF3C06E000BF4FF0010C02E000BF16
:101EC0004FF0010C4DF804CD4FEA410C7FEA6C5CF9
:101ED0004FEA430C18BF7FEA6C5C1BD001B050EA9C
:101EE000410C0CBF52EA430C91EA030F02BF90EA87
:101EF000020F0020704710F1000F91EA030F58BF46
:101F0000994208BF90422CBFD8176FEAE37040F0A7
:101F1000010070474FEA410C7FEA6C5C02D150EA45
:101F2000013C07D14FEA430C7FEA6C5CD6D152EA00
:101F3000033CD3D05DF8040B704700BF84461046C5
:101F400062468C461946634600E000BF01B5FFF7C4
:101F5000B7FF002848BF10F1000F01BD4DF808ED94
:101F6000FFF7F4FF0CBF012000205DF808FB00BF65
:101F70004DF808EDFFF7EAFF34BF012000205DF8BF
:101F800008FB00BF4DF808EDFFF7E0FF94BF01200C
:101F900000205DF808FB00BF4DF808EDFFF7CEFF0D
:101FA00094BF012000205DF808FB00BF4DF808ED4C
:101FB000FFF7C4FF34BF012000205DF808FB00BF1D
:101FC0004FEA410212F5001215D211D56FF4787361
:101FD000B3EB625212D94FEAC12343F0004343EA04
:101FE000505311F0004F23FA02F018BF40427047DF
:101FF0004FF00000704750EA013005D111F0004069
:1020000008BF6FF0004070474FF00000704700BFFE
:102010004FEA4102B2F1E04324BFB3F5001CDCF10A
:10202000FE5C0DD901F0004C4FEAC0024CEA507042
:10203000B2F1004F40EB830008BF20F00100704771
:1020400011F0804F21D113F13872BCBF01F0004074
:10205000704741F480114FEA5252C2F11802C2F1A6
:10206000200C10FA0CF320FA02F018BF40F0010027
:102070004FEAC1234FEAD32303FA0CFC40EA0C00D9
:1020800023FA02F34FEA4303CCE77FEA625307D116
:1020900050EA01331EBF4FF0FE4040F4400070474D
:1020A00001F0004040F0FE4040F40000704700BFE7
:1020B00080F0004002E000BF81F0004142001FBFFD
:1020C0005FEA410392EA030F7FEA226C7FEA236C06
:1020D0006AD04FEA1262D2EB1363C1BFD2184140FB
:1020E00048404140B8BF5B42192B88BF704710F091
:1020F000004F40F4000020F07F4018BF404211F034
:10210000004F41F4000121F07F4118BF494292EA9B
:10211000030F3FD0A2F1010241FA03FC10EB0C00C7
:10212000C3F1200301FA03F100F0004302D5494254
:1021300060EB4000B0F5000F13D3B0F1807F06D301
:1021400040084FEA310102F10102FE2A51D2B1F1F9
:10215000004F40EBC25008BF20F0010040EA0300EE
:102160007047490040EB000010F4000FA2F101029B
:10217000EDD1B0FA80FCACF1080CB2EB0C0200FA25
:102180000CF0AABF00EBC25052421843BCBFD04073
:102190001843704792F0000F81F4000106BF80F4ED
:1021A00000000132013BB5E74FEA41037FEA226CB0
:1021B00018BF7FEA236C21D092EA030F04D092F07B
:1021C000000F08BF0846704790EA010F1CBF0020AF
:1021D000704712F07F4F04D1400028BF40F000400C
:1021E000704712F100723CBF00F50000704700F02C
:1021F000004343F0FE4040F4000070477FEA226253
:1022000016BF08467FEA23630146420206BF5FEA23
:10221000412390EA010F40F4800070474FF0000323
:1022200004E000BF10F0004348BF40425FEA000CEA
:1022300008BF704743F0964301464FF000001CE092
:1022400050EA010208BF70474FF000030AE000BFE8
:1022500050EA010208BF704711F0004302D5404226
:1022600061EB41015FEA010C02BF84460146002098
:1022700043F0B64308BFA3F18053A3F50003BCFAB3
:102280008CF2083AA3EBC25310DB01FA02FC634460
:1022900000FA02FCC2F12002BCF1004F20FA02F267
:1022A00043EB020008BF20F00100704702F120025A
:1022B00001FA02FCC2F1200250EA4C0021FA02F2BB
:1022C00043EB020008BF20EADC707047000000000A
:1022D0004FF0FF0C1CEAD0521EBF1CEAD15392EA09
:1022E0000C0F93EA0C0F6FD01A4480EA010C4002E5
:1022F00018BF5FEA41211ED04FF0006343EA50103F
:1023000043EA5111A0FB01310CF00040B1F5000F80
:102310003EBF490041EAD3715B0040EA010062F12F
:102320007F02FD2A1DD8B3F1004F40EBC25008BF19
:1023300020F00100704790F0000F0CF0004C08BF37
:1023400049024CEA502040EA51207F3AC2BFD2F104
:10235000FF0340EAC250704740F400004FF0000312
:10236000013A5DDC12F1190FDCBF00F0004070474C
:10237000C2F10002410021FA02F1C2F1200200FA8A
:1023800002FC5FEA310040F1000053EA4C0308BF51
:1023900020EADC70704792F0000F00F0004C02BFA2
:1023A000400010F4000F013AF9D040EA0C0093F01D
:1023B000000F01F0004C02BF490011F4000F013B77
:1023C000F9D041EA0C018FE70CEAD15392EA0C0FE5
:1023D00018BF93EA0C0F0AD030F0004C18BF31F050
:1023E000004CD8D180EA010000F00040704790F026
:1023F000000F17BF90F0004F084691F0000F91F0CA
:10240000004F14D092EA0C0F01D142020FD193EA8F
:102410000C0F03D14B0218BF084608D180EA010017
:1024200000F0004040F0FE4040F40000704740F0F3
:10243000FE4040F4400070474FF0FF0C1CEAD052C1
:102440001EBF1CEAD15392EA0C0F93EA0C0F69D01D
:10245000A2EB030280EA010C49024FEA402037D088
:102460004FF0805343EA111143EA10130CF000407F
:102470008B4238BF5B0042F17D024FF4000C8B426F
:1024800024BF5B1A40EA0C00B3EB510F24BFA3EB4F
:10249000510340EA5C00B3EB910F24BFA3EB91031F
:1024A00040EA9C00B3EBD10F24BFA3EBD10340EA79
:1024B000DC001B0118BF5FEA1C1CE0D1FD2A3FF6BF
:1024C00050AF8B4240EBC25008BF20F00100704774
:1024D0000CF0004C4CEA50207F32C2BFD2F1FF0317
:1024E00040EAC250704740F400004FF00003013A48
:1024F00037E792F0000F00F0004C02BF400010F4EC
:10250000000F013AF9D040EA0C0093F0000F01F0FF
:10251000004C02BF490011F4000F013BF9D041EA21
:102520000C0195E70CEAD15392EA0C0F08D1420254
:102530007FF47DAF93EA0C0F7FF470AF084676E727
:1025400093EA0C0F04D14B023FF44CAF08466EE700
:1025500030F0004C18BF31F0004CCAD130F00042CE
:102560007FF45CAF31F000437FF43CAF5FE700BF26
:102570004FF0FF3C06E000BF4FF0010C02E000BF4F
:102580004FF0010C4DF804CD4FEA40024FEA4103F1
:102590007FEA226C18BF7FEA236C11D001B052EAA7
:1025A000530C18BF90EA010F58BFB2EB030088BF6D
:1025B000C81738BF6FEAE17018BF40F001007047DC
:1025C0007FEA226C02D15FEA402C05D17FEA236CBE
:1025D000E4D15FEA412CE1D05DF8040B704700BF05
:1025E000844608466146FFE70FB5FFF7C9FF00289C
:1025F00048BF10F1000F0FBD4DF808EDFFF7F4FFD5
:102600000CBF012000205DF808FB00BF4DF808ED6D
:10261000FFF7EAFF34BF012000205DF808FB00BF90
:102620004DF808EDFFF7E0FF94BF012000205DF8B2
:1026300008FB00BF4DF808EDFFF7D2FF94BF012063
:1026400000205DF808FB00BF4DF808EDFFF7C8FF5C
:1026500034BF012000205DF808FB00BF000000002F
:102660004BB942B9002908BF002802D04FF0FF3112
:10267000084600F065B882B0EC462DE9005000F045
:1026800047F8DDF804E002B00CBC70470000000021
:1026900070B5FFF7A1F900230022C3F6F0530446FA
:1026A0000D46FFF7EDF900F053F80646FFF772F913
:1026B00000230022C4F2F013FFF7E2F902460B46B2
:1026C00020462946FFF728F800F042F8002231465C
:1026D00042EA0004204670BD000000000000000037
:1026E0002DE9F0471746804689469A46089E00F035
:1026F0004FF8A7FB004507FB01F700FB0A721544E2
:10270000B8EB040469EB0505C6E90045BDE8F087B0
:102710002DE9F8431746804689461D46089E00F07D
:10272000E7F900FB05F3A0FB074507FB01373D4434
:10273000B8EB040469EB0505C6E90045BDE8F8837C
:10274000704700BF00000000000000000000000013
:102750004A0011D212F5001211D20DD56FF4787320
:10276000B3EB62520ED44FEAC12343F0004343EA75
:10277000505323FA02F070474FF00000704750EAC0
:10278000013002D14FF0FF3070474FF0000070472A
:102790002DE9F04F444261EB410500294FF0FF362F
:1027A000A2BF04460D460026002B85B0C0F2C780AC
:1027B0002046AA469446194690462746A946002B2D
:1027C00058D1AA426CD9B2FA82F35BB1C3F12002AC
:1027D00005FA03F924FA02F20CFA03F842EA0909AD
:1027E00004FA03F74FEA1844484621461FFA88FACC
:1027F00000F0FEFA21468346484600F027FC3A0CDA
:102800000AFB0BF042EA014188420BD911EB0801A7
:102810000BF1FF3305D2884284BFABF1020B414478
:1028200000D89B46C0EB010921464846BFB200F0E4
:10283000DFFA21460546484600F008FC0AFB05FA87
:1028400047EA01418A4509D911EB080805F1FF3330
:1028500003D2C24588BF023D00D81D4645EA0B435E
:1028600000241846214616B1404261EB410105B0F3
:10287000BDE8F08FAB4284BF00242346F1D8B1FA03
:1028800081F5002D40F0B580514528BF82428CBFB4
:10289000002401249CBF01232C46E2D92346E0E713
:1028A00022B91146012000F0A3FA8046B8FA88F355
:1028B000002B49D1C8EB09094FEA18451FFA88FADD
:1028C00001242946484600F093FA294683464846A3
:1028D00000F0BCFB3A0C0AFB0BF042EA01418842D3
:1028E0000CD911EB08010BF1FF3380F0F280884224
:1028F00084BFABF1020B414440F2EB800A1A294637
:102900001046019200F074FA019A2946BFB281463E
:10291000104600F09BFB0AFB09FA47EA01418A4591
:102920000AD911EB080809F1FF3304D2C24588BF68
:10293000A9F1020900D8994649EA0B4391E7F64309
:10294000524263EB430333E708FA03F8C3F1200B69
:1029500029FA0BF409FA03F94FEA184520462946EB
:1029600027FA0BFB9F4000F043FA29461FFA88FA2A
:102970004BEA090B02462046019200F067FB019AE0
:102980004FEA1B430AFB02F043EA014188420BD99C
:1029900011EB080102F1FF3380F0A180884284BF6F
:1029A000023A414440F29B80C0EB01092946484667
:1029B000019200F01DFA29461FFA8BFB0446484697
:1029C00000F044FB019A0AFB04F94BEA01418945F6
:1029D0000AD911EB080104F1FF3304D2894584BF01
:1029E000023C414400D81C46C9EB010944EA0244B8
:1029F00067E7C5F12003A94022FA03F82AFA03FB8E
:102A000048EA010820FA03F30AFA05FA58464FEAA1
:102A1000184902FA05FC494643EA0A0ACDF80CC0F7
:102A200000F0E6F949460446584600F00FFB1FFA4D
:102A300088F24FEA1A4E02FB04F04EEA014E70454E
:102A400009D91EEB080E04F1FF3146D2704584BF50
:102A5000023CC64441D9C0EB0E0C49466046019287
:102A6000CDF808C000F0C4F9DDF808C049461FFAE7
:102A70008AFA8346604600F0E9FA019A02FB0BF2FB
:102A80004AEA01418A420AD911EB08010BF1FF30F1
:102A900021D28A4284BFABF1020B41441BD9039877
:102AA0004BEA044B891AABFB002399420DD314BFA8
:102AB0000023012307FA05F494422CBF002403F0FD
:102AC00001045B46002C3FF4CCAE0BF1FF33002435
:102AD000C7E69B4612E78346E1E70C46BBE71A468A
:102AE00062E700BF000000000000000000000000DE
:102AF0002DE9F04F064683B00D461446074688463A
:102B0000002B51D18A4264D9B2FA82F35BB1C3F18E
:102B1000200801FA03F520FA08F802FA03F448EA5B
:102B2000050800FA03F7250C404629461FFA84FAE7
:102B300000F05EF929468146404600F087FA3B0CDA
:102B40000AFB09F043EA014188420AD9091909F14F
:102B5000FF3205D2884284BFA9F10209091900D8C1
:102B60009146C0EB010829464046BFB200F040F94B
:102B700029460646404600F069FA0AFB06FA47EA8B
:102B800001418A4509D90C1906F1FF3380F01981FA
:102B9000A24588BF023E40F2148146EA0940002661
:102BA000314603B0BDE8F08F8B4284BF002630462B
:102BB000F6D8B3FA83F4002C5AD18B4228BFB24224
:102BC0008CBF002601269CBF01202646E8D930464E
:102BD000E6E722B91146012000F00AF90446B4FAEA
:102BE00084F3002B40F0A2802D1B4FEA14481FFAFB
:102BF00084FA01264146284600F0FAF8414681460B
:102C0000284600F023FA3B0C0AFB09F043EA014195
:102C100088420BD9091909F1FF3280F0D48088422B
:102C200084BFA9F10209091940F2CD80C0EB010B64
:102C300041465846BFB200F0DBF8414605465846CB
:102C400000F004FA0AFB05FA47EA01418A4509D96E
:102C50000C1905F1FF3380F0B880A24588BF023D12
:102C600040F2B38045EA0940314603B0BDE8F08F39
:102C7000C4F12001A34022FA01F825FA01F748EA3D
:102C80000308384626FA01F3A5404FEA1849A24046
:102C9000494601921D4300F0ABF849468346384649
:102CA00000F0D4F91FFA88F22F0C02FB0BF047EA70
:102CB0000147B84206D917EB08070BF1FF31C0F006
:102CC0008D808B463F1A49463846009200F090F8B6
:102CD0004946ADB28246384600F0B8F9009A02FB88
:102CE0000AF245EA01418A4205D911EB08010AF1CD
:102CF000FF306CD38246019D4AEA0B40891AA0FB43
:102D0000052399420CD306FA04F614BF00210121D1
:102D100096422CBF002601F00106002E3FF440AF82
:102D200000260138314603B0BDE8F08F9C40C3F166
:102D3000200925FA09FA06FA03F74FEA1448504623
:102D400041469D4000F054F8414626FA09F949EA07
:102D500005098346504600F079F91FFA84FA4FEAD4
:102D600019430AFB0BF043EA0141884209D90919CA
:102D70000BF1FF333AD2884284BFABF1020B091941
:102D800034D90D1A414628461FFA89F900F030F867
:102D900041460646284600F059F90AFB06F549EA7D
:102DA00001418D4209D9091906F1FF3304D28D4240
:102DB00084BF023E091900D81E464D1B46EA0B4649
:102DC00018E71E46E9E6914630E71D464AE78A4283
:102DD00084BFAAF1020A41448DD88BE7B84284BF70
:102DE000ABF1020B47443FF66DAF6AE79B46C8E77D
:102DF0004A1E08BF7047C0F02481884240F2168105
:102E0000114200F01781B0FA80F3B1FA81F2A2EB1F
:102E10000303C3F11F0304A202EB03134FF00002EC
:102E20009F4600BFAFF30080B0EBC17F00BF42EB15
:102E3000020228BFA0EBC170B0EB817F00BF42EB64
:102E4000020228BFA0EB8170B0EB417F00BF42EBD4
:102E5000020228BFA0EB4170B0EB017F00BF42EB44
:102E6000020228BFA0EB0170B0EBC16F00BF42EBC4
:102E7000020228BFA0EBC160B0EB816F00BF42EB44
:102E8000020228BFA0EB8160B0EB416F00BF42EBB4
:102E9000020228BFA0EB4160B0EB016F00BF42EB24
:102EA000020228BFA0EB0160B0EBC15F00BF42EBA4
:102EB000020228BFA0EBC150B0EB815F00BF42EB24
:102EC000020228BFA0EB8150B0EB415F00BF42EB94
:102ED000020228BFA0EB4150B0EB015F00BF42EB04
:102EE000020228BFA0EB0150B0EBC14F00BF42EB84
:102EF000020228BFA0EBC140B0EB814F00BF42EB04
:102F0000020228BFA0EB8140B0EB414F00BF42EB73
:102F1000020228BFA0EB4140B0EB014F00BF42EBE3
:102F2000020228BFA0EB0140B0EBC13F00BF42EB63
:102F3000020228BFA0EBC130B0EB813F00BF42EBE3
:102F4000020228BFA0EB8130B0EB413F00BF42EB53
:102F5000020228BFA0EB4130B0EB013F00BF42EBC3
:102F6000020228BFA0EB0130B0EBC12F00BF42EB43
:102F7000020228BFA0EBC120B0EB812F00BF42EBC3
:102F8000020228BFA0EB8120B0EB412F00BF42EB33
:102F9000020228BFA0EB4120B0EB012F00BF42EBA3
:102FA000020228BFA0EB0120B0EBC11F00BF42EB23
:102FB000020228BFA0EBC110B0EB811F00BF42EBA3
:102FC000020228BFA0EB8110B0EB411F00BF42EB13
:102FD000020228BFA0EB4110B0EB011F00BF42EB83
:102FE000020228BFA0EB0110B0EBC10F00BF42EB03
:102FF000020228BFA0EBC100B0EB810F00BF42EB83
:10300000020228BFA0EB8100B0EB410F00BF42EBF2
:10301000020228BFA0EB4100B0EB010F00BF42EB62
:10302000020228BFA0EB0100104670470CBF012030
:1030300000207047B1FA81F2C2F11F0220FA02F0BB
:10304000704708B14FF0FF30FFF77ABB0029F8D086
:103050002DE90340FFF7CCFEBDE8064002FB00F37C
:10306000A1EB0301704700BF00000000000000005A
:1030700041F20463C2F200031868704700000000C8
:103080000F2AF0B445D940EA01039B0745D1A2F1CC
:1030900010070C4603463F0900EB0716103625685B
:1030A0001033103443F8105C54F80C5C43F80C5C9B
:1030B00054F8085C43F8085C54F8045C43F8045C7A
:1030C000B342ECD17B1C02F00F0CBCF1030F4FEAB2
:1030D00003131944034422D90E461D46644656F88C
:1030E000047B043C032C45F8047BF8D8ACF10404C1
:1030F00002F0030224F0030404342344214432B1D7
:103100000A4411F8014B914203F8014BF9D1F0BC8C
:1031100070470346002AF3D1F9E70346F0E7624619
:10312000002AEDD1F3E700BF00000000000000001E
:103130008307F0B448D0541E002A43D0CDB20346D2
:1031400002E0002C3ED0144603F8015B13F0030F9D
:1031500004F1FF32F5D1032C2DD9CDB20F2C45EA65
:10316000052545EA054518D9A4F1100703F1100615
:103170001A463F0906EB07161560103242F80C5C40
:1031800042F8085C42F8045CB242F5D104F00F0446
:103190000137032C03EB07130DD91E462246043AD0
:1031A00046F8045B032AFAD8221F04F0030422F035
:1031B0000302043213442CB1C9B21C4403F8011BAE
:1031C000A342FBD1F0BC704714460346C3E700BFDF
:1031D000C9B2F0B4002947D084070FD00278002A82
:1031E0003FD091423ED0431C05E013F8012B002A4A
:1031F00037D0914236D09A071846F6D141EA0127D6
:10320000036847EA0747A3F1013483EA070224EA87
:103210000303A2F1013424EA0202134313F0803FB6
:1032200011D1021D104652F8043B83EA0704A3F1B2
:103230000136A4F1013526EA030325EA04042343F9
:1032400013F0803FEED00378002B3BD0994209D099
:10325000431C01E0914205D0184613F8012B002AC7
:10326000F8D11046F0BC704781070DD00378002BD1
:10327000F8D0431C02E00278002AF3D013F0030FC9
:10328000184603F10103F6D10368A3F1013222EAE3
:10329000030313F0803F0AD1031D184653F8042B93
:1032A000A2F1013121EA020212F0803FF5D0037849
:1032B000002BD7D0431C184601330278002AFAD1DC
:1032C000F0BC70471846CDE7000000000000000089
:1032D00080EA0102844612F0030F4FD111F0030F70
:1032E00032D14DF8044D11F0040F51F8043B0BD0CE
:1032F000A3F101329A4312F0803F04BF4CF8043B23
:1033000051F8043B16D100BF51F8044BA3F1013230
:103310009A4312F0803FA4F101320BD14CF8043BE8
:10332000A24312F0803F04BF51F8043B4CF8044B19
:10333000EAD023460CF8013B13F0FF0F4FEA33238A
:10334000F8D15DF8044B704711F0010F06D011F869
:10335000012B0CF8012B002A08BF704711F0020F57
:10336000BFD031F8022B12F0FF0F16BF2CF8022B42
:103370008CF8002012F47F4FB3D1704711F8012B65
:103380000CF8012B002AF9D1704700BF00000000A3
:1033900020F0030110F00300C0F1000051F8043BDD
:1033A00000F1040C4FEACC0C6FF000021CBF22FAB3
:1033B0000CF213434FF0010C4CEA0C2C4CEA0C4C71
:1033C000A3EB0C0222EA030212EACC1204BF51F86A
:1033D000043B0430F4D013F0FF0F1FBF013013F48F
:1033E0007F4F013013F47F0F18BF0130704700BFCB
:1033F000F0B4002A4BD040EA010313F003032DD1AF
:10340000032A2BD904680D68AC4227D1043A3ED078
:10341000A4F1013525EA040414F0803F3DD10C46A7
:1034200005460EE06B68054666680C46A3F1013759
:10343000B34227EA030711D1043A28D017F0803F9E
:1034400028D1032A00F1040001F10401EAD8561E34
:103450002AB928792279801AF0BC7047561E037861
:103460000A7893421BD1E6B1BBB101368B1C0446EE
:10347000314405E08B4203F101030BD00028EBD06F
:1034800014F8010F13F8012C9042F3D0E3E7104633
:10349000F0BC70470020F0BC70471846DCE71846C7
:1034A000D9E73046D8E700BF000000000000000068
:1034B00040EA01039B0770B42BD1032A84BF0B465B
:1034C000054626D9194653F8044BA4F1013626EADD
:1034D000040616F0803F05D1043A45F8044B032A50
:1034E0001946EFD89AB10C78013A6B1C2C703CB19C
:1034F0006AB111F8014F013A03F8014B002CF7D1E2
:103500002AB11A44002103F8011B9342FBD170BC7D
:1035100070470546E6E700BF00000000000000001D
:1035200038B502460C46002511B909E0421C054693
:1035300010462146FFF74CFE0028F7D1284638BD3B
:10354000BDE83840FFF744BE000000000000000066
:103550004FF0010C2DE9F003644600254FF0FF36D3
:10356000631987198B420DD23F5D10F80380B8456F
:103570002FD21D460124C6EB030C63198B4200EBCE
:103580000607F1D34FF0010900254C464FF0FF37F5
:10359000C2F800C0631900EB070C99420ED91CF861
:1035A00004C010F80380E0451AD91D460124C7EB7A
:1035B00003096319994200EB070CF0D80137013673
:1035C000B74226BFC2F8009038463046BDE8F00347
:1035D00070470CD04FF0010C2E4664466544BFE79F
:1035E0000CD04FF001092F464C464D44D2E76445BC
:1035F00004F10104B4D11D460124B1E74C4504F1A6
:103600000104C7D11D460124C4E700BF2DE9F04FD6
:10361000ADF2244D164680460D461046194607AABF
:103620001C46FFF795FF07AB0DF21C42039043F8D1
:10363000044F9342FBD1671E002308A834B1F25C0B
:10364000F91A0133A34240F82210F8D10799304605
:10365000039A314400F04CFA002840F08180DDF8F4
:103660000CC02A468246671E0CF1FF3CCDF808C00C
:10367000B444CDF810C0DDF80CC005460196CCF17D
:10368000010CCDF814C008E025B1079A934238BF69
:10369000C2EB04039A44002532460AEB040608EB09
:1036A00002000021B21A00F0DBF9002853D1002EED
:1036B00051D008EB060308A913F8013C51F8233058
:1036C000002BE1D1039A954228BF2A46BA4212D272
:1036D000019908EB0A03985C11F802C01144844573
:1036E00006D032E011F8010F13F802C084452CD146
:1036F0000132BA42F6D3039B02989D4228BF184676
:103700001CD2DDF810C008EB0A039CF80010DDF8AD
:1037100008C013F80C20914240F08680DDF804B018
:10372000049AAB4406E012F8019D13F801C0E1458C
:1037300004D108465A4500F1FF31F4D101358542E4
:1037400074D8079DAA44651BA6E7DDF814C00025C0
:10375000E2449244A0E700200DF2244DBDE8F08F32
:10376000DDF80CC02A46DDF80CA04FF0000BCCEBC6
:1037700004030DF12009634538BF6346671E01331A
:10378000254607930CF1FF33B444CDF808C0DDF8AB
:103790000CC00193CCF1010CCDF810C00BEB05046B
:1037A00008EB02000021A21A00F05AF90028D2D139
:1037B000002CD0D008EB040313F8013C59F8233057
:1037C00053BBBA4508EB0B0013D2029B1A7810F8D2
:1037D0000A309A4218BF534621D1029A534605E057
:1037E00012F8011F10F803C08C4518D10133BB42F9
:1037F000F6D3019B5A1CAFD0DDF804C016F80C10AC
:1038000010F80C20914206D113F1FF33A4D3F15CE0
:10381000C25C9142F8D0079B9B442246BEE7DDF88C
:1038200010C0E3449B44F8E7039887E708EB0A00DD
:1038300092E700BF2DE9F04F8046037887B00E462F
:10384000002B00F001810A789AB1844601310124ED
:1038500002E011F8012B5AB1934214BF002404F086
:1038600001041CF8013F0D46002BF2D12B7813BB4D
:103870001CB1404607B0BDE8F08F08F10100317877
:10388000FFF7A6FCAD1B012D18BF0028074608BF97
:103890000046EFD0A844474594BFC7EB0804012475
:1038A0001F2D0CD93846214632462B46FFF7AEFE77
:1038B00007B0BDE8F08F002007B0BDE8F08F2946C3
:1038C00005AA3046FFF744FE0599314400900246B0
:1038D000304600F00DF9002857D1009B8346804602
:1038E0002246013B019333440293009BC3F1010341
:1038F000039308EB0504B8180021A21A00F0B0F8F1
:103900000028D8D1002CD6D0009B9B4528BF5B4611
:103910009D4214D9F918F05CF21811F80810884289
:1039200040F08C8007EB080C06E012F8011F1CF831
:103930000300884240F0828001339D42F5D8009B0D
:1039400001995B4540F28380029B07EB08091A78D6
:1039500019F801309A427AD1029B06EB0B0A06E075
:1039600013F801CD19F80200844504D111465345DE
:1039700001F1FF32F4D10BF1010B8B4569D8059BA6
:103980009844C3EB050B2246B3E700984FF0000BB9
:1039900022462B1A8146834238BF0346B144013385
:1039A0000593009B38440190C3F101030293009BEF
:1039B00003F1FF389A460BEB0504B8180021A21A50
:1039C00000F04EF800287FF476AF002C3FF473AF80
:1039D000554598BF07EB0B0014D9019899F80020C2
:1039E00010F80B309A4224D14A46534607EB0B009D
:1039F00005E012F8011F10F803C08C451AD10133FD
:103A00009D42F6D8B8F1FF3F43463FF433AF16F876
:103A1000081010F80820914207D113F1FF33FFF48A
:103A200029AFF15CC25C9142F7D0059B9B442246D2
:103A3000C1E75346029A93449B44F8E703994FF039
:103A4000000B884498449EE70D4601240EE7009938
:103A500091E707EB08000DE7000000000000000000
:103A60008307C9B270B43FD0541E2AB303788B4287
:103A700023D0431C04E0FCB1057814468D421CD0D1
:103A800013F0030F184604F1FF3203F10103F2D1E2
:103A9000032C14D8651E4CB303788B420DD0421C06
:103AA000002302E004788C4207D0AB42104603F1B9
:103AB000010302F10102F5D1002070BC704741EA18
:103AC0000126034646EA0646184604330268724059
:103AD000A2F1013525EA020212F0803FDAD1043C5E
:103AE0001846032CF0D8D5E71446D1E72046E4E782
:103AF000032A70B412D940EA01039B070FD10C4688
:103B0000034621461846043404330D680668AE4265
:103B100004D1043A1846032A2146F2D8C2B10578E6
:103B20000C78A54204BF02F1FF32002306D00CE05E
:103B300010F8015F11F8014FA54206D1934203F13D
:103B40000103F5D1002070BC7047281B70BC704782
:103B50001046F8E700000000000000000000000030
:103B6000704700BFAFF30080AFF30080AFF3008079
:103B7000FEE700BFAFF30080AFF30080AFF300803B
:103B800072B641F20060C2F2000080F309884EF67E
:103B90003472CEF200024EF68853CEF200034FF09C
:103BA000404111601A6842F470021A600023E1EE8D
:103BB000103A4EF63C73CEF2000300221A60062340
:103BC00083F31488BFF36F8F40F2000341F20002C9
:103BD000C2F20003C2F2000293420BD2D943114455
:103BE00021F0030119444FF05532043B43F8042FF0
:103BF0008B42FBD141F20003C2F2000383420CD29C
:103C000037491A1D891A21F0030119444FF0553222
:103C1000043B43F8042F8B42FBD108F079FB41F2BF
:103C2000006141F63C13C2F20001C2F20003994266
:103C30000ED2CC431C4424F0030444F280300434FC
:103C4000C0F603000023C258CA500433A342FAD17D
:103C500041F640134AF27812C2F20003C2F20102A6
:103C600093420AD2D943114421F00301194400229E
:103C7000043B43F8042F8B42FBD1FFF771FF40F266
:103C8000AC1540F24823C0F60005C0F600039D4283
:103C90000BD2EE431E44B6080136043D0024013425
:103CA00055F8043F9847B442F9D1FDF731FA40F294
:103CB000482540F24823C0F60005C0F600039D42A7
:103CC0000BD2EE431E44B6080136043D00240134F5
:103CD00055F8043F9847B442F9D1FFF749FF00BFB8
:103CE00003160020AFF30080AFF30080AFF3008035
:103CF000FEE700BFAFF30080AFF30080AFF30080BA
:103D000072B6FEE7AFF30080AFF30080AFF3008040
:103D100000F0DEF900F02CFD00F0FAF900DF00BF42
:103D20004EF63073CEF200035A6822F001025A6058
:103D3000EFF30983683383F30988002383F3118841
:103D4000704700BFAFF30080AFF30080AFF3008097
:103D500008B54FF46D43CEF200034FF44072C0F249
:103D6000FA52002199600720DA60102100F0E0F893
:103D70000A20202100F0DCF80B206021BDE808407B
:103D800000F0D6B8AFF30080AFF30080AFF300804F
:103D9000202383F311884FF46D43CEF200035B6858
:103DA00013F4006329D0F1EE10FAEFF309834EF615
:103DB0003072CEF200024FF08071D26843F84C1C92
:103DC00043F8082CA3F1680282F3098840F2A85254
:103DD000C1F20002916991F8220088B110688A68E6
:103DE0008168914294BF0022012292B143F61152A0
:103DF000C0F6000243F8502C704783F311887047D7
:103E000010688A688168914234BF00220122002A2A
:103E1000ECD143F61C52C0F6000243F8502C704718
:103E200008B500F0DDF9202383F3118800F090F944
:103E300000F0EEF800F0ACF9002383F3118800F0F5
:103E4000FFF9BDE80840FFF7A3BF00BFAFF3008054
:103E50002DE9F04F2DED108AC1F80CD0D0F80CD020
:103E6000BDEC108ABDE8F08FAFF30080AFF30080A7
:103E700008B500F04DF9002383F311882846A047C8
:103E800000F08EFD08BD00BFAFF30080AFF30080EF
:103E900020F0030303F1604303F56143F0B400F045
:103EA00003024409D3F80053D200FF26A400964031
:103EB00004F1604404F5614425EA060501279140B8
:103EC00000F01F0007FA00F045EA0102C3F80023E2
:103ED000C4F880012060F0BC704700BFAFF30080E1
:103EE00041094FF4614230B4203100F01F04012534
:103EF000CEF2000220F0030305FA04F403F160435C
:103F000042F8214003F5614300F00300D3F8002399
:103F1000C000FF2101FA00F022EA0000C3F800030C
:103F200030BC7047AFF30080AFF30080AFF3008088
:103F300020F0030303F1604303F56D4300F0030039
:103F400010B4C0009A69FF24844022EA0402814030
:103F50000A439A615DF8044B704700BFAFF30080DD
:103F600040F2A852C1F2000248F680739269C0F68E
:103F700002039361FEE700BFAFF30080AFF3008060
:103F800010B582B0FFF7E4FE00F07AFA00F000FA14
:103F900001F03EF901F08CF900F0BAF940F20000AE
:103FA0004021C1F2000000F0F3FB41F2000240F2B8
:103FB000A8530121C2F20002C1F2000380F82010D0
:103FC000C261986100F064F8002383F3118862B63F
:103FD00040F2A853C1F2000349F260129C69C0F696
:103FE0000202002140F2500043F66173A261C0F664
:103FF0000003009101224FF4AB61C1F2000000F018
:1040000057FC02B010BD00BFAFF30080AFF30080DB
:10401000F8B500F03DF940F2A853C1F200039A69E7
:1040200092F8223013B1013B82F82230516A40F2FB
:10403000C453C1F2000301315162DA681C680132D5
:104040009C42DA601DD0A768013FA760CFB91E4629
:104050002268E568E76053601A6000F099F8002371
:1040600083F311882069A847202383F3118800F087
:104070006FF83468A26840F2C453C1F20003002A0A
:10408000E6D0F8BDAFF30080AFF30080AFF300805F
:1040900041F64013C2F200031B682BB941F64C53A2
:1040A000C2F200031B685BB148F6C07048F6987115
:1040B000C0F60200C0F602014FF48C721EF0E8BB9D
:1040C000704700BFAFF30080AFF30080AFF3008014
:1040D00041F64013C2F2000310B51B6841F64C5480
:1040E000C2F200040BB923685BB148F6C87048F609
:1040F0009871C0F60200C0F602014FF48C721EF0F7
:10410000C7FB0123236010BDAFF30080AFF3008035
:1041100041F64013C2F2000310B51B6841F64C543F
:10412000C2F200042BB92368002B02DD00232360B8
:1041300010BD48F6E47048F69871C0F60200C0F66B
:1041400002014FF48C721EF0A3FB0023236010BD0C
:1041500041F64013C2F2000310B51B6841F64C54FF
:10416000002BC2F2000401DD23685BB148F6EC705D
:1041700048F69871C0F60200C0F602014FF48C7246
:104180001EF086FB0123236010BD00BFAFF300804B
:1041900041F64013C2F2000310B51B6841F64C54BF
:1041A000002BC2F2000405DD2368002B02DD002392
:1041B000236010BD49F20C0048F69871C0F6020069
:1041C000C0F602014FF48C721EF062FB00232360E4
:1041D00010BD00BFAFF30080AFF30080AFF30080ED
:1041E00010B5202383F3118841F64014C2F2000475
:1041F0002268002A05DB41F64C53C2F200031B681B
:1042000063B149F2140048F698714FF48C72C0F60D
:104210000200C0F602011EF03BFB226848F2AC33FC
:10422000C2F200030132196822608A42C8BF1A60D4
:10423000002383F3118810BDAFF30080AFF300803B
:1042400010B5202383F3118841F64014C2F2000414
:104250002268002A05DD41F64C53C2F200031B68B8
:1042600063B149F21C0048F698714FF48C72C0F6A5
:104270000200C0F602011EF00BFB2268013A226028
:10428000002383F3118810BDAFF30080AFF30080EB
:1042900041F64013C2F200031B68002B07DB41F616
:1042A0004C53C2F200031B68002B00DD704749F23B
:1042B000240048F69871C0F60200C0F602014FF4DF
:1042C0008C721EF0E5BA00BFAFF30080AFF3008040
:1042D00041F64013C2F200031B683BB941F64C5350
:1042E000C2F200031B68002B00DD704749F2480052
:1042F00048F69871C0F60200C0F602014FF48C72C5
:104300001EF0C6BAAFF30080AFF30080AFF30080B9
:1043100041F64413C2F200031A46402142F8081B3A
:104320005A607047AFF30080AFF30080AFF30080B6
:1043300010B441F6441340F2C45440F2A851C2F202
:104340000003C1F20004C1F200015A68E4688969FF
:1043500014605160816A916090F8204002F1100170
:1043600003F58160814214732ABF03F1080259608A
:104370005A605DF8044B7047AFF30080AFF30080E4
:1043800048F69871C0F602014FF48C721EF080BAA4
:1043900040F2C453C1F200034FF0FF3100225B60D2
:1043A0001B609960DA607047AFF30080AFF3008064
:1043B000F8B5054616460C461F46FFF769FF002E66
:1043C00018BF002D1CD0DCB140F2C451C1F2000175
:1043D0002F610B68EE609A68944204D91B68A41A96
:1043E0009A68A242FAD35A682B606A608B425D6079
:1043F0001560AC601EBF9A68C4EB02049C60F8BDF7
:1044000049F2500049F26001C0F60200C0F6020114
:1044100051221EF03DFAD7E7AFF30080AFF30080E2
:1044200010B50446FFF734FF9CB1E368EBB1236895
:1044300040F2C452C1F2000293421FBF9968A268C1
:1044400052189A6062681360236800215A60E16024
:1044500010BD49F2800049F26001C0F60200C0F6CA
:1044600002016D221EF014FADFE749F29000C0F657
:104470000200FFF785FFDAE7AFF30080AFF30080BB
:1044800040F2A853C1F2000300225B601B605B6135
:104490001B619A60704700BFAFF30080AFF30080EC
:1044A00010B50446FFF7F4FE94F82030002B18BF37
:1044B0000E2B12D0002240F2A853A16884F82020CD
:1044C000C1F200031B689A688A42FBD25A682360D3
:1044D000626020465C60146010BD49F2B000C0F616
:1044E0000200FFF74DFFE5E7AFF30080AFF3008078
:1044F00038B50446202383F31188FFF729FE94F88A
:104500002050032D0ED00D2D10D0ADB14FF0FF3344
:10451000A3622046FFF7C4FFFFF73AFE002383F3B0
:10452000118838BDA36A9A6801329A6094E80C0039
:104530001A6022685360E9E7FFF72AFE2B4683F3EF
:10454000118838BDAFF30080AFF30080AFF3008077
:1045500070B540F2A854C1F200040646FFF7B8FE59
:104560002368A5691A6885F820600121142085F860
:1045700022005460284683F820102260A361FFF7D0
:10458000D7FE284617F05CFF002805DBA069294606
:10459000BDE87040FFF75CBC284624F0F1FBA06941
:1045A0002946BDE87040FFF753BC00BFAFF3008061
:1045B00070B50D4686B00646FFF78AFE6B1C18D014
:1045C00040F2A854C1F2000444F2F142A369294622
:1045D00001A8C0F60002FFF7EBFE3046FFF7B8FF78
:1045E000049B13B101A8FFF71BFFA369986A06B0EB
:1045F00070BD40F2A854C1F200043046FFF7A8FF96
:10460000A369986A06B070BDAFF30080AFF3008075
:1046100070B540F2A855C1F2000504460E46FFF7FA
:1046200057FEA869A3688268A662934213D9FFF770
:1046300037FF0123064684F82030AC61FFF778FE8F
:10464000304617F0FDFE00280ADB20463146BDE863
:104650007040FFF7FDBB2046BDE87040FFF720BF6C
:10466000304624F08DFBF0E7AFF30080AFF300801D
:1046700070B540F2A854C1F2000414212368A56962
:104680001A6801265460284683F8206085F82210B5
:104690002260A361FFF704FF2846FFF749FE284682
:1046A00017F0CEFE002805DBA0692946BDE8704062
:1046B000FFF7CEBB284624F063FBA0692946BDE87E
:1046C0007040FFF7C5BB00BFAFF30080AFF30080C1
:1046D00070B540F2A856C1F2000601203268B569F3
:1046E0001368AC68336000215E6082F820001346D6
:1046F000B26185F8201000E01B689A68A242FBD8DE
:104700005A682B606A6028465D601560FFF710FEEE
:10471000284617F095FE002805DBB0692946BDE85C
:104720007040FFF795BB284624F02AFBB069294664
:10473000BDE87040FFF78CBBAFF30080AFF30080A3
:1047400008B5FFF7C5FD40F2A853C1F200031A688F
:104750009B6992689B689A4200D808BDBDE80840F2
:10476000FFF7B6BFAFF30080AFF30080AFF3008078
:1047700040F2A853C1F200039B6993F822300BB1B9
:10478000FFF7A6BFFFF774BFAFF30080AFF3008061
:104790002DE9F00140F2A852C1F20002002455694F
:1047A00080F8214000F12C064FF0020800F14C0780
:1047B0004FF0140C45610261816080F82080C46371
:1047C0008463446284610164506180F822C028617E
:1047D000C7610663C662BDE8F0017047AFF30080B1
:1047E000884203D200F8012B8842FBD1704700BFFA
:1047F0002DE9F84F99460D4604469046FFF748FDCF
:10480000B5F5AC7F2CBF00230123002C08BF43F07B
:1048100001034BB9D9F1010338BF0023B8F17F0F71
:1048200088BF43F0010353B149F2D00049F2E401DB
:10483000C0F60200C0F60201A6221EF029F840F2DE
:10484000A856C1F20006A5F1640121440A9F7369CC
:10485000E16043F671600025C0F600004FF0020BE6
:104860004FF0140A0866C1F840904F6404F12C021E
:1048700004F14C0C84F820B084F8215084F822A074
:10488000C4F8088026616361C4F840807461E56300
:10489000A5636562A56120461C612263E262C4F8DB
:1048A0001CC0BDE8F88F00BFAFF30080AFF30080FD
:1048B0002DE9F04F83B080460C9F894693469A4677
:1048C00000F14C050446FF2604F8016BA542FBD11C
:1048D00008EB0904A54204D2552605F8016BA54250
:1048E000FBD1202383F31188FFF7F2FB53465A468E
:1048F000494600974046FFF77BFF00210446FFF73B
:1049000087FEFFF705FC002383F31188204603B0E0
:10491000BDE8F08FAFF30080AFF30080AFF300800D
:1049200010B5044658B949F2341049F2E401C0F612
:104930000200C0F602014FF493721DF0A9FF20237C
:1049400083F31188FFF7C4FB21460620FFF730FEF2
:10495000FFF7DEFB002383F3118810BDAFF3008067
:1049600008B540F2A853C1F200039B6993F82120D7
:104970009862920701BF5A69196911611B694FF06A
:104980000E0008BF5A61FFF7E3FD49F24410C0F67C
:104990000200BDE80840FFF7F3BC00BFAFF30080A2
:1049A00010B52023044683F31188FFF791FB2046BE
:1049B000BDE81040FFF7D4BFAFF30080AFF3008035
:1049C00010B5202383F31188FFF782FB40F2A85330
:1049D000C1F200031C69FFF79BFB002383F31188DE
:1049E000204610BDAFF30080AFF30080AFF300802E
:1049F00010B52023044683F31188FFF769FB24696F
:104A000040F2A853C1F200039C4208BF0024FFF704
:104A10007FFB002383F31188204610BDAFF3008095
:104A200038B5D0F1010338BF002353EAD1730446EF
:104A30000D460AD049F2801049F29011C0F60200EA
:104A4000C0F6020158221DF023FF64602460A560B7
:104A500038BD00BFAFF30080AFF30080AFF300803C
:104A600038B504460D46FFF733FC5CB3A3682268F3
:104A7000002B0EDBA2420ED049F21020C0F602003D
:104A8000FFF77EFCA268531E002BA36008DB00200A
:104A900038BDA242F0D01A46531E002BA360F6DAAE
:104AA000E5B140F2A853C1F2000329469B699C621C
:104AB00062681C605A60032063601360BDE8384080
:104AC000FFF776BD49F2F81049F29011C0F60200E6
:104AD000C0F60201FD221DF0DBFEC7E7A2604FF029
:104AE000FF3038BDAFF30080AFF30080AFF300803C
:104AF00010B50446FFF7CCFB14B3A3682268002B63
:104B00000DDBA24206D049F26020C0F60200FFF79A
:104B100037FCA3680133002BA36006DD10BDA24261
:104B2000F1D00133002BA360F8DC23681A68002160
:104B30002260546099621846BDE81040FFF7B0BC8F
:104B400049F24C2049F29011C0F60200C0F6020171
:104B50004FF499721DF09CFECFE700BFAFF30080C9
:104B600010B5044620B1002364602460A36010BD2A
:104B700049F2B02049F2C021C0F60200C0F602019D
:104B800058221DF085FEEEE7AFF30080AFF3008002
:104B9000F8B540F2A853C1F2000305469C69FFF73F
:104BA00097FB002D5BD0A868002848D0A1688368D7
:104BB0008B421ED290F820308160002B44D0042B11
:104BC00017D103684268866A1360076833467A60C3
:104BD00002E09A688A4202D31B689E42F9D15A6861
:104BE0000360426058601060B068A16883688B42BF
:104BF000E0D32B4603E09968A268914202D31B6878
:104C00009D42F8D15A682360626004205C601460A1
:104C1000A562FFF79DFCAB68A34205D049F2F020E6
:104C2000C0F60200FFF7ACFBE36BAB420BD049F2DE
:104C30000430C0F60200BDE8F840FFF7A1BBE36B0B
:104C4000AC60EB60E563F8BD90E80C00012180F8F2
:104C500020101A6002685360FFF722FCC9E749F28E
:104C6000E02049F2C021C0F60200C0F602017D2218
:104C70001DF00EFE97E700BFAFF30080AFF300809A
:104C800010B52023044683F31188FFF721FA20464C
:104C9000FFF77EFFFFF73CFA002383F3118810BD76
:104CA00040F2A852C1F2000270B52023956983F347
:104CB0001188FFF70DFAEC6B002C30D0A368AB42E3
:104CC00006D049F24030C0F60200FFF759FBEC6B0A
:104CD0002668E368A642EB631ED0296C4BB11A68C4
:104CE0009A4203D09268914238BF1146DB68002B8C
:104CF000F5D1F26B3368A9603046236000215C6017
:104D0000A660E260F463FFF783FCFFF701FA00237B
:104D100083F31188204670BD0023A360F5E749F2B4
:104D20002C30C0F60200FFF72BFBEC6BC6E700BF90
:104D3000002918BF0028F8B505460C4617460AD1C9
:104D400049F2803049F29831C0F60200C0F6020103
:104D500057221DF09DFD202383F31188FFF7B8F93A
:104D600040F2A853C1F200032A689B692260002622
:104D70002C606360A760E660FFF7CAF9334683F3EF
:104D80001188F8BDAFF30080AFF30080AFF300806F
:104D900038B504460D46FFF77BFAC4B1A26B94F810
:104DA000203045EA0201082BA1630CD0092B00D06A
:104DB00038BDA36A19408B42FAD12046FFF770FB39
:104DC0000023836238BDA36A1942F6D138BD49F287
:104DD000D03049F29831C0F60200C0F60201FE223E
:104DE0001DF056FDDAE700BFAFF30080AFF300809F
:104DF00070B505460E46FFF74BFA65B12C68A54223
:104E000008D0201D0BC83343E360FFF7C1FF2468BF
:104E1000A542F6D170BD49F2E43049F29831C0F6AE
:104E20000200C0F60201BC221DF032FDE6E700BF21
:104E300003460022C068DA60704700BFAFF300800D
:104E400010B4024679B140F2A853C1F200030D201C
:104E50009B699A62546883E81400536023605DF88C
:104E6000044BFFF7A5BB4FF0FF305DF8044B7047D4
:104E700030B4029C406000250A44856004620261EF
:104E8000006041618161C160C36130BC704700BF97
:104E900038B50446FFF7FCF92068E3680022A04219
:104EA0006361A260A3610AD06FF00105036823600B
:104EB0005C60FFF7F5FA85622068A042F6D138BD44
:104EC00038B504460D46FFF7E3F96369A269A168A6
:104ED00093421BD05A1C01316261A1601D7062694E
:104EE00023699A420BD22068A0420DD00368236048
:104EF0005C60FFF7D5FA00238362184638BD20684E
:104F0000E368A0426361F1D1002038BD0029E1D0FF
:104F10006FF0030038BD00BFAFF30080AFF3008037
:104F2000F8B504460E46202383F31188FFF7D0F826
:104F3000E36933B12046984703E0FFF781FF071E7E
:104F400018DBA56820463146002DF6D0A2692169FC
:104F5000531C8B42A36105F1FF3528BFE368A560B0
:104F6000177828BFA361FFF7D3F8002383F31188D4
:104F70003846F8BDFFF7CCF82B4683F31188384646
:104F8000F8BD00BFAFF30080AFF30080AFF3008047
:104F90002DE9F047044615460F461E46D0F81C8002
:104FA000002A3DD0202383F31188FFF791F807EB07
:104FB000050A4FF000090137B8F1000F05D020466F
:104FC000C04702E0FFF73CFF10BBA5682046314612
:104FD000002DF7D0A369013D5A1CA261A5601B7882
:104FE00007F8013C2369A2699A4224BFE368A361E0
:104FF000FFF78EF8002383F31188574509F1010963
:105000000BD0202383F31188FFF762F80137D3E731
:10501000FFF77EF82B4683F311884846BDE8F087FA
:1050200049F2404049F25441C0F60200C0F6020184
:10503000E7221DF02DFCB5E7AFF30080AFF3008051
:1050400030B4029C40608D1805610462006082608B
:1050500041618161C160C36130BC7047AFF30080C2
:1050600038B50446FFF714F9E368226920686361E4
:10507000D21AA042A361A2600AD06FF001050368B2
:1050800023605C60FFF70CFA85622068A042F6D1CD
:1050900038BD00BFAFF30080AFF30080AFF30080F6
:1050A0002DE9F041202304468846164683F31188F3
:1050B000FFF70EF803E0FFF7C3FE071E1DDBA56830
:1050C00020463146002DF6D06369013D5A1C6261CD
:1050D000A56083F80080236962699A4224BFE3686F
:1050E0006361E3690BB120469847FFF711F800238D
:1050F00083F311880020BDE8F081FFF709F82B4603
:1051000083F311883846BDE8F08100BFAFF300801B
:1051100038B50446FFF7BCF8A3696269A0689A42F3
:1051200016D021695A1C0130A060A2618A421D7804
:105130000BD22068A04206D0036823605C60FFF7B2
:10514000AFF900238362284638BDE368A361F0E726
:105150000028E6D06FF0020038BD00BFAFF300803A
:105160002DE9F84F044617460E469B46D0F81CA082
:10517000002A3AD0202383F31188FEF7A9FF4FF0CD
:105180000009A56806F1010820466A1EFDB16369A1
:10519000A2605A1C626132781A70236962699A426D
:1051A00024BFE3686361BAF1000F00D0D047FEF777
:1051B000AFFF002383F31188013F09F1010911D0EA
:1051C000202383F31188FEF783FF4646D9E7204664
:1051D0005946FFF735FE0028D3D0FEF799FF2B463E
:1051E00083F311884846BDE8F88F49F2784049F2C8
:1051F0005441C0F60200C0F6020140F29B121DF0BD
:1052000047FBB7E7AFF30080AFF30080AFF3008058
:105210004CF2000140F2D45240F2D8530648C2F298
:105220000101C1F20002C1F2000321F0070120F0E8
:1052300007001160186070477FA10120AFF3008064
:1052400010B50446FFF724F840F2D85340F2D45288
:10525000C1F20003C1F2000219681268E01D20F0DB
:105260000700521A90429DBF40181860084600205F
:1052700010BD00BFAFF30080AFF30080AFF300803C
:1052800010B52023044683F31188FEF721FF204642
:10529000FFF7D6FF0446FEF73BFF002383F3118898
:1052A000204610BDAFF30080AFF30080AFF3008065
:1052B00040F2E053C1F2000345F281220021C0F622
:1052C000000203F110001A609960D960FFF748BC32
:1052D000F8B540F2E056C1F20006002818BF0646B5
:1052E000073106F1100021F0070506F10804FFF769
:1052F000C7FC03E05A68954211D91C462368002B6D
:10530000F8D1FFF7CDFC33681BB305F108009847CF
:10531000F8B10660456000F108042046F8BD05F1CB
:105320000801914208D91A6822601C4644F8086BAB
:10533000FFF7B6FC2046F8BD4FF6F870CFF6FF70C9
:10534000401B5F180244186858507A6027605D60FF
:10535000EBE70024E1E700BFAFF30080AFF300808C
:10536000F8B5074600285AD057F8086C06F1100027
:10537000FFF786FC08363446A7F10805AC4204D88E
:105380006368083323449D420BD3B44211D0AC422E
:105390000FD32468AC42F8D86368083323449D4295
:1053A000F3D249F2D040C0F60200FEF7E9FFB44262
:1053B000EDD123681BB19D4201D31C46DEE757F8AF
:1053C000042C47F8083C256002F1080357F8080C44
:1053D000E918814209D0636803F10802224495422A
:1053E00011D0BDE8F840FFF75BBC4968EB580A44B0
:1053F000083247F8042C47F8083C636803F10802B8
:1054000022449542EDD157F8041C57F8082C0B4460
:10541000083384E80C00BDE8F840FFF741BC49F2CE
:10542000C04049F2A041C0F60200C0F60201C62207
:105430001DF02EFA98E700BFAFF30080AFF30080B5
:10544000F0B4002B08BF0B4600F10B0700F10A0572
:10545000B1FBF2F602FB161101F13004392CC8BF82
:1054600001F13704E4B2B3FBF2F331462E4605F8FE
:105470000149002BECD1BA1B3346024401E013F87A
:10548000014F00F8014B9042F9D1F0BC704700BFCA
:105490002DE9F04717469846064600220023384675
:1054A0004146DDF82090FCF763FD60B12D2408F142
:1054B00000483846414606F8014B00220023FCF71D
:1054C00057FD0028F3D138464146FBF731FE00284E
:1054D0003CD0B9F1000F34D04CF6CD4ACCF6CC4AD2
:1054E000AAFB093A4FEADA0A41463846FCF768FD5A
:1054F000044621460A2230460023FFF7A1FF064654
:105500002E2306F8013B2046FCF754FA02460B46D0
:1055100038464146FCF700F9044648460D46FCF77C
:1055200039FA02460B4620462946FCF7A9FAFCF751
:1055300047FD534601460A223046BDE8F047FFF7D3
:105540007FBF4FF00A0A4FF06409CDE74E23612276
:105550003370B3707270F01CBDE8F087AFF3008059
:105560002DE9F04F40F2A853C1F200038DB0074679
:1055700098690C46164616F063FF402840F35C819C
:105580000DF119000DF1180B49F2F0430390C0F62C
:105590000203CBEB0000059004932178631C51B10A
:1055A00025290BD03A681C469268384690472178E6
:1055B000631C0029F4D10DB0BDE8F08F62782D2A6C
:1055C00003BFA278A31C4FF0010C4FF0000C2E2A51
:1055D00018BF302A03BF5A7801334FF030084FF01C
:1055E00020081C46002506E03378043605EB8505C7
:1055F000227803EB4505A2F13003DBB2092B04F15D
:105600000104F3D92A2AEFD02E2A4FF0000949D0FD
:1056100002F0DF034C2B03D123780BB101341A467F
:10562000A2F14403342B00F2EF80DFE813F0D50041
:10563000ED00ED00ED00ED00D500ED00ED00ED001A
:10564000ED00ED00EB00ED00ED00ED00ED00ED00F4
:105650004500ED00ED00E900ED00ED00ED00ED008E
:10566000ED00ED00ED00ED00ED00ED00CB00D5000C
:10567000ED009C00ED00ED00D500ED00ED00ED002B
:10568000ED00ED00EB00ED00ED00ED007800ED0029
:105690004500ED00ED00E9003378043609EB890997
:1056A00003EB490914F8012BA2F13003DBB2092BFB
:1056B000F4D92A2AF0D0ABE70A22316858460023F1
:1056C000FFF7BEFE0436DA46CBEB0009C9EB050551
:1056D00025EAE575BCF1000F0DD16D425DB19AF878
:1056E00000102D2900F096803B6838469B684146A3
:1056F00098470135F8D1B9F1000F05DD3B685146F7
:105700004A461B6838469847002D3FF446AF3B6831
:1057100038469B6841469847013DF8D13DE7D6F8A9
:1057200000A0049BBAF1000F08BF9A4647F6FF722B
:105730009AF800300436B9F1000F08BF9146002BEB
:1057400000F083800AEB0902D14601E091456ED05A
:1057500099F8013009F10109002BF7D1CAEB0909C9
:105760004FF02008B2E7073626F00706D6E9000119
:10577000CDF808C0FCF74CFC07EE900AF5EEC07AB5
:10578000F1EE10FADDF808C044BFF1EE677A2D2380
:1057900017EE900A4ABF0DF1190ADA468DF8183053
:1057A000CDF808C0FCF718F9CDF8009002460B467A
:1057B0005046FFF76DFE0836DA46CBEB0009DDF800
:1057C00008C083E73368DDF814908DF8183004368C
:1057D0004FF02008DA4679E731680029BFBF2D2055
:1057E0008DF8180049420DF11900A8BF58460A2249
:1057F0000023FFF725FE0436DA46CBEB000965E708
:1058000010225AE7082258E78DF81820DDF8149086
:10581000DA465BE7B8F1300F7FF466AF3B68384695
:105820009B6898470AF1010A09F1FF395CE7CAEB66
:1058300002094FF0200849E749F2F840C0F602009B
:1058400023F0BEFA0DB0BDE8F08F99464FF0200866
:105850003CE700BFAFF30080AFF30080AFF3008000
:10586000C36882689A421FBF4268D154C36801333B
:105870001ABFC36000206FF001007047AFF30080D3
:105880000269C168914218BF416803461DBF885C28
:1058900001321A616FF00100704700BFAFF3008062
:1058A00038B5044608462369E5686168ED1AAA42DE
:1058B00038BF154619442A46FDF7E2FB23692B44FD
:1058C0002361284638BD00BFAFF30080AFF30080EE
:1058D00038B5C36885680446ED1A4068AA4238BFE7
:1058E000154618442A46FDF7CBFBE3682B44E360DA
:1058F000284638BDAFF30080AFF30080AFF30080DF
:1059000030B449F21054C0F6020400250460056169
:1059100041608260C36030BC704700BFAFF300805D
:10592000002910B41CDD02464418002012F8011BA7
:105930000823484010F0800F4FEA40001CBF80F061
:105940002700C04303F1FF3314BF00F0FE00C0B2D4
:1059500013F0FF03EED1A242E8D15DF8044B70478B
:105960000020FAE7AFF30080AFF30080AFF30080D0
:1059700010B4A1B149F220540144C0F602044FF022
:10598000FF3310F8012B5A40D2B2884254F822203B
:1059900082EA1323F5D1D8435DF8044B70470846DB
:1059A000FAE700BFAFF30080AFF30080AFF30080F1
:1059B0002DE9F04104461E468846174619F008F9BD
:1059C000E368054613B12046FEF72AFD204641460E
:1059D0003A463346FEF7ECFC0DB1BDE8F081BDE878
:1059E000F04119F01DB900BFAFF30080AFF30080A4
:1059F00008B503F07DF94AF69040C0F6020004F0C5
:105A0000B7FA00F045F800F0C3F800F0D9F900F05B
:105A100017FA00F0A5FA00F0B3FA01F059F801F016
:105A2000FFF801F08DFB01F083FD00F0D1FD01F0E6
:105A30003FFA01F095F8BDE8084006F081BC00BFD0
:105A40004FF48053CEF2000310B45A681C46104441
:105A5000824263680BD2984294BF002101219A428E
:105A600088BF00210029F3D15DF8044B70479A42AA
:105A70008CBF00210121984288BF41F0010100291B
:105A8000E6D1F1E7AFF30080AFF30080AFF3008021
:105A900003F01EBAAFF30080AFF30080AFF30080D5
:105AA00000230122027043608360C360036143618D
:105AB0001830FFF755B800BFAFF30080AFF3008098
:105AC00038B504460D46D8B1202383F31188FEF77C
:105AD000FFFA2378013BDBB2012B05D949F64C10C4
:105AE000C0F60200FEF74CFC2046656003F020FA89
:105AF00002232370FEF70CFB002383F3118838BDCB
:105B000049F6201049F63011C0F60200C0F6020135
:105B100071221CF0BDFED7E7AFF30080AFF3008029
:105B2000F8B504460E4617461D46FEF7B1FB002E9B
:105B300018BF002C1BD0D7B1012D01D0EB0716D414
:105B400023781A1FD2B2022B18BF012A05D949F6B1
:105B50009010C0F60200FEF713FC0323A760E56077
:105B6000266123702046BDE8F84003F049BA49F6A3
:105B7000781049F63011C0F60200C0F60201C322C7
:105B80001CF086FEDCE700BFAFF30080AFF30080BF
:105B900003F0DEBFAFF30080AFF30080AFF300800F
:105BA00038B50123002504460370456029460830B6
:105BB000FEF736FF294604F11400FEF731FF04F129
:105BC000200504F1240004F1280104F12C0204F161
:105BD000300325626062A162E262236338BD00BFC8
:105BE00038B504460D4668B3202383F31188FEF7C9
:105BF0006FFA23785A1ED2B2022A05D90EE0062087
:105C00000121FEF7D5FC2378022BF8D0012B0DD013
:105C1000FEF77EFA002383F3118838BD49F67C2015
:105C2000C0F60200FEF7ACFB2378EDE72046656086
:105C300003F0AEFF03232370FEF76AFA002383F319
:105C4000118838BD49F6502049F66021C0F602009F
:105C5000C0F602016D221CF01BFEC5E7AFF3008009
:105C60002DE9F043002A18BF002883B0044691466E
:105C70000E4698462DD003292BD8202383F3118874
:105C8000FEF726FA2578EB1EDBB2012B06D949F682
:105C9000B820C0F60200FEF773FB257804F1080770
:105CA00000E02578042D3146204602D003F0D8FFCD
:105CB000D8B938464146FEF7D3FE0028F1D001900E
:105CC000FEF726FA002383F31188019803B0BDE89C
:105CD000F08349F6A82049F66021C0F60200C0F61C
:105CE0000201AF221CF0D4FDC7E7204631464A46E8
:105CF00003F0D6FFFEF70CFA002383F3118800208F
:105D000003B0BDE8F08300BFAFF30080AFF30080C5
:105D10002DE9F043002A18BF002883B004469146BD
:105D20000E46984601D001290AD949F6CC2049F6F9
:105D30006021C0F60200C0F60201DC221CF0A8FDC2
:105D4000202383F31188FEF7C3F92578EB1EDBB21D
:105D5000012B06D949F6DC20C0F60200FEF710FB45
:105D6000257804F1140700E02578042D31462046FB
:105D700002D003F0D5FF78B938464146FEF770FEF1
:105D80000028F1D00190FEF7C3F9002383F31188B6
:105D9000019803B0BDE8F083204631464A4603F03F
:105DA000DFFFFEF7B5F9002383F31188002003B06D
:105DB000BDE8F083AFF30080AFF30080AFF3008065
:105DC00004F036B8AFF30080AFF30080AFF300808B
:105DD0000122002302704360704700BFAFF30080D0
:105DE000002918BF002838B504460D461BD02023D3
:105DF00083F31188FEF76CF92378013BDBB2012BAA
:105E000005D949F65C30C0F60200FEF7B9FA204623
:105E1000656004F08DF802232370FEF779F9002302
:105E200083F3118838BD49F6303049F64031C0F669
:105E30000200C0F6020162221CF02AFDD7E700BF73
:105E400005F0A6BCAFF30080AFF30080AFF3008095
:105E50000122002302704360704700BFAFF300804F
:105E6000002918BF002838B504460D461BD0202352
:105E700083F31188FEF72CF92378013BDBB2012B69
:105E800005D949F64C40C0F60200FEF779FA2046E3
:105E9000656005F08DFC02232370FEF739F90023BD
:105EA00083F3118838BD49F6204049F63041C0F6E9
:105EB0000200C0F6020160221CF0EAFCD7E700BF36
:105EC00038B504460D46FEF7E3F984B12378022B7A
:105ED00005D049F6F440C0F60200FEF751FA04235B
:105EE000294623702046BDE8384005F0A1BC49F69C
:105EF000DC4049F63041C0F60200C0F60201D22271
:105F00001CF0C6FCE2E700BFAFF30080AFF30080F7
:105F100010B50446FEF7BCF98CB12378023BDBB226
:105F2000022B05D949F62050C0F60200FEF728FAE8
:105F3000022323702046BDE8104005F089BC49F6D5
:105F40000C5049F63041C0F60200C0F60201F222C0
:105F50001CF09EFCE1E700BFAFF30080AFF30080D0
:105F600004F06EBAAFF30080AFF30080AFF30080AF
:105F700001220023027043600C30FEF7F1BD00BF28
:105F800005F006BDAFF30080AFF30080AFF30080F3
:105F90000122002302704360704700BFAFF300800E
:105FA000002918BF002838B504460D461BD0202311
:105FB00083F31188FEF78CF82378013BDBB2012BC9
:105FC00005D949F67C50C0F60200FEF7D9F9204603
:105FD000656005F00DFD02232370FEF799F800239C
:105FE00083F3118838BD49F6505049F66051C0F628
:105FF0000200C0F6020160221CF04AFCD7E700BF95
:1060000010B50446D0B1202383F31188FEF760F861
:106010002378013BDBB2012B05D949F69850C0F635
:106020000200FEF7ADF9204605F0B2FD0123237012
:10603000FEF76EF8002383F3118810BD49F68C50EB
:1060400049F66051C0F60200C0F6020174221CF04D
:106050001FFCD8E7AFF30080AFF30080AFF3008000
:1060600010B50446C0B1202383F31188FEF730F841
:106070002378022B05D049F6B850C0F60200FEF78F
:106080007FF9204605F0DCFD03232370FEF740F87E
:10609000002383F3118810BD49F6A85049F66051DA
:1060A000C0F60200C0F6020187221CF0F1FBDAE71D
:1060B00010B50446D0B1202383F31188FEF708F809
:1060C0002378023BDBB2032B05D949F6D850C0F642
:1060D0000200FEF755F9204605F0E2FD0223237089
:1060E000FEF716F8002383F3118810BD49F6C85057
:1060F00049F66051C0F60200C0F6020199221CF078
:10610000C7FBD8E7AFF30080AFF30080AFF30080A8
:10611000002918BF002838B504460D460BD0237956
:10612000052B01BFA36A4FF40072002085E80C0024
:1061300018BF012038BD49F6307049F64071C0F6ED
:106140000200C0F602014FF44F721CF0A1FBE6E71B
:1061500030B5054683B010242B680121186801AAC8
:1061600001F096F99DF80430FF2B0FD0013CF3D1DC
:1061700002E00120FEF7D4FB2B680121186801AA78
:1061800001F086F99DF80430FF2BF2D103B030BD49
:1061900070B5154682B00C4606462C30FFF7D8FF86
:1061A0002A0C2B0A44F04001280E49F600648DF8B1
:1061B00004508DF802208DF803308DF800108DF812
:1061C00001006B46C0F6020401AD002201E013F8A5
:1061D000011F81EA4202AB42A25CF8D15200F36A8D
:1061E00042F001028DF8052018686A46062101F088
:1061F000FFF802B070BD00BFAFF30080AFF30080C6
:1062000030B5054683B009242B680121186801AA1E
:1062100001F03EF99DF80400FF2801D1013CF3D1C3
:1062200003B030BDAFF30080AFF30080AFF3008068
:10623000F8B50446C06A0F46154600681E4600F0D1
:10624000EFFF39462A462046FFF7A2FF04F12C0053
:10625000FFF7D6FFE16A054632460868042101F0DF
:1062600017F9E36A186801F003F82846F8BD00BF83
:10627000C36A70B504460E461868154600F0D0FF94
:106280002A4631462046FFF783FF04F12C00FFF732
:10629000B7FFE36A0546186800F0EAFF284670BDBC
:1062A000F0B5C36A85B005460C461868164600F07E
:1062B000B7FF214628460022FFF76AFF05F12C00B0
:1062C000FFF79EFF42F2107410B131E0013C36D06E
:1062D000EB6A012118686A4601F0DAF89DF800308F
:1062E000FE2BF3D1EB6A102118686A4601F0D0F852
:1062F0006B4606F10C01321F58781F78DE789C78C7
:10630000000440EA0760304340EA042041F80409F1
:10631000914203F10403EFD1EB6A0221186800F007
:10632000CFFFEB6A186800F0A3FF002005B0F0BDB6
:10633000EB6A186800F09CFF012005B0F0BD012059
:1063400005B0F0BDAFF30080AFF30080AFF3008085
:1063500070B5054682B0002800F09A802B79052B95
:1063600018BF022B40F08D80EB6A0022032493E8D3
:1063700003002C7185F8302000F0F2FEEB6A10214A
:10638000186800F09DFF0A2402E00A20FEF7C8FA10
:1063900000210A462846FFF76BFF01280AD0013C7E
:1063A000F3D1EB6A186800F00BFF02232B71012078
:1063B00002B070BD01AB284608214FF4D572FFF73B
:1063C00037FF052825D0642404E0013CE9D00A20E9
:1063D000FEF7A6FA284637210022FFF749FF0128D9
:1063E0000646F2D14FF4D572C4F2000228462921A4
:1063F00001ABFFF71DFF0028E7D1024601AB28469D
:106400003A21FFF715FF9DF804305B0648BF85F879
:106410003060642405E0012BC3D1013CC1D0FEF7FC
:106420007FFA284601210022FFF722FF03460A20B7
:10643000002BF0D1EB6A1868996800F091FE2846AD
:1064400010214FF40072FFF713FF0028A9D105F1C6
:106450001804224628460921FFF722FF0028A0D170
:10646000204600F00DFBA86200289AD028460A2199
:1064700005F10802FFF714FF002892D105232B71C4
:1064800096E749F67070C0F60200FDF779FF6BE7FA
:1064900049F6607049F64071C0F60200C0F602018C
:1064A00040F2C3121CF0F4F958E700BFAFF30080CC
:1064B00010B50368044682B0186800F0B1FE02E02F
:1064C0000120FEF72DFA23680121186801AA00F0C7
:1064D000DFFF9DF80430FF2BF2D12368186800F02D
:1064E000C7FE02B010BD00BFAFF30080AFF3008065
:1064F00038B50446A0B3202383F31188FDF7E8FDE7
:106500002379052B18BF022B1AD1022B21D004238B
:106510002371FDF7FDFD002383F31188254655F80F
:106520002C3F9968186800F01BFE2846FFF7C0FF53
:10653000E36A186800F044FE02232371002038BD8E
:1065400049F69870C0F60200FDF71AFF2379022B76
:10655000DDD1FDF7DDFD002383F31188002038BD78
:1065600049F6847049F64071C0F60200C0F6020197
:1065700040F22D221CF08CF9BDE700BFAFF3008084
:1065800070B5044698B12579052D01D0012070BD64
:106590002646082256F82C3F22711868996800F0A8
:1065A000DFFD3046FFF784FF2571002070BD49F6FE
:1065B000AC7049F64071C0F60200C0F6020140F22C
:1065C0001E321CF065F9DEE7AFF30080AFF3008008
:1065D000704700BFAFF30080AFF30080AFF30080DF
:1065E00049F610730022C0F6020301210360017115
:1065F000C26280F830207047AFF30080AFF30080B4
:10660000002918BF002838B504460D460ED023795E
:10661000013BDBB2012B05D949F6C870C0F6020078
:10662000FDF7AEFE0223E562237138BD49F6B8706E
:1066300049F64071C0F60200C0F6020140F2951220
:106640001CF026F9E3E700BFAFF30080AFF3008052
:1066500010B5044688B12379013BDBB2012B05D983
:1066600049F6E470C0F60200FDF78AFEE36A186896
:1066700000F0A6FD0123237110BD49F6D87049F63C
:106680004071C0F60200C0F602014FF4D3721CF054
:10669000FFF8E0E7AFF30080AFF30080AFF30080D6
:1066A00038B504460D4670B32379052B05D04AF260
:1066B0001000C0F60200FDF763FEE36A06221868C8
:1066C0009968227100F04CFDE36A186800F0A8FD9B
:1066D00094F830308BB12A4620461221FFF758FD3E
:1066E00004F12C00FFF78CFD30B1E36A186800F06C
:1066F00067FD05232371012038BD6A02204612215F
:10670000FFF746FDECE749F6F47049F64071C0F634
:106710000200C0F602014FF414721CF0B9F8C3E78E
:10672000002918BF002870B506460D4620D03379E1
:10673000062B01D0012070BD42F2107401E0013C33
:1067400023D0F36A012118682A4600F0A1FE2B78B5
:10675000FE2BF4D1F36A2A4618684FF4007100F05A
:1067600097FEF36A0221186800F0AAFD002070BDB0
:106770004AF2300049F64071C0F60200C0F602014C
:106780004FF41E721CF084F8D1E7F36A186800F029
:106790006FFDF36A186800F013FD052333710120C3
:1067A00070BD00BFAFF30080AFF30080AFF3008097
:1067B00038B50446D0B12379062B01D0012038BD6D
:1067C000254649F6007255F82C3FC0F602021868BB
:1067D000072100F00DFE2846FFF712FDE36A186856
:1067E00000F046FD05232371002038BD4AF2480021
:1067F00049F64071C0F60200C0F602014FF427725C
:106800001CF046F8D7E700BFAFF30080AFF300807D
:1068100070B514461D460646FFF742FF58B915B934
:106820000BE0013D09D021463046FFF779FF04F522
:1068300000740028F5D0012070BD3046BDE87040DE
:10684000FFF7B6BFAFF30080AFF30080AFF3008077
:1068500038B504460D4670B32379052B05D04AF2AE
:106860008000C0F60200FDF78BFDE36A072218687E
:106870009968227100F074FCE36A186800F0D0FC9B
:1068800094F830308BB12A4620461921FFF780FC5E
:1068900004F12C00FFF7B4FC30B1E36A186800F093
:1068A0008FFC05232371012038BD6A02204619217F
:1068B000FFF76EFCECE74AF2640049F64071C0F65F
:1068C0000200C0F6020140F2BA221BF0E1FFC3E76A
:1068D00030B5002918BF002883B004460D4606D005
:1068E0002379072B18BF012012D003B030BD4AF224
:1068F000A00049F64071C0F60200C0F6020140F265
:10690000E1221BF0C5FF2379072B18BF0120ECD132
:10691000E36A49F6F0521868C0F60202022100F05C
:1069200067FDE36A2A4618684FF4007100F060FDC5
:10693000E36A0221186800F0C3FCE36A01211868C9
:1069400001AA00F0A5FD9DF8043003F01F03052BFC
:106950000CD0E36A186800F08BFCE36A186800F05A
:106960002FFC05230120237103B030BD04F12C005E
:10697000FFF7EEFB0020B8E7AFF30080AFF3008035
:1069800010B50446A8B12379072B01D0012010BD12
:10699000E36A4AF2F0021868C0F60202022100F02F
:1069A00027FDE36A186800F063FC052323710020CB
:1069B00010BD4AF2B80049F64071C0F60200C0F6B8
:1069C00002014FF441721BF063FFDCE7AFF300807C
:1069D00070B514461D460646FFF73AFF58B915B97B
:1069E0000BE0013D09D021463046FFF771FF04F569
:1069F00000740028F5D0012070BD3046BDE870401D
:106A0000FFF7BEBFAFF30080AFF30080AFF30080AD
:106A1000914270B50D461446064615D38B1A1F2BAE
:106A200012D805F01F026309013201206D0900FA36
:106A300002F2AB4202F1FF3204F01F0410D356F809
:106A400023001040E04070BD4AF200104AF21411D9
:106A5000C0F60200C0F6020149221BF019FFE0E770
:106A600056F8250056F823101040C4F12003984032
:106A700021FA04F4204370BDAFF30080AFF300802F
:106A8000C3689B0F70B504460AD0012B06D145217F
:106A90003022FFF7BDFF0130800270BD002070BDC5
:106AA00049213E22FFF7B4FF312106462F2220461E
:106AB000FFF7AEFF5321054650222046FFF7A8FFFF
:106AC0000136023506FA05F5093805FA00F070BD01
:106AD00005F096B9AFF30080AFF30080AFF300800C
:106AE0000122002302704360704700BFAFF30080B3
:106AF000002918BF002838B504460D461DD02023B4
:106B000083F31188FDF7E4FA2378013BDBB2012B14
:106B100005D94AF25C10C0F60200FDF731FCAB88E3
:106B200065602381204605F08BF902232370FDF771
:106B3000EFFA002383F3118838BD4AF230104AF28D
:106B40004011C0F60200C0F6020165221BF0A0FE53
:106B5000D5E700BFAFF30080AFF30080AFF3008054
:106B600004F0F6BAAFF30080AFF30080AFF300801B
:106B700010B5044620B12046BDE8104004F030BBFB
:106B80004AF200204AF21021C0F60200C0F60201CB
:106B9000BB221BF07DFE2046BDE8104004F020BB68
:106BA0000C30FEF7F5B900BFAFF30080AFF3008003
:106BB0000C304FF0FF33FEF7EBB900BFAFF30080AE
:106BC0003030FEF7CDBA00BFAFF30080AFF30080E6
:106BD00030304FF0FF33FEF7C3BA00BFAFF3008091
:106BE0000C30FEF79DB900BFAFF30080AFF300801B
:106BF0000C304FF0FF31FEF793B900BFAFF30080C8
:106C00003030FEF74DBA00BFAFF30080AFF3008025
:106C100030304FF0FF32FEF743BA00BFAFF30080D1
:106C200005F0C6BAAFF30080AFF30080AFF3008089
:106C300070B54AF2E023C0F60203044682B040F881
:106C4000043B012600940B461546606004F1540194
:106C500004F10C0026721022FEF70AF900942B466C
:106C600004F1300004F164011022FEF7E9F902B0EA
:106C700070BD00BFAFF30080AFF30080AFF30080C2
:106C800038B504460D46D8B1202383F31188FDF7AB
:106C90001FFA237A013BDBB2012B05D94AF2882087
:106CA000C0F60200FDF76CFB2946204605F0B8FA55
:106CB00002232372FDF72CFA002383F3118838BDD9
:106CC0004AF260204AF26C21C0F60200C0F60201CE
:106CD000A1221BF0DDFDD7E7AFF30080AFF300800A
:106CE00038B504460D46FDF7D3FAD4B163693BB11C
:106CF000294604F10C00FEF7E3F800280BDB38BD51
:106D0000201D0421FEF774F8294604F10C00FEF75B
:106D1000D7F80028F3DA201D8021BDE83840FEF7BF
:106D200067B84AF2B4204AF26C21C0F60200C0F6FD
:106D30000201D8221BF0ACFDD8E700BFAFF3008002
:106D400070B5046AD4F854321A681178042900D056
:106D500070BD217A0229FBD112891B7942FA03F313
:106D600013F00105F4D1216CE36BA26BC91A8E1AE2
:106D7000EED0FDF7CDF92B4683F31188D4F85422D9
:106D800033461068117904F1300200F071FC2023C1
:106D900083F31188FDF79CF9D4F85432BDE87040B4
:106DA0001868197900F09CBCAFF30080AFF3008045
:106DB000F8B5046AD4F8542213681978042900D06D
:106DC000F8BD217A0229FBD15279598903EB82035C
:106DD00041FA02F2DB6812F001075D8AF0D1E66940
:106DE000A2696369B61AF61AB542E9D8FDF790F9B7
:106DF0003B4683F31188D4F85422B6FBF5F305FB28
:106E000003F31068517904F10C0200F021FC2023F7
:106E100083F31188FDF75CF9D4F854321868597976
:106E2000BDE8F84000F034BCAFF30080AFF3008061
:106E30000C30FEF7ADB800BFAFF30080AFF30080B9
:106E40000C304FF0FF33FEF7A3B800BFAFF3008064
:106E50003030FEF785B900BFAFF30080AFF300809C
:106E600030304FF0FF33FEF77BB900BFAFF3008047
:106E70000C30FEF755B800BFAFF30080AFF30080D1
:106E80000C304FF0FF31FEF74BB800BFAFF300807E
:106E90003030FEF705B900BFAFF30080AFF30080DC
:106EA00030304FF0FF32FEF7FBB800BFAFF3008089
:106EB000704700BFAFF30080AFF30080AFF30080F6
:106EC00010B502464AF25033C0F6020342F8043BC2
:106ED00082B00446012146F6B1530090C0F600038B
:106EE000426001724FF4807204F154010C30FDF7DE
:106EF000BFFF46F64153009404F1300004F5AA7137
:106F0000C0F600034FF48072FEF79AF802B010BD8D
:106F100070B50D4604460E6828B3202383F311880C
:106F2000FDF7D6F8237A013BDBB2012B05D94AF2F3
:106F30003030C0F60200FDF723FA2A7906EB820210
:106F4000022394616A79093246F82240AA7906EB55
:106F50008206B4612372C4F85452FDF7D9F80023B5
:106F600083F3118870BD4AF200304AF21031C0F646
:106F70000200C0F60201DA221BF08AFCCDE700BF56
:106F800070B5D0F8543200F10C06044630461D6846
:106F9000FDF77EFF04F13000FEF762F8201D0121AD
:106FA000FDF726FFD4F85432597905EB81032846C2
:106FB000DB6832465B8A00F04BFBD4F8543228463B
:106FC0005979BDE8704000F063BB00BFAFF30080AB
:106FD00090F8443003F06003202B01D0002070476C
:106FE00090F84530212B03D0222B0CD0202BF5D14B
:106FF00041F2F863C2F20003072100228363C163F8
:1070000002640120704700238363C363036401208B
:10701000704700BFAFF30080AFF30080AFF3008094
:10702000F8B500EB810306469C690D46CCB12023E0
:1070300083F31188FDF78CF80821201DFDF7D8FE99
:10704000216CE26BA36B8A1AD71A19D106EB850360
:10705000DA6853695B682BB9FDF79AF8002383F36C
:107060001188F8BD128A013A12EA0307F4D1FDF73C
:107070008FF83B4683F31188002304F1300207E0C8
:10708000FDF786F8002383F3118804F130023B46B4
:107090003046294600F0ECFA202383F31188FDF7EF
:1070A00057F83046294600F01BFBD5E7AFF30080C8
:1070B00001F109032DE9F04150F823400D46064641
:1070C000CCB1202383F31188FDF742F8201D042161
:1070D000FDF78EFE06EB8503E169D868A269636956
:1070E000478A8A1AC3EB0208474506D9FDF750F8CC
:1070F000002383F31188BDE8F081FDF749F80023F0
:1071000083F31188B8FBF7F307FB03F304F10C02D8
:107110003046294600F09CFA202383F31188FDF7BE
:1071200017F83046294600F0B3FADFE7AFF30080E6
:10713000704700BFAFF30080AFF30080AFF3008073
:1071400004F0F6B8AFF30080AFF30080AFF3008037
:10715000002301220270436083600C30FDF700BD04
:10716000002918BF002838B504460D461BD020233F
:1071700083F31188FCF7ACFF2378013BDBB2012BD2
:1071800005D94AF29C30C0F60200FDF7F9F8204616
:10719000656004F025F902232370FCF7B9FF002392
:1071A00083F3118838BD4AF270304AF28031C0F65C
:1071B0000200C0F602016D221BF06AFBD7E700BF98
:1071C00010B50446E8B1202383F31188FCF780FF53
:1071D0002378013BDBB2012B05D94AF2B830C0F667
:1071E0000200FDF7CDF8204604F01AFA204604F01C
:1071F000C7F901232370FCF78BFF002383F3118869
:1072000010BD4AF2AC304AF28031C0F60200C0F63E
:10721000020183221BF03CFBD5E700BFAFF30080E7
:1072200010B50446B0B1202383F31188FCF750FF5A
:107230002378022B05D04AF2D830C0F60200FDF7C1
:107240009FF8204604F0DCF9FCF762FF002383F38B
:10725000118810BD4AF2C8304AF28031C0F60200EF
:10726000C0F6020197221BF013FBDCE7AFF30080AE
:1072700010B50446B0B1202383F31188FCF728FF32
:107280002378022B05D04AF2F830C0F60200FDF751
:1072900077F8204604F0C4F9FCF73AFF002383F3A3
:1072A000118810BD4AF2E8304AF28031C0F602007F
:1072B000C0F60201A9221BF0EBFADCE7AFF3008075
:1072C000002918BF002838B504460D4633D02023C6
:1072D00083F31188FCF7FCFE2378022B05D04AF2D9
:1072E000D040C0F60200FDF74BF863681B682BB175
:1072F0004AF2E040C0F60200FDF742F80323237093
:107300002946204604F09CF9A3682BB14AF2F040CC
:10731000C0F60200FDF734F840F2A853C1F20003B2
:1073200002209B69A360FDF713F9FCF7F1FE00232F
:1073300083F3118838BD4AF2BC404AF28031C0F66E
:107340000200C0F602014FF495721BF0A1FABEE7ED
:10735000002918BF0028F8B504460D4617461E46FA
:1073600039D0002A18BF002B35D0202383F3118891
:10737000FCF7AEFE2378022B05D04AF21050C0F67F
:107380000200FCF7FDFF63681B682BB14AF2245032
:10739000C0F60200FCF7F4FF0320334620702946B4
:1073A0003A46204604F06CF9A3682BB14AF2F0404B
:1073B000C0F60200FCF7E4FF40F2A853C1F200035C
:1073C00002209B69A360FDF7C3F8FCF7A1FE002330
:1073D00083F31188F8BD4AF200504AF28031C0F6BA
:1073E0000200C0F602014FF4A5721BF051FABCE78F
:1073F000002918BF002870B504460D46164635D042
:10740000A2B3202383F31188FCF762FE2378022BBA
:1074100005D04AF24450C0F60200FCF7B1FF6368A1
:107420001B682BB14AF25450C0F60200FCF7A8FFCB
:107430000323237029463246204604F041F9A3680D
:107440002BB14AF2F040C0F60200FCF799FF40F27F
:10745000A853C1F2000302209B69A360FDF778F8EE
:10746000FCF756FE002383F3118870BD4AF23850B2
:107470004AF28031C0F60200C0F6020140F2671203
:107480001BF006FABDE700BFAFF30080AFF300804A
:10749000002918BF002870B504460D46164635D0A1
:1074A000A2B3202383F31188FCF712FE2378022B6A
:1074B00005D04AF27450C0F60200FCF761FF636821
:1074C0001B682BB14AF28850C0F60200FCF758FF47
:1074D0000323237029463246204604F011F9A3689D
:1074E0002BB14AF2F040C0F60200FCF749FF40F22F
:1074F000A853C1F2000302209B69A360FDF728F89E
:10750000FCF706FE002383F3118870BD4AF2645035
:107510004AF28031C0F60200C0F602014FF4C27296
:107520001BF0B6F9BDE700BFAFF30080AFF30080FA
:1075300003F0CEB9AFF30080AFF30080AFF300806B
:107540000023012202704360C36183620362C3624D
:107550004362036303814381704700BFAFF3008040
:10756000002918BF002870B504460E4620D02023FD
:1075700083F31188FCF7ACFD2378013BDBB2012BD0
:1075800005D94AF21C60C0F60200FCF7F9FE00259E
:1075900020466660E56025616561A56103F0C0F97C
:1075A00002232370FCF7B4FD2B4683F3118870BDD2
:1075B0004AF2F0504AF20061C0F60200C0F6020141
:1075C00040F20F121BF064F9D1E700BFAFF3008067
:1075D000F8B5044615460E46FCF75AFE002D18BFB6
:1075E000002C25D02378042B05D04AF26060C0F629
:1075F0000200FCF7C5FE04EB8607FB682BB14AF2DC
:107600007C60C0F60200FCF7BBFE686918B100217F
:107610001422FBF78DFDA86918B100211422FBF795
:1076200087FDFD6020463146BDE8F84003F070BAA2
:107630004AF248604AF20061C0F60200C0F6020158
:1076400040F241121BF024F9CCE700BFAFF30080F9
:1076500070B400EB81040126E468A4690025E260AF
:1076600063602670A56070BC03F04ABBAFF3008076
:1076700070B400EB81040126E46864690025E260CF
:1076800063602670A56070BC03F0B2BBAFF30080EE
:1076900070B504460D46FCF7FBFD8CB1638943FAD7
:1076A00005F010F0010601D0012070BD0122AA40B2
:1076B000134320466381294603F0E2FC304670BD47
:1076C0004AF2D0604AF20061C0F60200C0F6020140
:1076D0004FF4F4721BF0DCF8E0E700BFAFF300807A
:1076E00070B504460D46FCF7D3FD8CB1238943FAEF
:1076F00005F010F0010601D0012070BD0122AA4062
:10770000134320462381294603F0CAFC304670BD4E
:107710004AF2E8604AF20061C0F60200C0F60201D7
:1077200040F203221BF0B4F8E0E700BFAFF30080A3
:10773000002202210170A0F84C2080F84E2080F831
:107740004F2002814281C26002614261826180F801
:10775000342003F05DB900BFAFF30080AFF30080C9
:1077600070B50023044680F8343000F1440203F081
:10777000B7FA63689B68002B31D02046984770B3F6
:10778000E06B94F8443094F84B1094F84A2042EAA5
:10779000012282423CBFE263104613F0800FE3688F
:1077A00040F09180002871D15B69052284F8342073
:1077B00001461870D86058609860204603F018FBA6
:1077C000202383F31188FCF7C3FC00212046FFF738
:1077D00087FFFCF7DDFC002383F3118870BD94F86C
:1077E000443013F0600611D02046002103F080FCE5
:1077F0002046002103F06CFC63681B6813B120462F
:1078000005219847062384F8343070BD94F845501C
:1078100003F07F0242EA0525B5F5407F00F0ED80D8
:1078200016DDB5F5C06F00F0D08063DDB5F5106FE3
:1078300073D040F60242954200F0F280B5F5006F39
:10784000D2D104F14F0201202664A263E0639AE7DB
:10785000022D00F0A18040F39680B5F5807F00F006
:107860008280B5F5817FBFD194F84620002ABBD134
:1078700094F8482012F00F014AD01206204600F179
:10788000FD8003F045FC94F8443041E09B69A56B12
:107890000022042184F834101146DD6058601A700B
:1078A0009A60204603F02CFA202383F31188FCF71A
:1078B0004FFC00212046FFF7EBFEFCF769FC00239C
:1078C00083F3118870BD58B15B69A56B002201215B
:1078D00084F834101146DD6058601A709A606CE7C5
:1078E0009B69032284F8342001461870D8605860E0
:1078F0009860D6E740F20232954221D0B5F5A06FEC
:107900007FF472AFB4F84420B2F5A06F00F0A48009
:107910000020A063E063206435E794F8462084F8F3
:107920004F20002A40F0868003222270626812688D
:10793000002AEDD020460221904794F84430E7E732
:1079400094F84620002A7FF44FAF94F8482012F0B4
:107950000F01DDD01306204600F1958003F0B8FB3F
:1079600094F84430D4E794F84620012A7FF43CAFE1
:10797000B4F84C20A66322F00202E6632664304687
:10798000A4F84C20FFE6002D47D104F14C02022060
:107990002564A263E063F6E694F8481011F0800FC6
:1079A000204601F00F0148D103F07AF9012848D0B0
:1079B00002287FF419AF4AF2E053C0F60203A36332
:1079C000E063266494F84430DDE6626894F8490088
:1079D00094F84830556894F8471094F8462043EAE4
:1079E00000232046A84700283FF4FEAE09C82664BD
:1079F000A363E06394F84430C5E694F84620012A76
:107A00007FF4F2AEB4F84C20A66342F00202E663C3
:107A100026643046A4F84C20B5E6012D7FF4E4AE90
:107A20004AF2D052C0F6020202200021A263E063B3
:107A30002164A8E60422227078E703F041F90128C6
:107A4000B6D14AF23073C0F60203A363E56326643D
:107A5000284694F8443096E694F84630204684F858
:107A60004E3003F045F863681B6813B120460121CE
:107A700098470323237094F8443049E703F058FBF8
:107A800094F8443044E703F033FB94F844303FE784
:107A900038B590F83430022B044647D0052B3ED041
:107AA000012B10D0002103F023FB2046002103F01E
:107AB0000FFB63681B6813B1204605219847062316
:107AC00084F8343038BD90F84B1090F84A30C26BCF
:107AD00043EA01239342C36805D9198AB2FBF1F541
:107AE00001FB152222B39A690321002384F8341084
:107AF000204619461370D3605360936003F000F979
:107B0000202383F31188FCF723FB00212046FFF795
:107B1000BFFDFCF73DFB002383F3118838BD036CE8
:107B200003B19847002384F8343038BDC368DAE7DE
:107B30005B6911461A70DA605A609A6003F058F96E
:107B4000202383F31188FCF703FB00212046FFF775
:107B5000C7FDFCF71DFB002383F31188022384F883
:107B6000343038BDAFF30080AFF30080AFF3008056
:107B700090F83430032B10B504462FD0042B11D0CD
:107B80002046002103F0B4FA2046002103F0A0FAB9
:107B900063681B6813B1204605219847062384F8C3
:107BA000343010BDC3685A690521002380F83410B1
:107BB00019461370D3605360936003F019F92023C2
:107BC00083F31188FCF7C4FA00212046FFF788FDF3
:107BD000FCF7DEFA002383F3118810BDC3689B69AC
:107BE0009B68002BCCD1036C03B19847002384F829
:107BF000343010BDAFF30080AFF30080AFF30080EE
:107C0000022909D003290CD04AF6F000C0F6020080
:107C1000012918BF002070474AF27070C0F60200B8
:107C20007047032A06D84AF6C000C0F6020000EBEF
:107C3000C200704700207047AFF30080AFF30080B0
:107C4000022910B504461FD1202383F31188FCF7C5
:107C50007FFA4AF240722046C0F602020121FFF785
:107C6000B7FC4AF28072C0F6020202212046FFF7FA
:107C7000AFFC41F66850C2F20000FFF781F9FCF753
:107C800087FA002383F3118810BD00BFAFF3008093
:107C900038B541F66855C2F200054AF6E0042846B8
:107CA000C0F60204FFF70CF921462846FFF730F929
:107CB0002468236D9A6B22F400229A6340F2DC5010
:107CC000FCF72EFE4AF2B0712046C0F60201FFF723
:107CD00047FC236D9A6B42F6381042F400229A63F7
:107CE000C2F200000021BDE83840FEF7C9BF00BF66
:107CF00041F66853C2F20003D3F854321B68187877
:107D0000031F584258417047AFF30080AFF3008023
:107D100002464FF00060CAB1531EDBB2032B11D9EB
:107D2000042B08BF4FF4803206D0063AD2B2062A9E
:107D300094BF4FF40032002210441A46531EDBB2A7
:107D4000032BEDD800F58040002BF6D1704700BF23
:107D50004FF47053C4F2020370B51A69002A064644
:107D6000C0F28D804FF47051C4F20201CA684FF422
:107D70007053D403C4F20203F8D41A6922F4807257
:107D80001A611A6942F400721A611A6922F07802C3
:107D90001A61F00742BF1A6942F008021A61B1077E
:107DA00041BF4FF47053C4F202031A6942F010024B
:107DB00048BF1A61720741BF4FF47053C4F2020307
:107DC0001A6942F0200248BF1A61330741BF4FF4DD
:107DD0007053C4F202031A6942F0400248BF1A61AC
:107DE0004FF47053C4F202031C461A6942F00202B7
:107DF0001A611A6942F480321A61E3684FF47051D3
:107E000013F48035C4F20201F7D10B6923F00203A9
:107E10000B610B6943F000430B613046FFF778FFBD
:107E2000032E15D9042E27D0053EF6B2062E98BF94
:107E30004FF4003206D9002070BD043A032A00F145
:107E4000040008D901680131F7D06FF00A0070BD55
:107E50004FF48042F6E7002AEDD00178FF29F4D1F3
:107E60000244013A034603E013F8011FFF29ECD155
:107E70009342F9D1002070BD4FF48032E2E740F226
:107E8000231148F6AB12C4F26751CCF6EF52596099
:107E90005A601B69002BBFF665AF4FF0FF3070BD15
:107EA000F8B58C46074639B3002500E025466C1C22
:107EB000E4B22046FFF72CFFB8420646F6D9284622
:107EC000FFF746FFB8B9032D98BF4FF480430BD995
:107ED000042D08BF4FF4803306D06B1FDBB2062B96
:107EE00094BF4FF400330023634505D2BCEB030C71
:107EF00002D03746D8E7F8BD0020F8BDAFF30080C8
:107F000008B5034608461946FBF7BAF8002008BD35
:107F10004FF470532DE9F043C4F20203054618698B
:107F2000002883B00F461646C0F297804FF4705277
:107F3000C4F20202D3684FF47054D803C4F20204AE
:107F4000F8D4236923F480732361236943F4007315
:107F5000236115F0030338D1032E40F28F80A6F180
:107F6000040C05F1040828464FEA9C0C4FF47055A8
:107F700008EB8C08391AC4F202052A690B5842F042
:107F800001022A6140F8043BEC684FF47053E203AD
:107F9000C4F20203F8D41C69404524F001041C61BA
:107FA000EBD10CF1010C07EB8C0706F00306002E59
:107FB00033D14FF47053C4F2020300201A6942F027
:107FC00000421A6103B0BDE8F083C3EB050902A8C3
:107FD000D9F80020C3F1040840F8042DB04528BFAB
:107FE000B046184442463946FBF74AF82269019BDD
:107FF00042F001022261C9F80030E1684FF4705389
:10800000C903C4F20203F8D41A6922F001024544FC
:108010004744C8EB06061A619EE7D8F8003002A86C
:10802000394640F8043D3246FBF72AF84FF47051C8
:10803000C4F20201019B0A6942F001020A61C8F818
:108040000030CA684FF47053D503C4F20203F8D469
:108050001A6922F001021A61ABE740F2231148F6D7
:10806000AB12C4F26751CCF6EF5259605A601B69EB
:10807000002BBFF65BAF4FF0FF30A3E7A84696E7B3
:10808000704700BFAFF30080AFF30080AFF3008014
:10809000704700BFAFF30080AFF30080AFF3008004
:1080A000704700BFAFF30080AFF30080AFF30080F4
:1080B00041F6E873C2F2000300221A60704700BF65
:1080C00070B441F6E874C2F200042568092D16DC8C
:1080D000002DD8BFAE000EDD636898420FD0211F7F
:1080E000AE003144234604E09A68904203F1040351
:1080F00005D08B42F8D1264401357060256070BCF4
:10810000704700BFAFF30080AFF30080AFF3008093
:1081100030B441F6E875C2F200052C68002C0DDD84
:108120006B68984224D02A46002304E09168884274
:1081300002F1040204D00133A342F7D130BC7047EE
:10814000002BFBDBA3420BDA05EB8301E31A0431BE
:108150009B000022486804329A4241F8040BF9D18E
:10816000013C05EB840300222C605A6030BC704750
:108170000023E9E7AFF30080AFF30080AFF30080A6
:1081800010B90846FFF7C4BF0846FFF799BF00BF04
:1081900030B441F6E874C2F200042568002D056091
:1081A00008DDAD000023E218C11852680433AB4269
:1081B0004A60F8D130BC7047AFF30080AFF3008065
:1081C00041F6E873C2F2000318680028D4BF00200B
:1081D00001207047AFF30080AFF30080AFF3008061
:1081E000002930B4054611DD4A1E002092000346E6
:1081F000EC5C392C94BF303C573C013394408B42AB
:108200002044A2F10402F3D130BC70470020FBE708
:108210002DE9F0432DED028B83B008EE900AF9F7BB
:10822000DBFB6A46F8F7ACFF00230022C4F25903D7
:1082300080468946DDE90001F9F74CFDF9F7C0FEFB
:1082400007EE100A9FED368AF8EEC77A064667EE0B
:10825000887A17EE900AF9F7BFFBF8F7E9FF642375
:1082600003FB06F607EE106AF8EEC77A044678EECE
:10827000E78A0D46FDEEE88AF8EEE88A68EE888A1D
:1082800018EE900AF9F7A8FBF8F7D2FF002306468C
:108290000F46404649460022C4F24E03F9F7F0FB70
:1082A0001DA3D3E90023F9F7EBFBF8F7C1FF8046E4
:1082B000894630463946F9F7ABFEDFED1A7A07EE0C
:1082C000100A87EE278A29462046F9F7A1FE49467B
:1082D00007EE900A404638EE278AF9F799FEDFED5F
:1082E000127A07EE100AC7EE277A78EE277A17EE91
:1082F000900AF9F771FBF8F79BFF07A3D3E9002376
:10830000F9F7E8FCF9F784FE03B0BDEC028BBDE899
:10831000F08300BFAFF300800000000080842E4196
:10832000002474490000704200006145AFF30080F2
:108330004E2970B504461DBFD4ED007AF1EE677A80
:1083400017EE900A0068452B1CBFD2ED007AF1EEC3
:10835000677A15460CBF166817EE906AFFF758FF4C
:1083600020603046FFF754FF286070BDAFF30080F7
:1083700038B504460D46FBF70BF82378B0F5807F3F
:10838000B4BF01464FF4807100222C2B10460BD055
:10839000002902DC08E0884206D0AB5414F8013F03
:1083A00001302C2B0246F6D10023AB5438BD00BF60
:1083B00070B50D46C0B02C21FAF70AFF2C21013010
:1083C000FAF706FF0446461C30466946FFF7D0FF21
:1083D00063780BB940B070BD68461DF089FF2C2151
:1083E00028603046FAF7F4FE034601305B784E2BE6
:1083F00004D0532B02D02C2B02D1002385F84C3013
:108400002C21FAF7E5FE441C69462046FFF7B0FF31
:1084100068461DF06DFF2C2168602046FAF7D8FEF3
:10842000034601305B78452B04D0572B02D02C2B10
:1084300002D1002385F84D302C21FAF7C9FE441CE7
:1084400069462046FFF794FF68461DF0B9FE2C21CF
:1084500068642046FAF7BCFE441C69462046FFF7D4
:1084600087FF68461DF0ACFE2C21A8642046FAF771
:10847000AFFE2C210130FAF7ABFE69460130FFF761
:1084800077FF68461DF034FFE86040B070BD00BF64
:108490002DE9F0410C46CCB02C21FAF799FE451C91
:1084A0000CA92846FFF764FF0CA8FAF771FF05280E
:1084B00023D99DF830109DF832209DF834309DF876
:1084C00031709DF833609DF835003039303A303BDB
:1084D0004FEA41084FEA420C4FEA430E08EBC10154
:1084E0000CEBC2020EEBC30339443244034430396F
:1084F000303A303B03910292019328462C21FAF73F
:1085000067FE451C28460CA9FFF732FF9DF8303066
:10851000562B04BF0023636470D004236364284691
:108520002C21FAF755FE451C0CA92846FFF720FF21
:108530000CA81DF0DDFE2C2120602846FAF748FE2D
:10854000034601305B784E2B5CD0532B5AD02C2B3A
:1085500057D02C21FAF73CFE451C0CA92846FFF702
:1085600007FF0CA81DF0C4FE2C2160602846FAF716
:108570002FFE034601305B78452B47D0572B45D063
:108580002C2B42D02C21FAF723FE451C0CA928469F
:10859000FFF7EEFE0CA81DF0ABFE2C21A0602846D4
:1085A000FAF716FE451C0CA92846FFF7E1FE0CA8B9
:1085B0001DF09EFE2C2120612846FAF709FE0CA929
:1085C0000130FFF7D5FE0CA8FAF7E2FE052820D807
:1085D00001AB5A69002A11DD1E46143409AF354635
:1085E0000FCDBD4220606160A260E3602E4604F1C1
:1085F0001004F4D107CE20606160A2604CB0BDE8E9
:10860000F081002384F84C30A3E7002384F84D3038
:10861000B8E79DF830009DF832109DF834309DF891
:1086200031709DF833609DF83550303B303830392B
:108630005A004FEA40084FEA410C02EBC30208EB34
:10864000C0000CEBC101384431442A443038303981
:10865000343201AB049005910692BBE7AFF3008082
:1086600010B52A210446FAF75BFF88B102210130D8
:10867000FFF7B6FD63782A2B04F102014FF00002E8
:1086800004D05A4011F8013B2A2BFAD1824201D082
:10869000802010BD002010BDAFF30080AFF300803C
:1086A00010B50446FFF7DCFF48B94AF60011C0F6E2
:1086B00002012046FBF7BEF818B1022010BDC0B27F
:1086C00010BD4AF608112046C0F60201FBF7B2F8C9
:1086D000003018BF012010BDAFF30080AFF3008061
:1086E00070B5044608460D46FFF7DAFF012884F806
:1086F000400010D002280DD128462146FFF758FE31
:108700002046221D94F84C1094F84D30BDE870407E
:10871000FFF70EBE70BD28462146BDE87040FFF74A
:10872000B7BE00BFAFF30080AFF30080AFF30080AF
:1087300010B5FBF755FD4FF4C042C4F2020242F2FD
:108740001403C2F2000311681C6801F03D0191603E
:108750000CB15868A047FBF773FDBDE81040FBF76C
:1087600017BB00BFAFF30080AFF30080AFF3008012
:1087700010B5FBF735FD4FF4C042C4F2020242F2DD
:1087800014031168C2F20003890901F03D019C68DD
:10879000880190600CB1D868A047FBF751FDBDE897
:1087A0001040FBF7F5BA00BFAFF30080AFF30080D5
:1087B00010B5FBF715FD4FF4C042C4F2020242F2BD
:1087C00014031168C2F20003090C01F03D011C6999
:1087D000080490600CB15869A047FBF731FDBDE873
:1087E0001040FBF7D5BA00BFAFF30080AFF30080B5
:1087F00010B5FBF7F5FC4FF4C042C4F2020242F29E
:1088000014031168C2F20003890D01F03D019C6957
:10881000880590600CB1D869A047FBF711FDBDE851
:108820001040FBF7B5BA00BFAFF30080AFF3008094
:1088300010B5FBF7D5FC4FF4C042C4F2020242F27D
:108840001403C2F2000351681C6A01F03D01D160BB
:108850000CB1586AA047FBF7F3FCBDE81040FBF7EA
:1088600097BA00BFAFF30080AFF30080AFF3008092
:1088700010B5FBF7B5FC4FF4C042C4F2020242F25D
:1088800014035168C2F20003890901F03D019C6A9A
:108890008801D0600CB1D86AA047FBF7D1FCBDE8D5
:1088A0001040FBF775BA00BFAFF30080AFF3008054
:1088B00010B5FBF795FC4FF4C042C4F2020242F23D
:1088C00014035168C2F20003090C01F03D011C6B56
:1088D0000804D0600CB1586BA047FBF7B1FCBDE8B1
:1088E0001040FBF755BA00BFAFF30080AFF3008034
:1088F00010B5FBF775FC4FF4C042C4F2020242F21D
:1089000014035168C2F20003890D01F03D019C6B14
:108910008805D0600CB1D86BA047FBF791FCBDE88F
:108920001040FBF735BA00BFAFF30080AFF3008013
:1089300010B5FBF755FC4FF4C842C4F2020242F2F4
:108940001403C2F2000311681C6C01F03D01916038
:108950000CB1586CA047FBF773FCBDE81040FBF767
:1089600017BA00BFAFF30080AFF30080AFF3008011
:1089700010B5FBF735FC4FF4C842C4F2020242F2D4
:1089800014031168C2F20003890901F03D019C6CD7
:10899000880190600CB1D86CA047FBF751FCBDE892
:1089A0001040FBF7F5B900BFAFF30080AFF30080D4
:1089B00010B5FBF715FC4FF4C842C4F2020242F2B4
:1089C00014031168C2F20003090C01F03D011C6D93
:1089D000080490600CB1586DA047FBF731FCBDE86E
:1089E0001040FBF7D5B900BFAFF30080AFF30080B4
:1089F00010B5FBF7F5FB4FF4C842C4F2020242F295
:108A000014031168C2F20003890D01F03D019C6D51
:108A1000880590600CB1D86DA047FBF711FCBDE84C
:108A20001040FBF7B5B900BFAFF30080AFF3008093
:108A300010B5FBF7D5FB4FF4C842C4F2020242F274
:108A40001403C2F2000351681C6E01F03D01D160B5
:108A50000CB1586EA047FBF7F3FBBDE81040FBF7E5
:108A600097B900BFAFF30080AFF30080AFF3008091
:108A700010B5FBF7B5FB4FF4C842C4F2020242F254
:108A800014035168C2F20003890901F03D019C6E94
:108A90008801D0600CB1D86EA047FBF7D1FBBDE8D0
:108AA0001040FBF775B900BFAFF30080AFF3008053
:108AB00010B5FBF795FB4FF4C842C4F2020242F234
:108AC00014035168C2F20003090C01F03D011C6F50
:108AD0000804D0600CB1586FA047FBF7B1FBBDE8AC
:108AE0001040FBF755B900BFAFF30080AFF3008033
:108AF00010B5FBF775FB4FF4C842C4F2020242F214
:108B000014035168C2F20003890D01F03D019C6F0E
:108B10008805D0600CB1D86FA047FBF791FBBDE88A
:108B20001040FBF735B900BFAFF30080AFF3008012
:108B300042F29403C2F2000330B400214AF69015C9
:108B400042F2140419600A460B46C0F60205C2F24E
:108B50000004E8580C33C02B0160A15002F1080258
:108B6000F7D14FF4C0414FF4C842C4F20201C4F23D
:108B700002024FF0FF338B6030BCCB609360D36058
:108B8000704700BFAFF30080AFF30080AFF3008009
:108B90002DE9F043064683B08946904600284ED022
:108BA00042F29404C2F20004777A2268012505FAA1
:108BB00007F1114218BF28463ED142F2140CC2F20E
:108BC000000C0A430CEBC70012F0FF0F4CF8378083
:108BD00043601CBF4FF46053C4F20203226018BF0D
:108BE000196B34681CBF41F40011196312F47F4FF4
:108BF0001FBF4FF46053C4F202031A6B42F48002A9
:108C000018BF1A63236823F01F032360236813F03F
:108C10000105FBD1327A73683D2191402122196010
:108C2000404625606261B8F1000F05D0B07A4FEA86
:108C30000911FBF72DF9284603B0BDE8F0834AF689
:108C400010104AF62811C0F60200C0F6020140F2E8
:108C5000CF12019319F01CFE019BA1E7AFF3008036
:108C600038B50546002835D042F29404C2F200041B
:108C70006A7A2368012101FA02F21A4223D0A87A03
:108C8000FBF72EF96B7A2268012101FA03F322EA3D
:108C9000030313F0FF0F04BF4FF46052C4F202024B
:108CA000236002BF116B21F40011116313F47F4F95
:108CB00001BF4FF46053C4F202031A6B22F4800226
:108CC00008BF1A6338BD4AF67010C0F60200FBF701
:108CD00057FBD4E74AF658104AF62811C0F60200AE
:108CE000C0F6020140F2FB1219F0D2FDBCE700BF52
:108CF0004FF46053C4F20203F0B400224FF0FF348B
:108D000019691C611A6159695C615A611E6A4EF2E7
:108D10001001CEF2000166F0805649F23F054EF692
:108D2000F0501E62CEF200001A62C0F20205072661
:108D30005F6A5C625A624D608A600E60C4684FF47C
:108D40008051CEF2000144F08074C460086840F0A5
:108D500001000860186C4FF4E041C4F2000140F0DB
:108D600080501864086840F480700860196F01F43E
:108D70004071B1F5007F1EBF4FF4803119671A674B
:108D80004FF46053C4F202031A6F120407D41A6F2F
:108D900042F400721A671A6F42F400421A674FF4E5
:108DA000E043C4F20003F0BC5A6822F400725A6037
:108DB000FFF7BEBEAFF30080AFF30080AFF30080DB
:108DC0004FF460514FF4E043C4F20201C4F20003D7
:108DD0004FF080504FF4404208641A600B6843F033
:108DE00001030B600A684FF460539007C4F202035A
:108DF000F8D59A6822F003029A609A6819469A6038
:108E00008B684FF4605213F00C03C4F20202F7D1E6
:108E1000116801F0F90111609360136843F4803325
:108E2000136011684FF460538903C4F20203F8D54C
:108E30005A6F42F001025A6719464A6F4FF4605365
:108E40009207C4F20203F8D545F20842C0F240721C
:108E50005A6019684FF4E04241F080711960C4F221
:108E6000000253685B04FCD54FF46051C4F2020168
:108E70000A684FF460539001C4F20203F8D54FF42E
:108E80007052C4F202024FF41441C3F6080140F2DA
:108E90000570996010609A6842F002029A60194663
:108EA0008A6802F00C024FF46053082AC4F20203ED
:108EB000F6D15A6C42F480425A645A6E42F48042AF
:108EC0005A667047AFF30080AFF30080AFF30080C5
:108ED00070B542F29805C2F20005284642F2CC0471
:108EE000FCF7DEFDC2F20004104E4FF4005242F6D1
:108EF0001643C4F20102C0F202032046AA622B63A9
:108F0000EE62FCF7CDFD4FF4045242F61643183ED4
:108F1000C4F20102C0F20223E662A26223631220BD
:108F20006021BDE87040FAF7B3BF00BF20AA020875
:108F300038B50378012B044600D038BD42F29805BD
:108F4000C2F20005A84216D042F2CC05C2F20005DA
:108F5000A8422AD04FF40C52C4F20102A36A54680A
:108F600004F44004002144F480340120546059602A
:108F70009960986038BD49F2F112C0F60002C06AEB
:108F800006212346FFF704FE48BBEB6A42F24C027F
:108F900019684FF46053C4F20102C4F202038A60FC
:108FA0005A6C42F480725A64D4E749F2F112C0F666
:108FB0000002C06A06212346FFF7EAFDB0B9EB6A5A
:108FC00042F24C1219684FF46053C4F20102C4F229
:108FD00002038A605A6C42F400725A64BAE74AF695
:108FE0005020C0F60200FBF7CBF9CEE74AF664202A
:108FF000C0F60200FBF7C4F9E1E700BFAFF3008061
:109000000369026B19782DE9F003C56829B1012DB8
:1090100094BF42F4807242F48472C16A5E88096827
:109020008468D3F80C80CC6006FB05F44C600A60C1
:10903000D1F800909F69DE691D6A5C6AD3F814C09C
:109040001B69826A49F00109C1F80090590044BFC8
:1090500023F0804121F0020148F0806046BF41F4D6
:10906000407143F4407343F440734FF0000840F400
:10907000807046BF41F0030143F0030343F0010356
:10908000C2F80080C2F80CC01761D6621563546341
:109090005060BDE8F00348BF91609360704700BF27
:1090A000C16A0A68136823F01F0310B413601368C1
:1090B00013F00103FBD10C7A826A48683D2101FA62
:1090C00004F40121046053605DF8044B93609160E7
:1090D000704700BFAFF30080AFF30080AFF30080B4
:1090E00010B5FBF77DF84FF40053C4F201030021E3
:1090F0001A681960940608D542F29804C2F2000476
:10910000E36A1B685B68002B41D14FF40453C4F23F
:10911000010300211A681960900632D542F2CC048E
:10912000C2F20004E36A1B685B6853B3236943B36C
:109130002046FFF7B5FF23699B684BB105222270DB
:109140002046012198472378052B04BF0223237072
:1091500000232361202383F31188FAF7F9FF42F2F9
:10916000CC03C2F20003586930B14FF0FF32826283
:1091700000225A61FBF794F9FBF70AF8002383F306
:109180001188FBF75DF8BDE81040FAF701BE2369CE
:10919000002BBAD02046FFF783FF23699B684BB1B1
:1091A000052222702046012198472378052B04BF11
:1091B0000223237000232361202383F31188FAF70D
:1091C000C7FF42F29803C2F20003586930B14FF072
:1091D000FF32826200225A61FBF762F9FAF7D8FF88
:1091E000002383F3118890E7AFF30080AFF3008092
:1091F00038B540F2A853C1F20003044698690D4601
:1092000013F01EF940284BDD15F00C0F21D1236916
:10921000F3B1AA0613D51D78002D49D05D68BDB104
:10922000E268012A83BF5988A3685208204683BF99
:10923000514303EB410120468168A84738BDED0644
:1092400006D55B6823B1E268A168204652089847BA
:1092500038BD2046FFF724FF23699B684BB10522E8
:1092600022702046002198472378052B04BF022353
:10927000237000232361202383F31188FAF768FF0A
:1092800063693BB100214FF0FF32616118469A6279
:10929000FBF706F9FAF77CFF002383F3118838BD4A
:1092A0004AF67820C0F60200BDE838401FF088BDBD
:1092B0002046FFF7F5FE23695B68D3B104222270D4
:1092C0002046A168E26898472378042B02BF022356
:1092D00025612370202383F31188FAF739FF63692E
:1092E000002BD7D00022626118469A62FBF7D8F8AB
:1092F000D0E7022223612270ECE700BFAFF30080C9
:1093000008B5FAF76DFF42F27010C2F200004FF498
:1093100070534268C4F2010301215268596100216F
:109320009047FAF78DFFBDE80840FAF731BD00BF5E
:1093300008B5FAF755FF42F27010C2F200004FF480
:1093400070534268C4F201030221D26859610121BD
:109350009047FAF775FFBDE80840FAF719BD00BF5E
:1093600008B5FAF73DFF42F27010C2F200004FF468
:1093700070534268C4F20103042152695961022109
:109380009047FAF75DFFBDE80840FAF701BD00BF5E
:1093900008B5FAF725FF42F27010C2F200004FF450
:1093A00070534268C4F201030821D2695961032154
:1093B0009047FAF745FFBDE80840FAF7E9BC00BF5F
:1093C00008B5FAF70DFF42F27010C2F200004FF438
:1093D00070534268C4F201031021526A596104219A
:1093E0009047FAF72DFFBDE80840FAF7D1BC00BF5F
:1093F00010B5FAF7F5FE4FF47053C4F201035C693F
:1094000004F478725A61A30634D4600628D4210685
:109410001CD4E20510D4A30508D542F27013C2F2A1
:10942000000318465B680921DB6C9847FAF708FFD0
:10943000BDE81040FAF7ACBC42F27013C2F2000370
:1094400018465B6808215B6C9847E4E742F27013AA
:10945000C2F2000318465B680721DB6B9847D8E728
:1094600042F27013C2F2000318465B6806215B6B80
:109470009847CCE742F27013C2F2000318465B68CB
:109480000521DB6A9847C0E7AFF30080AFF30080A7
:1094900010B5FAF7A5FE4FF47053C4F201035C69EE
:1094A00004F47C4261055A6140D4220534D4E304BB
:1094B00028D4A0041CD4610410D4220408D542F29C
:1094C0007013C2F2000318465B680F21DB6F9847E8
:1094D000FAF7B6FEBDE81040FAF75ABC42F2701334
:1094E000C2F2000318465B680E215B6F9847E4E701
:1094F00042F27013C2F2000318465B680D21DB6E66
:109500009847D8E742F27013C2F2000318465B682E
:109510000C215B6E9847CCE742F27013C2F2000355
:1095200018465B680B21DB6D9847C0E742F2701369
:10953000C2F2000318465B680A215B6D9847B4E7E6
:1095400008B5FAF74DFE42F27010C2F200004FF477
:1095500070534268C4F201034FF48031D2F8842082
:10956000596110219047FAF76BFEBDE80840FAF701
:109570000FBC00BFAFF30080AFF30080AFF30080FB
:1095800008B5FAF72DFE42F27010C2F200004FF457
:1095900070534268C4F201034FF40031D2F88C20BA
:1095A000596111219047FAF74BFEBDE80840FAF7E0
:1095B000EFBB00BFAFF30080AFF30080AFF30080DC
:1095C00008B5FAF70DFE42F27010C2F200004FF437
:1095D00070534268C4F201034FF48021D2F8942002
:1095E000596112219047FAF72BFEBDE80840FAF7BF
:1095F000CFBB00BFAFF30080AFF30080AFF30080BC
:1096000008B5FAF7EDFD42F27010C2F200004FF417
:1096100070534268C4F201034FF40021D2F89C2039
:10962000596113219047FAF70BFEBDE80840FAF79D
:10963000AFBB00BFAFF30080AFF30080AFF300809B
:1096400008B5FAF7CDFD42F27010C2F200004FF4F7
:1096500070534268C4F201034FF48011D2F8A42081
:10966000596114219047FAF7EBFDBDE80840FAF77D
:109670008FBB00BFAFF30080AFF30080AFF300807B
:1096800008B5FAF7ADFD42F27010C2F200004FF4D7
:1096900070534268C4F201034FF48001D2F8B42041
:1096A000596116219047FAF7CBFDBDE80840FAF75B
:1096B0006FBB00BFAFF30080AFF30080AFF300805B
:1096C00008B506206021FAF7E3FB07206021FAF7CE
:1096D000DFFB08206021FAF7DBFB09206021FAF7A5
:1096E000D7FB0A206021FAF7D3FB17206021FAF795
:1096F000CFFB28206021FAF7CBFB01206021FAF78D
:10970000C7FB2920F021FAF7C3FB2A206021FAF7D2
:10971000BFFB3E206021FAF7BBFB4C206021FAF72B
:10972000B7FB0220F021FAF7B3FB0320F021BDE8DC
:109730000840FAF7ADBB00BFAFF30080AFF3008085
:109740004FF46053C4F20203F0B41C6C4FF4C845EC
:10975000C4F2000544F000741C64D5F800321B0C00
:109760001B0443F0010343EA0023C5F8003200293B
:1097700065D00020C5F81C020346C5F80402044663
:10978000C5F80C02C5F81402D80000F1804000F5BD
:10979000C84001331C2BC0F84042C0F84442F3D10A
:1097A0004FF4C843C4F20003002501271079146860
:1097B00010F0010F18BFD3F804024FEAC40607FAED
:1097C00004F41EBF2043C3F80402107910F0020F06
:1097D0001FBFD3F80C022043C3F80C0210794007D6
:1097E00042BFD3F814022043C3F8140206F18046A6
:1097F000906806F5C8460135C6F84002D068C6F83C
:109800004402D3F81C028D4244EA000402F1100223
:10981000C3F81C42CAD14FF4C842C4F200024FF44C
:109820006053D2F80012C4F2020321F00101C2F821
:1098300000121A6C22F000721A64F0BC7047C30068
:10984000012203F1804303F5C84302FA00F01043FC
:10985000C5F84012C5F84412C3F84012C3F84412C8
:10986000C5F80412C5F81412C5F80C02C5F81C029C
:10987000D1E700BFAFF30080AFF30080AFF300800B
:1098800038B5426B40F20113C0F201039360044605
:10989000202383F31188FAF75BFC2369002BB8BF00
:1098A00004F1080505DA2846FBF722F92369002BA5
:1098B000F9DB04F124000121FBF79AFAFAF768FCBE
:1098C000002383F3118838BDAFF30080AFF300802D
:1098D000436B70B5DE68B207044614D1F30611D5A8
:1098E000636B1022DA60202383F31188FAF730FCCF
:1098F00004F128001021FBF77BFAFAF749FC00235A
:1099000083F3118870BD5A6922F002025A61202344
:1099100083F31188FAF71CFCE369002BB8BF04F14C
:10992000140505DA2846FBF7E3F8E369002BF9DBB9
:1099300004F120000121FBF75BFAFAF729FC002370
:1099400083F31188CAE700BFAFF30080AFF3008054
:10995000436B70B51E690446B00714D1F10611D5EA
:10996000636B10221A61202383F31188FAF7F0FB4E
:1099700004F128001021FBF73BFAFAF709FC002359
:1099800083F3118870BD5A6922F010025A612023B6
:1099900083F31188FAF7DCFBE369002BB8BF04F10D
:1099A000140505DA2846FBF7A3F8E369002BF9DB79
:1099B00004F120000221FBF71BFAFAF7E9FB002370
:1099C00083F31188CAE700BFAFF30080AFF30080D4
:1099D000426B70B555681C232E07044653601FD494
:1099E0006D071CD5636B9D699A6905F0070622F027
:1099F000700215F0700F9A6118BF46F00806202318
:109A000083F31188FAF7A4FB04F1280046EA054124
:109A1000FBF7EEF9FAF7BCFB002383F3118870BD66
:109A20001168064621F00201032306F8303B20238B
:109A3000116083F31188FAF78BFB30460021FBF7A6
:109A4000D7F9FAF7A5FB002383F31188C8E700BF15
:109A500008B5FAF7C5FB42F20010C2F20000FFF7AA
:109A60000FFFFAF7EDFBBDE80840FAF791B900BF28
:109A700008B5FAF7B5FB42F20010C2F20000FFF79A
:109A800027FFFAF7DDFBBDE80840FAF781B900BF10
:109A900008B5FAF7A5FB42F20010C2F20000FFF78A
:109AA00057FFFAF7CDFBBDE80840FAF771B900BFE0
:109AB00008B5FAF795FB42F20010C2F20000FFF77A
:109AC00087FFFAF7BDFBBDE80840FAF761B900BFB0
:109AD00008B5FAF785FB42F23810C2F20000FFF732
:109AE000CFFEFAF7ADFBBDE80840FAF751B900BF69
:109AF00008B5FAF775FB42F23810C2F20000FFF722
:109B0000E7FEFAF79DFBBDE80840FAF741B900BF50
:109B100008B5FAF765FB42F23810C2F20000FFF711
:109B200017FFFAF78DFBBDE80840FAF731B900BF1F
:109B300008B5FAF755FB42F23810C2F20000FFF701
:109B400047FFFAF77DFBBDE80840FAF721B900BFEF
:109B500038B542F20015C2F20005284642F2381428
:109B6000FCF71EF8C2F200044FF4C843C4F200032D
:109B700020466B63FCF714F84FF4D043C4F20003A3
:109B8000002163630A460E20BDE83840FFF7D8BDC8
:109B900042F20013C2F20003984210B504463CD0D2
:109BA00042F23812C2F2000290421AD0636B0221D4
:109BB000012221701A605A68D10707D406200121BA
:109BC000FAF7F6FC636B5A68D207F7D5616848F676
:109BD0005B7248680968D861C0F2010219605A6175
:109BE00010BD1B78012B31D03F20B021FAF750F97E
:109BF0004020B021FAF74CF94120B021FAF748F99A
:109C00004220B021FAF744F94FF46053C4F2020342
:109C10001A6C42F080621A64C8E71320B021FAF788
:109C200037F91420B021FAF733F91520B021FAF7EB
:109C30002FF91620B021FAF72BF94FF46053C4F234
:109C400002031A6C42F000721A64AFE74AF68020F1
:109C5000C0F60200FAF794FBC6E700BFAFF300803E
:109C600003291AD8DFE801F0110C0702436B98684A
:109C7000C0F300707047436B9868C0F3C0607047D2
:109C8000436B9868C0F380607047436B9B6813F028
:109C9000E05F0CBF0020012070470020704700BF2C
:109CA00010B4032925D8DFE801F02F2B2702436BDE
:109CB00003F5D073117888064CBFC1F30010C1F3CF
:109CC000001001F00F0154BF9488546859609168E6
:109CD00048BF400099604CBF40EAC4006405D168A9
:109CE0004CBF40F0040044EA400040F00102D9605B
:109CF0001A605DF8044B7047436B03F5C873D9E7EE
:109D0000436B03F5C073D5E7416B8B68C3F3016305
:109D1000183301EB0313CDE7AFF30080AFF30080FE
:109D2000012911D00AD3022906D1436B186910F01A
:109D3000030018BF0120704700207047436BDA68AA
:109D40009207F3D001207047436BD86810F00300EE
:109D500018BF0120704700BFAFF30080AFF3008051
:109D600010B4002930D1436BD968890735D0D3F8B6
:109D7000B041D3F8B411D3F8B831D360436BD3F802
:109D8000BC311361436B2020D860D868800743D072
:109D90001079C4F3400363F30410C4F3800363F346
:109DA00045101071002B31D09368E40864F31C0354
:109DB000936013795DF8044B080A61F30303090CFF
:109DC000137110705180704701292AD0022908BFF1
:109DD000436B05D05DF8044B704719698C07F9D0C7
:109DE000D3F8C041D3F8C411D3F8C831D360436B62
:109DF000D3F8CC311361436B2020186118698007B8
:109E000002BF586940F010005861C1E71389640D22
:109E100064F30A031381CCE7586940F002005861EB
:109E2000B6E7436BA3E700BFAFF30080AFF300805A
:109E300042F27010C2F20000FBF7CABFAFF300801D
:109E40000F29F0B429D9436853F83100C2073DD532
:109E50004FF47054C4F201040122A5688A401543EE
:109E6000A560D44310F0020F4FF47050C4F201000B
:109E700003EBC101C5684B6814BF15432540C5609D
:109E80007BB34FF47053C4F2010319680A431A609C
:109E90005A6814405C60F0BC704721F003024368CC
:109EA00002F1804202F59C3253F83100976801F0CC
:109EB0000304A4000F25A540C0F3031627EA0505F7
:109EC00006FA04F42C439460C207C1D44FF47055D1
:109ED000C4F201050122AE688A40D4432640AE6038
:109EE000C0E74FF47053C4F2010359680A435A6043
:109EF0001A6814401C60F0BC704700BFAFF30080CC
:109F00004FF47053C4F201030122186802FA01F100
:109F1000CA43104018605868104058609868104054
:109F20009860D8680240DA6059617047AFF30080EA
:109F300038B50378012B054614D0002404E0013421
:109F4000FFF77EFF172C0CD06B6853F8343013F0FA
:109F5000040F21462846F2D10134FFF7D1FF172C18
:109F6000F2D138BDFFF7ACFBE7E700BFAFF30080ED
:109F70004FF46053C4F202031A6B6FEA52226FEA85
:109F800042221A631A6D6FEA52226FEA42221A6560
:109F900000234168C4F202034FF480625960816873
:109FA0009960C168D9600169596141691962816923
:109FB000596201681960016AC4F202024FF4006339
:109FC0005160416A9160816AD160C16A5161016BDF
:109FD0001162416B5162C1691160C4F20203C16B2D
:109FE0005960016C9960416CD960816C5961C16C98
:109FF0001962016D5962816B4FF440621960816D85
:10A00000C4F202024FF480535160C16D9160016E41
:10A01000D160416E5161816E1162C16E5162416DBC
:10A020001160C4F20203416F5960816F9960C16F82
:10A03000D960D0F880105961D0F884101962D0F836
:10A0400088105962016F4FF4A0521960D0F8901037
:10A05000C4F202024FF4C0535160D0F894109160E2
:10A06000D0F89810D160D0F89C105161D0F8A010B1
:10A070001162D0F8A4105162D0F88C101160D0F8A1
:10A08000AC10C4F202034FF4E0525960D0F8B010A3
:10A090009960D0F8B410D960D0F8B8105961D0F8F0
:10A0A000BC101962D0F8C0105962D0F8A810C4F2E0
:10A0B00002021960D0F8C8305360D0F8CC309360F9
:10A0C000D0F8D030D360D0F8D4305361D0F8D83045
:10A0D0001362D0F8DC305362D0F8C4104FF4005350
:10A0E0001160D0F8E420C4F202035A60D0F8E820EE
:10A0F0009A60D0F8EC20DA60D0F8F0205A61D0F8FD
:10A10000F4201A62D0F8F8205A62D0F8E0201A60E1
:10A11000704700BFAFF30080AFF30080AFF3008063
:10A120002DE9F00F002302F00307C2F38006C2F30B
:10A13000C105C2F341144FF00F09C2F3C3124FF02F
:10A14000010A04E07600AD00A400BF00013303F073
:10A15000070C4FEA8C0C11F0010F02FA0CF809FA07
:10A160000CFC3CD0072B95BFD0F820B0D0F824B021
:10A170002BEA0C0C2BEA0C0C95BF4CEA08084CEAB5
:10A180000808C0F82080C0F82480D0F804C00AFA7B
:10A1900003F82CEA080C4CEA060CC0F804C04FF097
:10A1A000030B4FEA430CD0F808800BFA0CFC6FEA63
:10A1B0000C0C0CEA080848EA0508C0F80880D0F83A
:10A1C0000C800CEA080848EA0408C0F80C80D0F8B3
:10A1D00000800CEA080C4CEA070CC0F800C04908E3
:10A1E000B0D1BDE8F00F7047AFF30080AFF300804F
:10A1F00070B542F27815C2F20005F9F7F1FF6C6B09
:10A20000238BA68AB6B246EA0343082223F07F4393
:10A21000C0F2030293425ED027D80122C0F20302AB
:10A2200093424CD00222C0F20302934213D1A3887E
:10A23000EA6A23F400731B0412681B0CA3801368E2
:10A2400043F001031360A3889BB243F48053A380BF
:10A250005368012B65D916F00A0F18BF238BF9F745
:10A26000EFFFBDE87040F9F793BD8222C0F207020C
:10A27000934217D08422C0F207029342EBD1EB6ADB
:10A280001B685B6863B323882A8C9BB243F4A0638A
:10A2900042F001022A842380F9F7D2FFBDE8704022
:10A2A000F9F776BDA3882A6B23F400731B041268A8
:10A2B0001B0CA380136843F001031360CBE72B8CC6
:10A2C0001A0A0BD003F0010343F0F00302F0060278
:10A2D0001A432282BFE72B8CC3F347032382BAE7DA
:10A2E000A38823F400731B041B0CA38023889BB258
:10A2F00043F400732380202383F31188F9F728FFA8
:10A30000E86942F27813C2F2000320B100228262AF
:10A31000DA61FAF7C5F8F9F73BFF002383F31188F8
:10A3200099E7238823F480631B041B0C238092E7A6
:10A33000F8B542F27814C2F20004636B9D8AADB2A4
:10A34000F9F74EFF266B616B326805F45F4383F4C7
:10A350007F4383F0FF038B82136823F01F03136096
:10A360001368DF07FCD4377AE06A736802683D2619
:10A37000BE401E60136823F01F0313601368DE07DE
:10A38000FCD4067A426805F480733D20B0409BB24D
:10A39000106003B10123AA05A36044BF43F0020388
:10A3A000A3606F050ED58A8822F400721204120C85
:10A3B0008A80088880B243F0040240F400730B8066
:10A3C0001346A2602E0544BF43F00803A36068044F
:10A3D00044BF43F02003A360E90444BF43F01003EB
:10A3E000A3602A0444BF43F04003A36006D42BB902
:10A3F000F9F726FFBDE8F840F9F7CABC202383F33C
:10A400001188F9F7A5FEE06942F27813C2F2000361
:10A4100030B16FF0010282620022DA61FAF740F88F
:10A42000F9F7B6FE002383F31188F9F709FFBDE8B9
:10A43000F840F9F7ADBC00BFAFF30080AFF3008088
:10A4400010B542F27814C2F200042046FBF790FDEA
:10A45000064B4FF4A8420020C4F2000203F10C01A5
:10A46000E0616263E362216310BD00BFCCA9020812
:10A470002DE9F04F40F2A851C1F2000185B08A6980
:10A48000046D02914AF64033C0F60203936181469F
:10A49000202383F31188F9F71BFEC846A14698F8DC
:10A4A0000030012B06D0D8F85C3083B9D9F81430CD
:10A4B000DA060CD40299D9F818208B6942F0100200
:10A4C000C9F818200220C8F86430FAF741F8F9F703
:10A4D0001FFE002383F311884FF0000AD9F81430CF
:10A4E000DB0623D5D8F850703D6A05F4F013B3F5B8
:10A4F000802F34D0B3F5402FF0D105F00F0208EBD8
:10A500008202C5F30A13D26803339B08106AE5D0B0
:10A5100007F580570222396812B140F8041B013A4E
:10A52000013BF8D1D9F81430DB06DBD4D8F85C3025
:10A53000012101FA0AF11942019108BF0AF1010B48
:10A5400040F08780D8F854309B685FFA8BFA9A45C0
:10A55000C4D9202383F31188F9F7BAFD9FE705F0EA
:10A560000F0608EB860BC5F30A15DBF80C3098696B
:10A570000378E3B9021D1CCA0332D21AEB1C9B08F4
:10A580004FEA92021CBF07F58057A64606D03968ED
:10A5900012B14EF8041B013A013BF8D12C44C460BF
:10A5A000DBF80C309B699A682A449A6096E7C46885
:10A5B00007F580572846AE46002D2BD0032807D933
:10A5C00063692269934242D3E36803286361F7D841
:10A5D0003E68F0B16369002200E06369D10026FAA9
:10A5E00001F15D1C65611970636921698B4224BFAB
:10A5F000E3686361013802F101020CBF002301230B
:10A60000032A8CBF002303F00103002BE5D10028AF
:10A61000D4D17546202383F31188F9F759FDA36837
:10A6200020682B44A042A36009D0036823605C60CB
:10A63000F9F736FF002282622068A042F5D1FAF7CE
:10A640007FF8F9F765FD002383F31188A8E73E68DA
:10A65000C1E7202383F31188F9F73AFDD9F80820E0
:10A66000D8F85C30019922F0010223EA0103C9F80D
:10A670000820C8F85C30F9F74BFD002383F31188FC
:10A6800008EB8A020092D1684C69A36862689A421A
:10A6900040F2D480D8F85000098A4FEA4A17C51909
:10A6A000D21AD5F818398A4234BF15460D469BB2E6
:10A6B000B5EB830F0AF1010B9EBF4FEA0B32CDF8C9
:10A6C0000C9091462DD82378002B43D1EB1CD4F865
:10A6D0000CE09B08484418BF724604D052F8041B93
:10A6E000013B0160FAD10EEB0503E360009AD168EB
:10A6F0004C69A36862682B449A42A36040F29A8036
:10A70000D8F85000098AC519D21AD5F818398A42E2
:10A7100034BF15460D469BB2B5EB830FD3D9DDF898
:10A720000C900024202383F31188F9F7D1FCD9F889
:10A73000083043F00103C9F808302CB9D9F834388F
:10A7400001990B43C9F83438F9F7E2FC002383F38D
:10A750001188F7E600EB090AE4682A46AE4615B30D
:10A7600096083DD02569A169681AC31C30EA20000B
:10A7700028BF184683109E4238BF33464FEA830CE9
:10A78000CCEB02023BB1084650F8046B013BCAF81F
:10A790000060F9D16144A942A16148D3E368A36193
:10A7A000002ADDD17546202383F31188F9F790FC48
:10A7B000A36820682B44A042A36009D003682360EB
:10A7C0005C60F9F76DFE002383622068A042F5D13A
:10A7D000F9F7B6FFF9F79CFC002383F3118885E7AE
:10A7E0001646FAB12569A1690026334600E0A16941
:10A7F000481CA06191F800C0D9000CFA01F1A842F0
:10A8000046EA010624BFE168A161013A03F10103B0
:10A810000CBF00210121032B8CBF002101F001019D
:10A820000029E4D1CAF80060002A99D1BAE7002AC9
:10A83000DAD1B7E7DDF80C90012473E70AF1010BD8
:10A84000FAE700BFAFF30080AFF30080AFF3008002
:10A85000D1F808C000212DE9F0010D464FF08048E5
:10A860004FF0FF3713E00319C3F81059C3F8087904
:10A87000D2F8006B002EA8BFC2F8005B18DB0444BE
:10A8800001316145C4F8105BC4F8087B18D84C014D
:10A890000219D2F80039002BA8BFC2F80059E2DA39
:10A8A000C2F800891646D6F808399B07FBD5DAE7C7
:10A8B000C2F8008B1A46D2F8083BDE06FBD5DEE76D
:10A8C0004FF00113C0F81C38BDE8F001704700BF1D
:10A8D000F8B542F2B014C2F200042046FCF730FE94
:10A8E00004F1B4054AF63033C0F60203294604F1F8
:10A8F000680000264FF0A047FF22276563652666A3
:10A900006666F9F76DFF284604F5B8615522BDE883
:10A91000F840F9F765BF00BFAFF30080AFF30080E8
:10A9200070B50378066D012B82B0054601D002B0E8
:10A9300070BD42F2B013C2F20003984251D02B6EA8
:10A940000022EA65002B3DD04FF4A2520323C0F24F
:10A950002023C4F2000200204FF45021F260C6F818
:10A960000038C6F8000EB1632C6D2020FBF768F8A4
:10A97000012323612369DA07FCD40C20FBF760F87C
:10A980002369002BFCDA0024B460286D696DFFF7A1
:10A990005FFF6B68C6F81048DB68C6F81448C6F855
:10A9A0001C485BB143F20803B3614FF0FF3373619E
:10A9B000B36843F00103B36002B070BD4FF440537D
:10A9C000B361F2E74AF271430095C0F6000305F166
:10A9D00068004FF4AB610222F9F70AFF6866286647
:10A9E000B2E74FF46053C4F202030022596B41F006
:10A9F00080015963596941F08001596143205A61CE
:10AA0000E021F9F745FA9AE7AFF30080AFF3008051
:10AA1000F8B5046D202307462361226912F0200552
:10AA2000FBD10C20FBF70CF87B6D9E682A46FF21BA
:10AA30004FF0006504EB42130132B242C3F80059F3
:10AA4000C3F8005BC3F80819C3F8081BF2D94FF02C
:10AA5000FF324FF00113C4F81828C4F81C387B6D7E
:10AA60001A68BA651B6863623A6D10231361136933
:10AA700013F01005FBD10C20FAF7E2FFD4F80038F0
:10AA800023F4FE63C4F80038A0694AF6703240F43B
:10AA9000402048F24003C1F200030921C0F602023F
:10AAA00040F01000A061C4F81018C4F81418FA603F
:10AAB000C4F8105BC4F8003BC4F81059C4F800395E
:10AAC000BD6D7A6D05F11003BB655268934205D9DF
:10AAD0004AF65030C0F60200F9F752FC45F48015F2
:10AAE000A562F8BDAFF30080AFF30080AFF3008044
:10AAF000036D90F84E10D3F8002822F4FE6242EA6B
:10AB00000112C3F800287047AFF30080AFF3008054
:10AB10002DE9F84F0FFA81F900EB89074FF400484F
:10AB2000FB68046D1A6802F00302022A0D4606460D
:10AB300008BFC1F208080CD0032A08BFC1F20C08F4
:10AB400007D04146C1F20001C1F20408012A18BF32
:10AB500088466A01A018D9684FF0000EC0F810EBC3
:10AB6000002959D0588A05F15801490148EA0000E6
:10AB700060504FF0010ED4F81C0805F110010EFAD8
:10AB800001F10143C4F81C18224499680020C2F85E
:10AB9000100900295BD09A8B198AD6F858908B0837
:10ABA000012A88BF534303EB0901726DB1655268F6
:10ABB00091424FEA034A05F1FF3B26D80BF1400BC7
:10ABC00004EB8B0B4AEA0903CBF80430326DAB017E
:10ABD00043F02003136113699806FCD40C20FAF7A4
:10ABE0002FFFFB681A8A05F1480342EA85525B0190
:10ABF00042EA0802E2500122D4F81C3802FA05F5B4
:10AC00001D43C4F81C58BDE8F88F4AF65030C0F612
:10AC10000200F9F7B5FBD1E704EB491105F110008B
:10AC2000D1F800EB2EF4004EC1F800EBD4F81C185C
:10AC30004FF0010E0EFA00F021EA0001C4F81C18D2
:10AC4000224499680020C2F810090029A3D105F117
:10AC50003F0204EB82024FF48063C0F20023536092
:10AC6000326DAB0143F02003136113699906FCD4E4
:10AC700004EB49190C20FAF7E3FED9F8003923F464
:10AC80000043C9F80039D4F81C38012202FA05F54E
:10AC900023EA0503C4F81C38BDE8F88FAFF3008041
:10ACA0005831036D49015B5813F4004004D013F48C
:10ACB000001F0CBF02200120704700BFAFF30080CF
:10ACC0004831036D49015B5813F4004004D013F47C
:10ACD000001F0CBF02200120704700BFAFF30080AF
:10ACE00000EB8101CB681B6A19685B6811605360D7
:10ACF000704700BFAFF30080AFF30080AFF3008078
:10AD000000EB810330B4DC68A2695368136141B978
:10AD1000402B06D940252B465560C6F200033F253F
:10AD200002E05D1E43F0C043628A006DAC18B4FBC4
:10AD3000F2F200EB411143EAC243C1F8103B30BCD0
:10AD4000704700BFAFF30080AFF30080AFF3008027
:10AD5000F8B5076D07EB41130546D3F8084BC3F868
:10AD6000084B23070E4603D5D7F814381A0719D411
:10AD7000E30716D5D7F81438DC0712D505EB8603A0
:10AD8000DA68936959681869814211D36989D3686F
:10AD9000012000FA06F221EA02026A8131462846C1
:10ADA0009847F8BD00EB8103DB685B689847DFE7F5
:10ADB000411A002259609A6028463146FFF7A0FFE9
:10ADC000202383F31188F9F7C3F92B6D03EB4616A3
:10ADD000D6F8003B43F08063C6F8003BF9F7D8F99A
:10ADE000002383F31188F8BDAFF30080AFF3008038
:10ADF00000EB810330B4DC68626953681361A3B16E
:10AE000069B15D1E228A006DAC18B4FBF2F200EB52
:10AE1000411143EAC243C1F8103930BC7047402B9E
:10AE2000EFD9402353603F25ECE7036D03EB41115D
:10AE30004FF40023C1F8103930BC7047AFF30080E5
:10AE4000F8B5056D05EB41130646D3F80849E2074E
:10AE50000F46C3F8084903D5D5F81038DB0708D4E6
:10AE6000220605D50122D5F83438BA401A422ED12F
:10AE7000F8BD00EB8103DA685369D3F804E0D3F836
:10AE800010C0E64540D2CEEB0C0E0022C3F804E021
:10AE90009A60FFF7ADFF202383F31188F9F758F983
:10AEA000336D03EB47120120D2F8001941F0044141
:10AEB000C2F80019D3F8341800FA07F20A43C3F8AD
:10AEC0003428F9F765F9002383F31188C8E72023B4
:10AED00083F31188F9F73CF9F36DD5F83428706ED7
:10AEE000012101FA07F73B4322EA0707F365C5F89A
:10AEF000347818B1F9F7D4FA00237366F9F748F9F2
:10AF0000002383F31188F8BDB0F808E093684FF090
:10AF1000010C0CFA01F22EEA0202028198479FE727
:10AF200070B542F2B016C2F20006F9F759F9356D64
:10AF30006B69AC691C40E3046C6138D4A00448BF61
:10AF4000D5F80838210707D57368DB6823B142F2CA
:10AF5000B010C2F200009847E20633D46303D5F87C
:10AF6000185807D5EE0763D4A8076AD4690771D4C7
:10AF70002A0778D4230307D5EE0346D4AC034DD477
:10AF8000680338D4290305D4F9F75AF9BDE87040AD
:10AF9000F8F7FEBE42F2B010C2F200000321FFF744
:10AFA000D7FEF9F74DF9BDE87040F8F7F1BE30462D
:10AFB000FCF7BEFB73681B68002BBFD03046002136
:10AFC0009847BBE7202383F31188F9F7C1F8AB69F1
:10AFD000706E23F0100342F2B016AB61C2F20006AD
:10AFE00018B1F9F75DFA00237366F9F7D1F8002379
:10AFF00083F31188B2E742F2B0100221C2F20000DE
:10B00000FFF7A6FE2903BFD5C4E742F2B010C2F293
:10B0100000000021FFF79CFEAC03B1D542F2B01056
:10B02000C2F200000121FFF793FE6803AAD5E2E710
:10B0300042F2B010C2F200000021FFF701FFA807A2
:10B0400094D542F2B0100121C2F20000FFF7F8FEE1
:10B0500069078DD542F2B010C2F200000221FFF75D
:10B06000EFFE2A0786D542F2B010C2F2000003219B
:10B07000FFF7E6FE7EE700BFAFF30080AFF300808E
:10B08000036D03EB4111D1F8003B43F08063C1F83D
:10B09000003B7047AFF30080AFF30080AFF3008058
:10B0A000036D03EB411210B4D2F8004944F004449C
:10B0B000C2F80049D3F834285DF8044B012000FAA7
:10B0C00001F11143C3F83418704700BFAFF300809B
:10B0D000036D03EB4111D1F8003B43F40013C1F8B9
:10B0E000003B7047AFF30080AFF30080AFF3008008
:10B0F000036D03EB4111D1F8003943F40013C1F89B
:10B1000000397047AFF30080AFF30080AFF30080E9
:10B11000036D03EB4111D1F8003B23F40013C1F898
:10B12000003B7047AFF30080AFF30080AFF30080C7
:10B13000036D03EB4111D1F8003923F40013C1F87A
:10B1400000397047AFF30080AFF30080AFF30080A9
:10B1500042F28C724FF42053C4F20003C2F2000298
:10B160005321CA20136058625962DA68D10614D498
:10B17000DA6842F08002DA601946CA684FF4205358
:10B180005206C4F20003F8D5F922C0F27F021A6118
:10B190001A61DA6822F08002DA607047AFF300804B
:10B1A00042F28C7310B4C2F200031A68D3689C0692
:10B1B000FCD51369946A106852684860C3F30E03A3
:10B1C000181B4FF47A7404FB00F00133B0FBF3F367
:10B1D000CB600A605DF8044B704700BFAFF300809E
:10B1E0002DE9F043202385B0044683F31188F8F756
:10B1F0006FFF20466946FFF7D3FFF8F789FF00236A
:10B2000083F311889DE80C00C3F30231C3F30320DC
:10B2100001EB8109C3F3021103F00F0500EB4909AB
:10B2200001EB8108C2F30030C3F38051C2F3011473
:10B2300002F00F0C4FEA491905EB480804EB8404AF
:10B2400086004D000CEB44073044C2F3032C49EA5E
:10B250005808C2F303460D44C2F30352C3F301512D
:10B260000CEB400448EA07471436AD0001EB8101BE
:10B2700002EB820247EA445406EB420205EB41002E
:10B28000C3F3034344EA4262184442EAC02005B0D3
:10B29000BDE8F083AFF30080AFF30080AFF3008030
:10B2A000704700BFAFF30080AFF30080AFF30080C2
:10B2B00038B50446406A0268136823F01F03136020
:10B2C0001368D907FCD4057A216A43680A683D20CF
:10B2D000A8401860136823F01F0313601368DB078E
:10B2E000FCD46368087A4A681B683D21814011607C
:10B2F000CBB104222270204698472378042B12D029
:10B30000202383F31188F8F723FFA3682BB10022D1
:10B31000A26018469A62F9F7C3F8F8F739FF0023DC
:10B3200083F3118838BD02232370E9E7AFF300806F
:10B330002DE9F04142F2907342F29476C2F2000697
:10B34000C2F20003254F4FF6FF72304642F2C47539
:10B35000C2F200051A80FBF7FBFE4FF440511622A3
:10B36000462307F1240EC4F20101C0F20162C0F2CB
:10B370000163284642F2F474C2F20004F1613762BC
:10B38000C6F824E0B262F3624FF01608FBF7E0FE65
:10B3900046264FF46053A7F13002C4F20003A7F130
:10B3A0003C01C0F20108C0F201062046EB616A626E
:10B3B0002962C5F82880EE62FBF7CAFE4FF470538D
:10B3C000A7F16002C4F200030C3FC4F82880E662D3
:10B3D000E36122626762BDE8F08100BFF0A9020864
:10B3E00038B50378012B04461DD0C3696268A06A92
:10B3F0005289E16A20F4F04021F4F041150544BF80
:10B4000040F4205041F42051A062E16242F44172C4
:10B410000020072118801A8099801A8892B242F081
:10B4200040021A8038BD42F29475C2F20005A8426B
:10B4300015D042F2C475C2F20005A84231D042F2E2
:10B44000F475C2F20005A8424CD0216A626AE36931
:10B450000868116803F10C0282608A60C6E74BF24B
:10B46000B122C0F60002006A0A212346FDF790FBD4
:10B4700000286CD14BF2A12242F29473686AC0F6A4
:10B480000002C2F200030A21FDF782FB002857D117
:10B490004FF46053C4F202035A6C42F480525A646F
:10B4A000D3E74BF2B122C0F60002006A0A2123461C
:10B4B000FDF76EFB00283CD14BF2A12242F2C4738F
:10B4C000686AC0F60002C2F200030A21FDF760FBC1
:10B4D00040BB4FF46053C4F202031A6C42F4804242
:10B4E0001A64B2E74BF2B122C0F60002006A0A21E8
:10B4F0002346FDF74DFBC0BB4BF2A12242F2F47391
:10B50000686AC0F60002C2F200030A21FDF740FBA0
:10B5100020BB4FF46053C4F202031A6C42F40042A1
:10B520001A6492E74AF6DC30C0F60200F8F728FF0A
:10B53000CFE74AF6C830C0F60200F8F721FFBBE7B4
:10B540004AF6B430C0F60200F8F71AFFA0E74AF650
:10B55000A030C0F60200F8F713FF8BE74AF604406C
:10B56000C0F60200F8F70CFFD3E74AF6F030C0F659
:10B570000200F8F705FFBFE7AFF30080AFF30080EC
:10B580000378022B10B5044600D010BDC369006AD1
:10B5900000221A809A80FDF763FB606AFDF760FB6A
:10B5A00042F29473C2F200039C4215D042F2C4737B
:10B5B000C2F200039C4218D042F2F473C2F20003BC
:10B5C0009C4201BF4FF46053C4F202031A6C22F490
:10B5D000004208BF1A6410BD4FF46053C4F2020366
:10B5E0005A6C22F480525A6410BD4FF46053C4F276
:10B5F00002031A6C22F480421A6410BDAFF300807B
:10B6000043681A895B68012101FA02F292B25A83F7
:10B61000704700BFAFF30080AFF30080AFF300804E
:10B6200043681A895B68012101FA02F292B21A8317
:10B63000704700BFAFF30080AFF30080AFF300802E
:10B64000026A436A12681B6870B4866AC56A42F669
:10B65000240442F29070C2F20004C2F20000D460EE
:10B6600051601660D86059601D60116841F0010199
:10B6700011601A6842F001021A6070BC704700BF86
:10B68000F0B4046A476A866AC56A24683868E36069
:10B6900046F4806645F4806561602660C260416062
:10B6A0000560236843F001032360036843F001034E
:10B6B0000360F0BC704700BFAFF30080AFF30080C1
:10B6C000F0B4036A476AC66A1C68806A3B6842F63F
:10B6D0002405C2F2000546F48066E56061602060E2
:10B6E000DA6059601E60226842F0010222601A6826
:10B6F00042F001021A60F0BC704700BFAFF3008057
:10B7000070B4436A046A866A24681B68C06AE2608F
:10B7100042F2907546F48066C2F2000561602660D0
:10B72000DD6059601860226842F0010222601A68E8
:10B7300042F001021A6070BC704700BFAFF3008096
:10B7400008B5F8F74DFD42F62803C2F200030021C8
:10B750001878DA680428116107D102201870116086
:10B760001161D16821F0FF01D1605B6842F62800C9
:10B770005B68C2F200009847F8F762FDBDE8084038
:10B78000F8F706BBAFF30080AFF30080AFF30080A3
:10B7900042F62803C2F200034FF44062C4F20002F2
:10B7A0001846DA60FAF754BBAFF30080AFF30080BD
:10B7B00038B50378012B04461BD06268A168136872
:10B7C000B1FBF3F5013DADB205FB0333994206D061
:10B7D0004AF62040C0F60200F8F7D2FD6268117AFE
:10B7E000E368002208201A6058609D62D9601A61DF
:10B7F00038BD42F62803C2F200039842DDD14FF46F
:10B800006053C4F202030022196C41F0080119646C
:10B81000196A41F00801196232201A624021F8F7D2
:10B8200037FB4FF43D43C0F20153A360C5E700BFAF
:10B83000C368002201390120D96258615A621A6135
:10B84000D96805220143D9601A607047AFF30080C0
:10B85000C36800221A601A61DA6822F0FF02DA6017
:10B86000704700BFAFF30080AFF30080AFF30080FC
:10B87000C368426870B51D69DE68117D3540ADB2A0
:10B88000EEB2F64304461E6189B9AE0706D50378C9
:10B890000421032B017001D0D368984768071BD49B
:10B8A000EB0703D5636820461B69984770BDA9075D
:10B8B00006D50378032B03D00521936801709847C0
:10B8C0006A07EDD523780422032B2270E8D0636841
:10B8D0002046DB689847E3E72378032BE0D06368D2
:10B8E00005229B68227020469847D9E7AFF3008075
:10B8F00008B5F8F775FC42F68000C2F20000FFF7C9
:10B90000B7FFF8F79DFCBDE80840F8F741BA00BF63
:10B9100008B5F8F765FC42F68000C2F20000FFF7B8
:10B92000A7FFF8F78DFCBDE80840F8F731BA00BF73
:10B9300008B5F8F755FC42F63800C2F20000FFF7F0
:10B9400097FFF8F77DFCBDE80840F8F721BA00BF83
:10B9500008B5F8F745FC42F65000C2F20000FFF7C8
:10B9600087FFF8F76DFCBDE80840F8F711BA00BF93
:10B9700008B5F8F735FC42F66800C2F20000FFF7A0
:10B9800077FFF8F75DFCBDE80840F8F701BA00BFA3
:10B9900070B542F68004C2F20004204642F6380632
:10B9A000FAF7F6FAC2F20006002342F65005C4F296
:10B9B00001033046C2F20005E360FAF7E9FA42F605
:10B9C00068044FF080432846F360C2F20004FAF79F
:10B9D000DFFA4FF48063C4F200032046EB60FAF70D
:10B9E000D7FA4FF48043C4F20103E36070BD00BF97
:10B9F000F8B543681B7D012B044605D94AF6404043
:10BA0000C0F60200F8F7BCFC2378012B4CD0E368A9
:10BA100000221A605A639A635A626268A168566883
:10BA20009769B1FBF6F0451E27F0FF074FF0000CB9
:10BA3000B5F5803FC3F810C0DF6003D206FB00F00D
:10BA4000814207D04AF64040C0F60200F8F798FC61
:10BA5000E3686268117D1278ADB24FF6FF709D62A7
:10BA6000D86269B940F20120542198619960C2B14D
:10BA700013221A6203F13802343322616361F8BD84
:10BA80004FF481706421986199603AB131221A6251
:10BA900003F13402383322616361F8BD13221A6264
:10BAA000F6E731221A62E5E742F68003C2F20003AC
:10BAB0009C4213D042F63803C2F200039C4229D0C4
:10BAC00042F65003C2F200039C423CD042F66803A7
:10BAD000C2F200039C4245D0E3689EE74FF46053F6
:10BAE000C4F202030022596C41F001015964596A01
:10BAF00041F00101596219205A623021F8F7C8F962
:10BB00001B203021F8F7C4F94FF4F443C0F60323A7
:10BB1000A360E1E74FF46053C4F202030022196C02
:10BB200041F001011964196A41F0010119621C20F8
:10BB30001A623021F8F7ACF94FF43D43C0F20153DB
:10BB4000A360E36869E74FF46053C4F20203002284
:10BB5000196C41F002011964196A41F0020119627D
:10BB60001D20E5E74FF46053C4F202030022596C34
:10BB700041F480315964596A41F480315962182086
:10BB80005A62BEE7AFF30080AFF30080AFF30080EE
:10BB900008B50378022B00D008BD42F68003C268C6
:10BBA000C2F20003002198421160D16011611DD0E2
:10BBB00042F63803C2F20003984226D042F6500300
:10BBC000C2F2000398422CD042F66803C2F200038E
:10BBD0009842E1D11820F8F783F94FF46053C4F28A
:10BBE00002035A6C22F480325A64D5E71920F8F720
:10BBF00077F91B20F8F774F94FF46053C4F202038D
:10BC00005A6C22F001025A6408BD1C20F8F768F94A
:10BC10004FF46053C4F202031A6C22F001021A645A
:10BC200008BD1D20F8F75CF94FF46053C4F202031D
:10BC30001A6C22F002021A6408BD00BFAFF3008044
:10BC4000C36842685869117D10B440F001000024B7
:10BC500058611C61B1B9D16819B1D96841F00201CC
:10BC6000D960916819B1D96841F00401D9601269AD
:10BC70001AB1DA6842F00102DA6005221A605DF852
:10BC8000044B7047916819B1D96841F00201D9603D
:10BC9000D1680029E7D1EAE7AFF30080AFF3008075
:10BCA000C36800221A601A61DA6822F0FF02DA60C3
:10BCB000704700BFAFF30080AFF30080AFF30080A8
:10BCC00038B542F69805C2F20005F8F789FA2B69F3
:10BCD0001A69DC681440A4B2E2B2D2431A61A30725
:10BCE0002CD4600722D4210718D4E2060ED4E3072F
:10BCF00006D56B6842F698009B68C2F20000984730
:10BD0000F8F79EFABDE83840F8F742B86B6842F69B
:10BD100098009B6AC2F200009847E8E76B6842F619
:10BD200098001B6AC2F200009847DEE76B6842F693
:10BD300098009B69C2F200009847D4E76B682846D8
:10BD40001B699847CDE700BFAFF30080AFF30080D9
:10BD500008B5F8F745FA42F6AC00C2F200004FF41D
:10BD600080634268C4F201036FF0010192681961B7
:10BD70009047F8F765FABDE80840F8F709B800BF42
:10BD800010B5F8F72DFA4FF48063C4F201031A6975
:10BD9000DC681440A4B2E2B2D2431A61A30725D4EE
:10BDA00060071AD421070FD4E20607D542F6AC0388
:10BDB000C2F2000318465B689B6A9847F8F740FA9E
:10BDC000BDE81040F7F7E4BF42F6AC03C2F200034F
:10BDD00018465B681B6A9847E6E742F6AC03C2F276
:10BDE000000318465B689B699847DBE742F6AC03A3
:10BDF000C2F2000318465B681B699847D0E700BF92
:10BE000038B542F69805C2F20005284642F6AC0461
:10BE1000FAF766FEC2F200044FF40063C4F20003B6
:10BE200020462B61FAF75CFE4FF48063C4F20103F5
:10BE3000236138BDAFF30080AFF30080AFF3008023
:10BE40000378012B70B5044664D0036900221A60A0
:10BE50005A639A63DA631A645A626268E168166820
:10BE6000B1FBF6F0451EB5F5803F03D206FB00F0AE
:10BE7000814207D04AF66040C0F60200F8F780FA27
:10BE8000626823692489D168D06A013C01F00F01FE
:10BE9000A4B2ADB201299D62DC62586003D00229D0
:10BEA0000CBF03210021506900F00F0001282ED0A3
:10BEB00002282AD0D06900F00F00012822D00228E1
:10BEC0001ED0506A00F00F00012803D0022803D1D1
:10BED00041F4005141F48051106B9268196220F0D6
:10BEE000FF00002A18BF40F00100012500244FF494
:10BEF000004185225D611C61D86059641A6070BD83
:10BF000041F4007141F48071DBE741F0200141F020
:10BF10001001CFE742F69803C2F2000398420BD01B
:10BF200042F6AC03C2F2000398421DD0236946F6E4
:10BF300068029A61DA6190E74FF46053C4F2020339
:10BF40000022196C41F004011964196A41F00401DE
:10BF500019621E201A627021F7F79AFF4FF43D43D1
:10BF6000C0F20153E360E1E74FF46053C4F202030F
:10BF70000022596C41F002015964596A41F00201F2
:10BF800059622C205A627021F7F782FF2E2070210F
:10BF9000F7F77EFF4FF4F443C0F60323E360C5E7F1
:10BFA0004FF48053C4F201039A8992B242F08002A6
:10BFB0009A817047AFF30080AFF30080AFF3008049
:10BFC0004FF48843C4F200039A8992B242F080028F
:10BFD0009A817047AFF30080AFF30080AFF3008029
:10BFE0004FF49043C4F200039A8992B242F0800267
:10BFF0009A817047AFF30080AFF30080AFF3008009
:10C000002DE9F041456FB5F80C802C88A4B2E2050B
:10C0100006461FFA88F85BD4202383F31188F8F7CB
:10C0200097F814F02F0F2DD0371D08E0A988A0062F
:10C0300089B21ED42C88A4B214F02F0F22D023076B
:10C04000F4D014F0080F14BF80210021E00748BF8E
:10C0500041F02001A20748BF41F04001630748BFFB
:10C0600041F480713846F8F7C3FEA988A00689B26A
:10C07000E0D5C9B23046FAF733FE2C88A4B214F0EA
:10C080002F0FDCD1F8F784F8002383F3118818F020
:10C09000800F01D022062ED4630601D4BDE8F081C2
:10C0A000202383F31188F8F753F8726CB36C9A422B
:10C0B00035D04FF6BF7308EA03034FF6BF72AB816A
:10C0C0002A80F8F765F8002383F31188BDE8F08132
:10C0D000202383F31188F8F73BF8301D4FF40071EB
:10C0E000F8F786FEF8F754F8002383F311884FF62B
:10C0F000FF632B8090E7202383F31188F8F728F85B
:10C1000006F13000F9F704F80028A4BF80B2A88037
:10C110000DDBF8F73DF8002383F31188BCE7B36B20
:10C12000002BC6D0301D1021F8F762FEC1E7301D8C
:10C130000821F8F75DFE28F0C00343F04003AB810F
:10C14000E7E700BFAFF30080AFF30080AFF30080FC
:10C1500008B5F8F745F842F6C000C2F20000FFF754
:10C160004FFFF8F76DF8BDE80840F7F711BE00BFC4
:10C1700008B5F8F735F842F63810C2F20000FFF7BC
:10C180003FFFF8F75DF8BDE80840F7F701BE00BFD4
:10C1900008B5F8F725F842F6B010C2F20000FFF734
:10C1A0002FFFF8F74DF8BDE80840F7F7F1BD00BFE5
:10C1B00070B542F6C006C2F200064BF6A1723046D8
:10C1C000C0F60002002142F63815FAF731FDC2F23E
:10C1D00000054FF480534BF6C172C4F201032846A8
:10C1E000C0F60002002142F6B0147367C2F20004E8
:10C1F000FAF71EFD4FF488434BF6E172C4F20003D8
:10C200002046C0F6000200216B67FAF711FD4FF4DB
:10C210009043C4F20003636770BD00BFAFF30080BA
:10C2200038B54AF68044037AC0F60204002918BFE4
:10C230000C46012B054631D06B6F4FF4A0514FF4E3
:10C240008052C4F20102C4F20101934218BF8B4232
:10C250000BBF216821684FF43D424DF680620CBF50
:10C26000C0F20152C0F28022B2FBF1F292B21A8106
:10C27000A288E188208942F4045241F0400442F04F
:10C280002C0240F0010092B2A4B280B200211C82C4
:10C2900098829A8119801A889B8838BD42F6C0031B
:10C2A000C2F20003984218D042F63813C2F20003DB
:10C2B00098421FD042F6B013C2F200039842BBD19D
:10C2C0004FF46053C4F2020327201A6C42F4802218
:10C2D0001A64C021F7F7DCFDAEE74FF46053C4F2F7
:10C2E000020325205A6C42F010025A64C021F7F76D
:10C2F000CFFDA1E74FF46053C4F2020326201A6C6D
:10C3000042F400321A64C021F7F7C2FD94E700BF7F
:10C31000FCF756BDAFF30080AFF30080AFF30080B1
:10C3200001207047AFF30080AFF30080AFF30080CF
:10C3300000207047AFF30080AFF30080AFF30080C0
:10C34000704700BFAFF30080AFF30080AFF3008011
:10C3500010B5022408B1204610BD48F64463C2F26D
:10C36000000318461C79053C18BF0124FFF7E0FFC5
:10C370000028F0D044F00404E4B2204610BD00BF11
:10C3800010B5022408B1204610BD48F64463C2F23D
:10C39000000318461C79053C18BF0124FFF7C8FFAD
:10C3A0000028F0D044F00404E4B2204610BD00BFE1
:10C3B00010B50C4682B010B1042002B010BD48F692
:10C3C0004460C2F200000179052918BF0320F4D1AE
:10C3D00011460193FAF764F9019B90B91BB912E079
:10C3E00013F0FF030FD048F644602146C2F200006C
:10C3F0000193FAF795F9019B04F50074013B0028BD
:10C40000EED00120D9E748F64460C2F2000002B045
:10C41000BDE81040FAF7CCB9AFF30080AFF300806D
:10C4200030B50D4683B010B1042003B030BD48F6DE
:10C430004464C2F200042179052918BF0320F4D115
:10C44000204601920093FFF773FF019A08B1022082
:10C45000EBE720461146FAF7FBF9009B90B91BB9B0
:10C4600012E013F0FF030FD048F644602946C2F2F1
:10C4700000000093FAF72CFA009B05F50075013BCC
:10C480000028EED00120D0E748F64460C2F2000058
:10C4900003B0BDE83040FAF773BA00BFAFF30080D5
:10C4A00008B10420704729B10229FAD14FF4007372
:10C4B0001380704708467047AFF30080AFF30080E9
:10C4C00042F28C70C2F20000FAF752BBAFF3008068
:10C4D00001460020F8F7FCBEAFF30080AFF3008008
:10C4E000F8F73EBFAFF30080AFF30080AFF30080FA
:10C4F0002DE9F041C56A8D4204460E4602D003790B
:10C5000073B916B90020BDE8F081607804F13001FC
:10C5100032460123FFF74CFF20BBE662BDE8F08105
:10C5200000F13008414640782A460123FFF778FFA2
:10C53000C0B9E369226A20711A449542E1D2E778D2
:10C54000012F01D8DDE7E3691D44013F2A466078E9
:10C5500041460123FFB2FFF763FF012FF3D1002E05
:10C56000D0D0D2E70120BDE8F08100BFAFF300805A
:10C5700038B504460A46407804F130010123FFF73C
:10C5800017FF08B1032038BD94F82F1294F82E221B
:10C590004AF6552342EA012212B2CFF6FF739A42BD
:10C5A00018BF022000D038BD94F8683094F8695064
:10C5B00094F8661094F867201B0443EA05630B4364
:10C5C00043EA022244F2461322F07F42C0F25403AF
:10C5D0009A42E8D094F8842094F8855094F8821018
:10C5E00094F88300120442EA05620A4342EA0020FA
:10C5F00020F07F40C01A18BF012038BDAFF3008083
:10C600002DE9F04103681C78303C092C154602D80E
:10C610005A783A2A18D042F62C23C2F200031C683A
:10C620000C6074B12378B3B16078FFF7A9FEC2073C
:10C6300011D405B310F0040F0CBF00200A20BDE890
:10C64000F0810C20BDE8F08102330360002CE2D0C1
:10C650000B20BDE8F081002020706070FFF778FEAD
:10C66000C30702D50320BDE8F0813DB1470705D5DA
:10C670000A20BDE8F0812846BDE8F081204600216F
:10C68000FFF776FF012818BF002506D0032800F029
:10C69000BA80C8B10D20BDE8F08194F8F231002BCA
:10C6A000F8D094F8F82194F8F91194F8F63194F848
:10C6B000F751120442EA0162134343EA0525294671
:10C6C0002046FFF755FFE1E794F83C2094F83B3013
:10C6D00043EA0223B3F5007FDCD194F8471094F8C5
:10C6E000463053EA01210DD194F8562094F85700B2
:10C6F00094F8543094F85510120442EA006213433F
:10C7000043EA012194F84000E161431EDBB2012BB2
:10C71000E070BFD894F83D20A270002ABAD0531E12
:10C720001342B7D194F8426094F8413043EA0623AB
:10C730001E072381AED194F8447094F8436056EA02
:10C7400007260FD194F852C094F8538094F85060A3
:10C7500094F851704FEA0C4C4CEA086C4CEA06060F
:10C7600046EA072694F83FC094F83E7057EA0C2733
:10C7700090D000FB01FC07EB13106044864289D384
:10C78000361AB6FBF2F2002A84D040F6F576B242B1
:10C7900040F2BC8006F57046B24200F29C80022650
:10C7A000023228442F44A261A0622762002B3FF48A
:10C7B00071AF022E1CBF03235343674418BF02F01E
:10C7C000010267620EBF520002EB5302012602F221
:10C7D000FF12B1EB522FFFF45DAF4FF0FF32002399
:10C7E000032E2261E36011D042F62823C2F2000337
:10C7F00000201A882670013292B220711A80E280DD
:10C80000E062BDE8F0810120BDE8F08194F861109C
:10C8100094F86020637142EA01222A4462616078E0
:10C8200004F130010123FFF7C3FD0028DCD194F8A7
:10C830002F1294F82E224AF6552342EA012212B210
:10C84000CFF6FF739A42CFD194F8322094F8330098
:10C8500094F8303094F83110120442EA00621A431E
:10C8600045F2522342EA0122C4F261139A42BBD13B
:10C8700094F8162294F8170294F8143294F81512CA
:10C88000120442EA00621A4347F2722342EA01228A
:10C89000C6F241139A42A7D194F81E7294F81A5224
:10C8A00094F81F8294F81BC294F81C2294F8183252
:10C8B00094F81D0294F819123F042D0447EA086702
:10C8C00045EA0C653A432B4342EA002243EA01233E
:10C8D000E260236188E7023228442F44A261A0620B
:10C8E0002762002B7FF4D6AE94F85E6094F85F70F8
:10C8F00094F85C3094F85D00360446EA07663343EA
:10C9000043EA002392006362032660E7012647E7BB
:10C9100008B508B103780BB9092008BDC3888B425C
:10C92000FAD14078FFF72CFD10F0010F0CBF00206A
:10C93000032008BDAFF30080AFF30080AFF30080A9
:10C94000F8B50378022B04460D4646D0032B28D0B9
:10C95000012B02D04FF0FF30F8BD016A05EB550600
:10C9600001EB5621FFF7C4FD0028F3D1C6F30803FD
:10C97000216A2344013601EB5621204693F830709A
:10C98000FFF7B6FD0028E5D1C6F308063444E907F1
:10C9900094F8303047EA03204CBF0009C0F30B0085
:10C9A000F8BD016A01EBD511FFF7A2FD0028D1D136
:10C9B000AD0005F4FE7505F1300323442C44D8780E
:10C9C00099785A7894F83030000640EA014040EAFD
:10C9D0000220184320F07040F8BD016A01EB1521D8
:10C9E000FFF786FD0028B5D16D0005F4FF756319CA
:10C9F0001C4693F8303094F8310043EA0020F8BD2B
:10CA0000836870B50446012B0D46E18003D00068B1
:10CA10008269934201D3022070BDB3B90378032B1E
:10CA200010D003890022AB42E260F4D9436A03EBE1
:10CA30001513236105F00F0500EB451030306061E0
:10CA4000002070BD436A002BEBD086783601B542DA
:10CA500019D3012BDFD9AD1B9A42ADB2DBD908E067
:10CA6000012BD8D9206882699A42D4D9AE420AD81B
:10CA70000D461946FFF764FFA91B0346013089B232
:10CA8000EED1012070BD991E023A9142E3603BBF96
:10CA90008278836A002102FB013101EB15112161CB
:10CAA000C8E700BFAFF30080AFF30080AFF30080B2
:10CAB000F8B50378022B04460D4616465BD0032BCF
:10CAC0003AD0012B18BF022002D001232371F8BDF8
:10CAD000216A05EB550701EB5721FFF709FD0028F7
:10CAE000F3D1C7F30803234415F0010518BF93F8E9
:10CAF0003010F2B21EBF01F00F0141EA0212D2B2B1
:10CB0000216A83F830200137012301EB572123717B
:10CB10002046FFF7EDFC0028D7D1C7F30807002D0A
:10CB20003DD12744C6F3032697F8303023F00F0396
:10CB30001E4387F83060C8E7016A01EBD511FFF7A3
:10CB4000D7FC0028C1D1AD0005F4FE7505F1300316
:10CB500023442544DA78120602F070421643C6F3E5
:10CB60000727310C320E85F830605F709970DA70EB
:10CB700001232371F8BD016A01EB1521FFF7B8FC11
:10CB80000028A2D16D0005F4FF756219C6F30723D2
:10CB900082F83130012382F830602371F8BDC6F38A
:10CBA00007162744C5E700BFAFF30080AFF300804E
:10CBB000F8B506460F4669B9C5688369CDB9012540
:10CBC0002C460134A34217D8012D25D9022B52D867
:10CBD0000120F8BD0129FBD983699942F8D2FFF7FA
:10CBE000AFFE0128F4D9B369834298BF3D46E7D927
:10CBF000F8BD9D42E3D2E3E7012CE9D93046214656
:10CC0000FFF79EFE50B1B0F1FF3F18BF0128EFD0F3
:10CC1000A54201D0B369D4E70020F8BDB3699C42B6
:10CC2000D6D2304621466FF07042FFF741FFD0F177
:10CC3000010338BF0023002F08BF00234BB1012F91
:10CC4000C6D9B3699F42C3D2394630462246FFF760
:10CC50002FFF58B93369F4605D1C05D00122013BF8
:10CC6000727133612046F8BD2046C1E70128AFD17B
:10CC70004FF0FF30F8BD0224C0E700BFAFF30080E3
:10CC80002DE9F047C5880135ADB204460E4615B909
:10CC90000420BDE8F0870369002BF9D015F00F07D9
:10CCA00008D0036803EB471330336361E58000204D
:10CCB000BDE8F087C16801330361036861B19A7808
:10CCC000013A12EA1512EDD1012902D99A6991426D
:10CCD00006D30220BDE8F0871A89AA42D8D9E1E735
:10CCE0001846FFF72DFE01288046F2D9B0F1FF3F2C
:10CCF0001BD023689A6982420AD8002EC8D01846F1
:10CD0000E168FFF755FF804690B90720BDE8F0873E
:10CD1000861E023A9642C4F80C803BBF99789A6A04
:10CD2000002601FB06262661BCE70120BDE8F0874E
:10CD30000128CED0B0F1FF3FF7D020680021FFF7E7
:10CD4000D7FB0028F1D12268014602F1300302F539
:10CD50000C7203F8011B9342FBD122689369A8F17E
:10CD60000206023B9E423BBF936A9178002301FB7F
:10CD70000633D3624FF000094FF0010A0EE082F84B
:10CD800004A02068FFF7B4FB09F101090028CCD109
:10CD90002268D36A01335FFA89F9D36290784845F3
:10CDA0004FF000011346EAD8D16A9269C9EB01013C
:10CDB000D962AEE7AFF30080AFF30080AFF300803D
:10CDC0002DE9F04FFF2785B0DFF850810546B946C1
:10CDD0004FF6FF7609E00F2942D04FF0FF092846B1
:10CDE0000021FFF74DFF002837D128682969FFF798
:10CDF0007FFB002831D16C692378002B75D0E27A53
:10CE0000E52B02F03F01E8D01207E4D40F2927D028
:10CE1000B9F1000F11D19C46224604F10A090346DC
:10CE200001E012F801CFD90141EA53035CFA83F320
:10CE30004A45DBB2F5D1BB420FD0AB692E84DA7A1A
:10CE4000D20758BF04F10B0CC7D414F8011B13F818
:10CE5000012B9142C1D16445F7D105B0BDE8F08FF7
:10CE6000EA69002ABBD058063BD5E988677B29844C
:10CE700003F0BF0994F80DA0BA45AED12378264F30
:10CE800023F04003013B03EB430C03EB8C0C4FF00E
:10CE9000010B03E0B04235D147452AD017F8013FD6
:10CEA000E018E35C407843EA0020BBF1000FF1D0CA
:10CEB0000CF101030192CDF808C0039301F0B0F822
:10CEC000DDF808C0019ABCF1FE0F83461AD832F88B
:10CED0001C0001F0A5F88345019A13D1DDF80CC0C0
:10CEE000DAE74B457FF479AFC4E7042005B0BDE82D
:10CEF000F08F2378590609D5BBF1000F06D032F820
:10CF00001C301BB157464FF0FF0968E709F1FF39A4
:10CF10005FFA89F9574662E72FAE02083CAE020875
:10CF20002DE9F04F0B782F2B18BF5C2B89464FF063
:10CF3000000408BF01F101098460054699F800006A
:10CF40001F2888BF4AF6905785B084BFA046C0F618
:10CF5000020740F26D815C2818BF2F2809D109F122
:10CF600001039946013399F800002F2818BF5C2867
:10CF7000F7D02F2818BF1F28EE698CBF002401248A
:10CF800031D95C2851D00121A6F1020BCA460124F7
:10CF900001F01EF818B37F280CD822281FD04AF6BB
:10CFA0001062C0F6020201E0984218D012F8013F68
:10CFB000002BF9D12BF8020F1AF8010F2F2818BFF8
:10CFC0001F2804F1010310D95C282FD0B3F5807F0E
:10CFD00005D001211C4600F0FBFF0028DBD1062014
:10CFE00005B0BDE8F08F002401231F28994498BFA5
:10CFF0004FF0040B1BD8002CF1D004F10043013B8F
:10D000005A0036F813302E2B18BF202B12D1931C48
:10D01000334407E033F8042C2E2A18BF202AA3F14A
:10D02000020307D1013CF5D1D9E7012399444FF020
:10D03000000BE0E7AB6926F8148003F10B0106EB67
:10D04000440E202203F8012B8B42FBD13388202B86
:10D0500018BF2E2B14BF4FF0000A4FF0010A40F00A
:10D06000F38032464FF0000A32F8020F202818BF32
:10D070002E280AF1010AF7D04BF0030B734633F860
:10D08000022D2E2A01D0013CF9D100239C46082212
:10D090000AF1010A00B3202864D0B4EB0A0E18BFCD
:10D0A0004FF0010E2E2814BF00210EF001010029BF
:10D0B00058D1544518BF934234BF0021012162D397
:10D0C0000B2A00F0C380BEF1000F00F09080A24553
:10D0D0004BF0030B40F28B80AB691978E52902BF56
:10D0E00005211970AB69082A04BF4FEA8C0C5FFA5E
:10D0F0008CFC0CF00C020C2A00F081800CF0030177
:10D1000003297CD01BF0020F0AD10CF0030CBCF1F8
:10D11000010F08BF4BF0100B042A08BF4BF0080B9F
:10D1200083F80BB028460021FFF76AFCF8B92846BF
:10D13000FFF746FEAB69DB7AD8B95C073FF550AF25
:10D140006B69DA7AD1067BD5587D1A7DD97E9B7EB4
:10D1500042EA002243EA012343EA0243AB6099F822
:10D160000000F8E64BF0030B36F81A0090E7AB69C5
:10D17000DB7A04287FF434AF13F0040F08BF0520D6
:10D1800005B0BDE8F08F7F2819D82B2828D04AF6A3
:10D190001C6EC0F6020E01E0884221D01EF8011F6D
:10D1A0000029F9D1A0F1410189B219299CBF4CF0A5
:10D1B000020CC0B22CD8A969C8540133D4E701923B
:10D1C0000293CDF80CC000F003FF01AA92E80C1006
:10D1D000C0B138444BF0020B10F8800C0028D4D1B9
:10D1E0004BF0030B5F20A969C8540133BCE74FEA39
:10D1F0008C0C5FFA8CFCA2460B220823B4E74BF0A0
:10D20000020B7FE74BF0020B4BF0030B5F20EAE7CA
:10D21000A0F1610189B2192998BF2038A9698CBF92
:10D22000C0B2C0B2C85498BF4CF0010C01339BE7A8
:10D2300028462146FFF7E4FB6C6105B0BDE8F08F9E
:10D24000052005B0BDE8F08F184617E74BF0030B3B
:10D2500042E700BFAFF30080AFF30080AFF3008080
:10D2600070B401F10B0683B0044611F8015BB142C2
:10D2700004F8015BF9D1052B0CD9148800E00C46A9
:10D28000D90341EA530332F8021F14FA83F39BB225
:10D290000029F4D1072203F00F0404F13001013A10
:10D2A00000AD3929154488BF04F137011B096970A5
:10D2B000F1D102A911447E2401F8084CE2B10178B1
:10D2C000202908D0014603E011F8014F202C02D09C
:10D2D00001339342F8D1072A9BBF02A98918202164
:10D2E00011F8081CC15403F1010398BF0132072B48
:10D2F000F1D903B070BC70471346ECE7AFF3008080
:10D3000008B10B20704742F62C23C2F200031A68C2
:10D3100002B1107009B100220A7019600020704734
:10D320002DE9F04F95B014AB914643F8441D00220F
:10D3300002600BA909F01E0204461846FFF760F9C7
:10D3400007464FF40070FFF7C3F805461120002D83
:10D3500000F0E88005AB1295119309F01F06002F2D
:10D3600000F08F8019F01C0F00F02B81042F40F08B
:10D370002881DDF844A0DDF8489052460DF11F03E6
:10D380000DF12B0012F8011B03F8011F8342F9D1A4
:10D390009DF82B30DA072BD500238AF80B304FF09D
:10D3A000010812930BE0FFF70BFD08F10108074697
:10D3B0001FFA88F888B9B8F1640F00F01081504660
:10D3C00008A94A464346FFF74BFF0BA80021FFF789
:10D3D00017FB07460BA8002FE5D0042F40F0F18083
:10D3E0009DF82B308AF80B309DF82B30CDF8489003
:10D3F0009B0758BF4FF0010915D5B9F8003033B17C
:10D40000002301339BB239F81320002AF9D14EF6DC
:10D410004F421933C4F6C46282FB0302DB17C3EB2D
:10D42000A2091FFA89F90BA80021FFF7E9FA0746BC
:10D43000002840F0C68023468246544698460BE0BA
:10D440000CB9BDF832A094B24C4500F00781FFF74B
:10D4500017FC0746002868D10F990B98FFF748F88A
:10D460000746621C0BA80121002F5ED1109B1B7880
:10D47000E52B18BF002B14BF00230123E0D01C466E
:10D48000E5E70BA80399FFF74BFDDDF84080074661
:10D4900000287FF467AFB8F1000F00F09B8019F00F
:10D4A0001C0F40F07F8198F80B30DA0600F1908075
:10D4B00019F0020F40F0908009F00803DBB2DDF8AC
:10D4C0002CA00BB146F02006DAF82C30C4F82080EE
:10D4D0002846E361FFF704F8A67198F8155098F80C
:10D4E0001A0098F8141098F81B200B9B41EA0521AC
:10D4F00040EA022242EA0142226198F81E6098F84E
:10D500001F5098F81C0098F81D10DA882360330427
:10D5100043EA0563034343EA01230020E360A2805A
:10D52000A060A06115B0BDE8F08F444646F0080643
:10D53000DDF84080002F44D1370758BFDDF82CA01C
:10D54000C2D5FEF7BDFF98F81A3098F815C098F8C4
:10D55000141098F81B20DDF82CA088F80E0043EA80
:10D56000022241EA0C210023C0F3072E070C4FF0E2
:10D570000109000E52EA014B88F80FE088F810709C
:10D5800088F8110088F80B3088F81C3088F81D30B6
:10D5900088F81E3088F81F3088F81A3088F81B3059
:10D5A00088F8143088F815308AF804908AD0DAF8B0
:10D5B0002C30CB45009303D0DAF818309B4510D3BC
:10D5C00002272846FEF78CFF384615B0BDE8F08FDD
:10D5D0000427F6E70627C5E6DF077FF56DAF0727C7
:10D5E000EFE7019627465E4621E00128E8D00130AA
:10D5F00000F0D680DAF818209642E1D23146504643
:10D600000022FFF755FA002840F0D880DAF81030F1
:10D61000591C1CBF0133CAF81030DAF8183018BF93
:10D620008AF80590A34209D9012CC9D9264650464B
:10D630003146FFF785F904460028D6D10B980099AA
:10D64000019E0BF1FF33C360FEF752FF3C46DDF84D
:10D650002CA0074600283FF435AFB2E7B9F1010F1F
:10D66000444671D051460BA8FFF7CAF90746002877
:10D67000A7D1119B024603F10B0013F8011BD70140
:10D6800047EA520251FA82F28342D2B2F5D109F14D
:10D69000FF339BB24AF630698DE86000C0F602099C
:10D6A0004FF6FF784FF0FF0B16461D4602940B987D
:10D6B0000F99FEF71DFF0246002A6ED15FFA85FA28
:10D6C0000AF1FF31109CDDF848C0667301EB4100A0
:10D6D00001EB80014FF00F001346E0722273A27637
:10D6E000E2760EE03CF8113027184FEA132E23544F
:10D6F000013187F801E0002B08BF434601320D2AB3
:10D7000009D0434519F80200ECD1271804F800B0FD
:10D7100087F801B0F2E7434502D03CF811300BB96D
:10D720004AF0400A84F800A00B9B4FF001011971E8
:10D730000BA80021FFF7A4FA78BB013DADB2002D84
:10D74000B5D19DE86000029C0B980F99FEF7D0FEC2
:10D75000074600287FF435AFDDF840E00EF12002E7
:10D76000734603F8017B9342FBD1119B724603F190
:10D770000B0013F8011B834202F8011BF9D1119A27
:10D780000B9BD17A012201F018018EF80C101A714E
:10D7900046F00806DDF84080CEE6009D074610E71B
:10D7A00001270EE798F80B3013F0110F7FF417AF35
:10D7B00019F0040F3FF4C0AE082702E7074600E760
:10D7C0002DE9F04F07469B46002383B00C46CBF86B
:10D7D00000300068B9889146FFF79AF840B9BB79E4
:10D7E000190648BF022003D49A0758BF072002D465
:10D7F00003B0BDE8F08FFA68B96819EB020F07D3E0
:10D80000914243F0200388BFF960BB710020EFE72D
:10D81000B9F1000FF4D007F12403019307F509785B
:10D82000C1F30805002D67D13B689D78013D05EAED
:10D83000512515F0FF050DD1002940F0868038698B
:10D84000002800F08D80012800F09D80461C76D0D5
:10D850003B687861BA79510664D479699A69A1F113
:10D86000020C023A944580F08E8099789A6A0CFBFB
:10D870000122002A00F087805FEA592605EB020AA0
:10D880002FD0AA198A4288BFC5EB010658782146D5
:10D890005246F3B2FEF7C4FD002850D1BB69CAEB73
:10D8A000030C66450CD9019D04EB4C2313F8012BA6
:10D8B00005F8012B4545F9D1BB7923F04003BB7135
:10D8C0007202B968A318DBF8000011441044B9EBE8
:10D8D0000209B9601C46CBF80000A1D1FA68BB79F7
:10D8E0008EE7BA69B968524502D0FA68914240D3CE
:10D8F000C7F818A0C1F30805C5F500724A4528BF4E
:10D900004A463D44243523463AB1A31814F8016B26
:10D910009C4205F8016BF9D1B968B87940F0400034
:10D92000B871D0E75878BA6901990123FEF778FDFC
:10D9300028B9BA793B6822F04002BA718DE7BB7909
:10D9400063F07F03BB71012052E718467969FFF746
:10D950002FF900287FF477AFB968FA68BB794FE7F1
:10D9600018462946FFF724F9386100287FF46BAF89
:10D97000F2E75878019952460123FEF719FD002875
:10D98000DDD1B968B4E7BB7963F07F03BB710220D6
:10D990002EE700BFAFF30080AFF30080AFF300804D
:10D9A0002DE9F84F04460068A188FEF7B1FFD8B909
:10D9B000A27902F0200303F0FF00ABB150060DD5B1
:10D9C0002146A26951F8240B01234078FEF728FD77
:10D9D000002849D1A37923F04003A3712068E169AD
:10D9E000FEF786FD06460EB1BDE8F88F256AEB7A94
:10D9F00043F02003EB72E3682B77A3891B0A6B7754
:10DA0000E389AB77E37BEB772369AB76238A1B0A49
:10DA1000EB76638A2B75638A1B0A6B75FEF750FDE4
:10DA2000C0F30721020C030EA8752A76E9756B7600
:10DA3000A179236821F020010122A1711A712568C2
:10DA400031462846FEF754FD034650B92B78032B88
:10DA50000DD0002168780A46FEF722FD031C18BF8E
:10DA600001231846BDE8F88F0120BDE8F88F6B79D7
:10DA7000002BEED005F13001E8620B4605F50C7283
:10DA800003F8010B93424FF00004F9D12A69EB68C7
:10DA900085F81822C2F3072B4FEA124A4FEA134CBB
:10DAA0004FEA136E52204FEA1269C3F3072861222E
:10DAB00085F819B285F81AA24FF0410B4FF0720A9F
:10DAC0005527AA2685F81C3285F8300085F83100E4
:10DAD00085F8322085F8172285F81B9285F81D827B
:10DAE00085F81EC285F81FE285F82E7285F82F6230
:10DAF00085F833B085F816B285F814A285F815A21A
:10DB000068786A690123FEF78BFC6C71A1E700BF9E
:10DB100010B50446FFF744FF00B9206010BD00BFF8
:10DB200070B504460D460068A188FEF7F1FE002896
:10DB300054D1A3791E0663D4E268AA4203D213F03B
:10DB4000020F08BF15460023A268A360002D59D01C
:10DB500020688678760242B1013A691EB2FBF6F37C
:10DB6000B1FBF6F1994280F08A80216900294BD0FF
:10DB70006161002933D1A3680D46C3F30802002A6E
:10DB800000F08380A269AA427FD0A3795E0658BFC5
:10DB900004F124060DD5236804F124065878314693
:10DBA0000123FEF73DFCA379002837D123F0400381
:10DBB000A3712368314658782A460123FEF7F8FB03
:10DBC00058BBA368E268A5619A4206D2A279E360D5
:10DBD00042F02003A371002070BD002070BDB5424B
:10DBE00088BF206856D9A3799A07C6EB05051AD4D1
:10DBF000012902D982698A423DD863F07F03A3716B
:10DC0000022070BD284670BDFEF7D2FF01280146F4
:10DC10002FD0013018BF2161AAD1A37963F07F030F
:10DC2000A371012070BDFEF7C3FF0146002830D06C
:10DC30004B1CF2D001291CD920688369994218D263
:10DC4000A36861613344AE42A360CCD32B44C5F3D7
:10DC50000802A360DAB12668B0698A1E02388242DF
:10DC600007D2B078B16A00FB021202EB5525002AF8
:10DC700083D1A379C1E7FEF763FE0146D8E773427B
:10DC80001A40A260AD1A616973E7E2689CE7154625
:10DC900073E73546A368D9E7AFF30080AFF30080A0
:10DCA00070B586B006AB044643F8141D0022184632
:10DCB0002146FEF7A5FC08B106B070BD4FF4007018
:10DCC000FEF706FC05461120002DF5D003ABE561FB
:10DCD000A36120460199FFF723F906462846FEF77F
:10DCE000FFFBBEB963696BB1DA7AD20617D55D7DE9
:10DCF0001A7DD87E997E42EA052241EA002343EA52
:10DD00000243A3602368DB882046A3800021FEF73E
:10DD100077FE0646042E04D0304606B070BD0526B8
:10DD2000FAE70520C8E700BFAFF30080AFF300803B
:10DD30002DE9F04F044687B00E460068A188FEF733
:10DD4000E7FD0546002D76D1002E7AD04FF4007005
:10DD5000FEF7BEFB80461120B8F1000F6BD003AB7D
:10DD6000FF27A3610423C4F81C803D46DFF85092CE
:10DD70004FF6FF7A184608E00F2820D0FF252046EE
:10DD80000021FEF77DFF00284AD12169002900F01B
:10DD900090802068FEF7ACFB002841D163691A78B7
:10DDA000002A00F0E680E52A18BF2E2AD97AE5D0AD
:10DDB00001F03F000907DFD40F2840F0EA80500649
:10DDC0003CD5E1885F7B218402F0BF0593F80DE02C
:10DDD000BE45D3D11978D4F81CC0784A01F03F0170
:10DDE000013901EB410001EB8000012708E0FE282A
:10DDF00013D82CF810100F4601304A4500F0BB80B4
:10DE000012F8011F03EB010B595C9BF801B041EACA
:10DE10000B21002FEBD15145EFD07746FF25AEE720
:10DE200003460022042B226110D040460193FEF7E6
:10DE300057FB019B184607B0BDE8F08FAA429DD161
:10DE4000C4E720463146FEF7DBFDF4E706F10902A0
:10DE500000251570B76917B3F36903B32369DBB104
:10DE6000228C4FF6FF739A4216D0E369188898B156
:10DE700099460CE0F369013BAB4205F1010507EB64
:10DE8000050309D903F8010C39F8020F28B1002164
:10DE900000F09EF80028EDD1002500237B55204698
:10DEA0000021FEF7EDFE0428034604BF0023236192
:10DEB000BBE703460028B4D106F109020029C7D008
:10DEC000616991F80CC00CF0080E5FFA8EFE734683
:10DED000481E8E4606F11107194610F8013F202B07
:10DEE0000ED0052B08BFE523A3F14105EDB219B112
:10DEF000192D9CBF2033DBB202F8013BBA42ECD1B2
:10DF00009EF80830202B71461BD015462E230CF0AE
:10DF1000100E05F8043B5FFA8EFE0132C81D10F8A2
:10DF2000013FA3F14107202BFFB20AD0BEF1000F41
:10DF300003D0192F9CBF2033DBB202F8013BAA4269
:10DF4000EDD1CB7A33728D7FCF7F0B7F487F2D044D
:10DF500045EA07652B4343EA00233360487E0B7E86
:10DF600043EA0023B380C87D8B7D43EA0023F3801E
:10DF70006EE7042355E71B78590606D5FE289CBF9B
:10DF800000232CF810303FF648AF013DEDB2774644
:10DF9000F5E675B903F10A0001E013F8012FE90174
:10DFA00041EA550552FA85F58342EDB2F5D1BD42FD
:10DFB00002D04FF6FF73238421697DE72FAE02085C
:10DFC0003CAE0208AFF30080AFF30080AFF30080F7
:10DFD0007F2810B40DD979B90F4B02E0A1B2802986
:10DFE00016D033F8022F824201F10104F6D18031BC
:10DFF00088B25DF8044B7047FF2809D84BF2200324
:10E000008038C0F602035DF8044B33F81000704707
:10E0100000205DF8044B70471EB00208AFF300808B
:10E0200061280DD04BF22012C0F60202002101E05F
:10E03000834206D032F8023F0131002BF8D17047FD
:10E0400000214AF64063C0F6020333F8110070471E
:10E0500041F20073C2F2000318607047AFF3008012
:10E0600041F2047241F20073C2F20002C2F20003F4
:10E070004CF6FF110120C3F69A31107019607047F9
:10E0800041F6F403C2F200031B6893F8DD355B062A
:10E0900005D54BF2A033C0F602031B5C0BB100F0B8
:10E0A00097BF7047AFF30080AFF30080AFF30080FD
:10E0B00041F6F403C2F200032DE9F0411B68064665
:10E0C0000F46C3F83803F0B942F620730022C2F2BB
:10E0D0000003C7F6C0729A6197F881322BB144F2FF
:10E0E0005810C2F2000004F0D3F943F29003C2F2D8
:10E0F00000034BF2003132461868C0F60201BDE859
:10E10000F04117F0CDBAD3F8E00106F081FF07EE39
:10E11000106AF8EEC76A07EE100ADFED0F7A66EEB6
:10E12000876A9FED0E7AC6EEA77A42F62078C2F291
:10E130000008C7EE276A16EE900AF4F7A9FAA8239A
:10E14000A0FB034503FB015520462946F4F778F868
:10E15000C8F81800C0E700BF0000704200247449EE
:10E160002DE9F041054643F27C0086B0C2F2000082
:10E1700018F006FA00283BD043F29004C2F20004E3
:10E1800043F27C00C2F20000266818F0F1F98046E4
:10E1900005F0FEFE074616F0BBFD4BF22831C0F637
:10E1A000020142463B460090304617F079FA20685B
:10E1B00006F02EFE41F6E803C2F200031C68D4F814
:10E1C000FC3D1A6803925A6804929B6804F521701A
:10E1D000059302F025FA03AB0146D4F8002E009314
:10E1E0002846032307F024FD0023CBF68073AB639E
:10E1F00006B0BDE8F08100BFAFF30080AFF3008050
:10E20000086D0969F8B58318013B93FBF0F400FB36
:10E21000143391E81100896810F903C0E756CE560F
:10E220008056A5568C561CF1000318BF01230037F9
:10E2300018BF0127003618BF0126834204D00030E2
:10E2400018BF0120FFF71CFFAF4205D0002D0CBF07
:10E2500002200320FFF714FFA64207D0002C0CBFBA
:10E2600004200520BDE8F840FFF70ABFF8BD00BF55
:10E2700038B541F20073C2F200030C461B688B42B2
:10E2800041F204730546C2F200030CD01B784BB177
:10E290000CF0D6FE41F6F403C2F200031B68B3F99A
:10E2A00050301BB938BD00221A7038BD43F28000CF
:10E2B00029462246C2F20000BDE83840FFF7A0BF61
:10E2C000F0B541F6F402C2F2000243F29003126884
:10E2D000C2F200030C4689B01860D2F83803FFF789
:10E2E000E7FED4F8FC3D1A6805925A6806929B68CE
:10E2F00004F52170079302F093F94EF261164EF285
:10E3000071254FF0030E0246C0F60006C0F6000568
:10E3100005AF42F620704BF25831D4F8003ECDF8EC
:10E3200000E0029603950197C2F20000C0F60201D8
:10E3300007F0AEFC44F23C104EF2B1012246C0F6AA
:10E340000300C0F6000117F0CBFB4BF268304EF231
:10E3500051012246C0F60200C0F6000117F0C0FBD2
:10E360004BF284304EF261012246C0F60200C0F644
:10E37000000117F095FB09B0F0BD00BFAFF30080BE
:10E38000002303600268036003684260002BC1BF82
:10E39000D0ED007AF8EEE77A9FED157AC7EE277A8E
:10E3A000F0B4D8BF002310A5D5E900450146D8BF79
:10E3B000C7F6C0734FF00007D8BF83604FF0000668
:10E3C000C7F6C0774FF000024FF00003C8BFC0EDA2
:10E3D000027AC0E90445CE618E61C1E904238F60F1
:10E3E000F0BC7047AFF30080003CDD9BFFFFFFFFF8
:10E3F000ABC22248AFF30080AFF30080AFF30080E0
:10E40000F8B5044616F07CFC41F6E803C2F20003BE
:10E410001B68D3E90C2352EA030509D00EA7D7E9FC
:10E420000067821A61EB03039F4208BF96420ED237
:10E43000D4E904450AA3D3E90023001B61EB0501DD
:10E440008B4208BF824234BF00200120F8BD00206B
:10E45000F8BD00BFAFF30080FF6D0A1E0000000092
:10E46000FF79030A00000000AFF30080AFF30080E3
:10E4700041F6E803C2F2000310B51C682046FFF71E
:10E48000BFFF08B9E061206043F29C102168C2F22E
:10E49000000017F0CDFE44F2581041F2C41143F2CF
:10E4A0009C12C2F20000C0F60301C2F20002BDE8F5
:10E4B000104004F0B5B800BFAFF30080AFF30080A8
:10E4C00080697047AFF30080AFF30080AFF3008046
:10E4D000C0697047AFF30080AFF30080AFF30080F6
:10E4E000D0ED007A90ED017AF8EEE77AB8EEC77ACF
:10E4F000C7EE276A16EE900A704700BFAFF30080A0
:10E5000010B50446FFF77CFF08B9E0612060206881
:10E5100010BD00BFAFF30080AFF30080AFF3008009
:10E5200010B50446FFF76CFF08B9E061206022686F
:10E53000002A0BDD41F6F403C2F200031B68B3F9B5
:10E5400068009042D4BF0020012010BD002010BD03
:10E5500041F6E803C2F200031868FFF7E1BF00BF0D
:10E5600041F6E803C2F200031B689869704700BFD8
:10E5700041F6E803C2F200032DE9F041D3F8008030
:10E58000064640460F46D8E90445FFF739FF18B95B
:10E59000C8F81C00C8F80000D8F80080B8F1000FD7
:10E5A00016D030463946001B61EB0501F3F748FEF3
:10E5B00007EE108AF8EEC77A9FED087AC7EE277A41
:10E5C00007EE100AC7EE277A17EE900ABDE8F08131
:10E5D000DFED037A17EE900ABDE8F081809FD54BFE
:10E5E0000000C07FAFF30080AFF30080AFF3008086
:10E5F0002DE9F84341F6E806C2F200068146884656
:10E60000376816F07DFB4FF480520D46CEF20002C3
:10E610003168526840F2A85301F50E51C1F200036F
:10E6200004460A6298690DF00BFFB0F5807F49DD62
:10E63000B8F1000F0AD041F6EC03C2F200031B68E8
:10E64000D3F81033012B45D0BDE8F8833846FFF7E7
:10E65000D7FEC8B1D7E90423A21A65EB030352EA37
:10E66000030149D14FF0FF323B683A603A687B6062
:10E67000002A6CDDD7ED007A9FED3B7AF8EEE77A61
:10E68000C7EE277AC7ED027A41F6EC03BA69C2F207
:10E69000000301321B68BA61FA69D3F81033013202
:10E6A000012BFA61C7E9044556D033684FF4805214
:10E6B00003F50E53CEF20002196A5268511A5962DC
:10E6C000BDE8F8834BF2B030C0F60200BDE8F84375
:10E6D0001AF076BB29462046FFF74AFF4FF47A71BD
:10E6E00001FB098107EE901AF8EE677ABDE8F8435E
:10E6F00017EE901A03F0CCBD41F6F401C2F200010E
:10E7000046F2B7000968096ECBF20B6080FB01E0AE
:10E710000844C917C1EB20204FF418414FEAE079B3
:10E720004FEA400EC5F6D00101FB09EEA0FB010146
:10E730007144F3F795FF47F230539842C8BF4FF04A
:10E74000FF303B6838603A687B60002A92DC002327
:10E75000C7F6C073BB6097E729462046FFF708FF5E
:10E76000002103F095FDA0E7ABC22248AFF3008083
:10E7700010B54BF2BC3104464EF611002246C0F6ED
:10E780000000C0F6020100F0D3FA4EF2F1504BF255
:10E79000CC312246C0F60000C0F60201BDE81040B0
:10E7A00000F0C6BAAFF30080AFF30080AFF3008093
:10E7B00030B4013847F22E54A04207EE902A029D51
:10E7C000039A16D892ED027A67EE277A002217EEA6
:10E7D000900AC7F6C072904212D0FDEEE77A4BF273
:10E7E000FC300295C0F6020017EE902A30BC07F00C
:10E7F00007BD4BF2DC30C0F6020030BC1AF0E0BAC4
:10E800004BF2F030C0F6020030BC1AF0D9BA00BFAB
:10E81000F0B583B041B941F6F403C2F200031B68BE
:10E8200093F8D0359B0601D403B0F0BD41F6E8055E
:10E83000C2F200052C682046A669FFF7E1FD08B981
:10E84000E0612060206847F22E53421E9A42EBD8C6
:10E85000104F2C6846F26043C1F20003D3ED6F7A8B
:10E8600097ED007A06F00106710077EE277A43F201
:10E87000A8123144C2F2000200254EF2714302EBAD
:10E88000C101019417EE902A0095C0F60003FFF72E
:10E890008FFFC9E79C410120AFF30080AFF30080F8
:10E8A0002DE9F04F41F6F408C2F2000844F2C01618
:10E8B000D8F80030C2F2000687B0074618683568FD
:10E8C00012F096FFD8F800308246D3F80402D3F84D
:10E8D00000B004F0B5FCD8F8004043F2B831C2F201
:10E8E0000101D4F80422034691F8E80D049205933F
:10E8F00017F0AEFBD8F80010044691F8DD05C0F320
:10E90000801017F0A5FB059B049A009343F2E019D1
:10E910004BF21041039001925B4628465246C0F6E6
:10E920000201C2F20009029416F0BAFE4BF2504105
:10E93000D9F840313068D9F83C21C0F6020116F010
:10E94000AFFE97F88532002B40F08D81D7F8F44D5B
:10E95000D7F8EC2DD7F8F03D306800944BF2A04189
:10E96000C0F6020116F09CFED8F8003097F8850238
:10E97000D3F80442356817F06BFB4BF2C0410346F5
:10E9800022462846C0F6020116F08AFED7F8900209
:10E99000D6F800A0F3F720F80446D7F894020D4605
:10E9A000F3F71AF8CDE900014BF2E44122462B4679
:10E9B000C0F60201504616F073FE97F884023568DF
:10E9C00017F046FB049002F05BFC17F041FB044695
:10E9D00043F2E010C2F20000D9F83CB0D9F844A0EC
:10E9E00001F03EFFD8F800308146B3F95000003006
:10E9F00018BF012017F02CFB4BF200510390049A32
:10EA0000CDF800B02346CDF804A0CDF808902846F4
:10EA1000C0F6020116F044FE97F8842244F2C013B7
:10EA2000C2F20003002A40F0048141F6EC04C2F275
:10EA3000000435682368D3F828010AF051F84BF236
:10EA400070510246C0F60201284616F029FE2368DE
:10EA50003568D3F860010AF043F823688146D3F89B
:10EA60006C0104F0DDFC2268D2F8D0204BF28C510E
:10EA70000346009228464A46C0F6020116F010FEF0
:10EA800097F8853244F2C015C2F2000553B32368EB
:10EA9000D5F80080D3F82C010AF022F84BF2B851D7
:10EAA0000246C0F60201404616F0FAFD2368D5F88A
:10EAB0000080D3F864010AF013F8236842F6207549
:10EAC0008146C2F20005D3F8700104F0A9FCAD6CD8
:10EAD0004BF2D45103464A4640460095C0F6020127
:10EAE00016F0DEFD2368D6F80080D3F8580209F04E
:10EAF000F7FF23680546D3F85C0204F091FC4BF263
:10EB000000612A460346C0F60201404616F0C8FDE1
:10EB100023683568D3F8840109F0E2FF4BF22061E5
:10EB20000246C0F60201284616F0BAFD2368346892
:10EB3000D3F8880109F0D4FF4BF238610246C0F6E1
:10EB40000201204616F0ACFD46F6686307F50D5449
:10EB5000C2F200034BF2546107F50E571B68E26BDB
:10EB60003068C0F6020116F09BFD4BF274617A68C2
:10EB70003068C0F6020116F093FD616B626AE36AC9
:10EB800000914BF28C613068C0F6020116F088FDEE
:10EB9000796A7A69FB6900914BF2C0613068C0F60E
:10EBA000020116F07DFD41F2447243F2D813C2F225
:10EBB0000102C2F200034BF2E461306812681B6884
:10EBC000C0F6020116F06CFD46F67063C2F2000357
:10EBD0004BF210711A683068C0F6020116F060FD41
:10EBE00049F68013C2F200034BF228711A683068AC
:10EBF000C0F6020116F054FD47F2D003C2F2000342
:10EC00004BF2447144F2C4141A683068C2F2000432
:10EC1000C0F6020116F044FD4BF2587130682268CC
:10EC2000C0F6020116F03CFD0023236007B0BDE8EA
:10EC3000F08F07F6DC52D3F800801068F2F7CCFEB4
:10EC400007F55E63044618680D46F2F7C5FECDE988
:10EC500000014BF25C51404622462B46C0F60201B1
:10EC600016F01EFDE1E64BF27841C0F60201306875
:10EC7000D9F84421D9F8483116F012FD66E600BFF4
:10EC80002DE9F04344F2C017C2F2000783B00646F4
:10EC900090F8E80D3C6817F0DBF94BF2787102460A
:10ECA000C0F60201204616F0FBFC06F6DC53D7F84E
:10ECB00000901868F2F790FE06F55E630446186847
:10ECC0000D46F2F789FECDE900014BF25C51224678
:10ECD0002B464846C0F6020106F5217816F0E0FC06
:10ECE00006F5616500240FE055F8040B3E68F2F765
:10ECF00073FECDE900014BF2847122463046C0F626
:10ED0000020116F0CDFC0134404601F089FC84423A
:10ED1000EADB03B0BDE8F083AFF30080AFF300801F
:10ED200043F2E010C2F2000001F08ABDAFF30080B0
:10ED300038B504464BF290701546C0F6020010F04C
:10ED40009FF821462A460248BDE8384016F000BE2A
:10ED5000A0320020AFF30080AFF30080AFF300805B
:10ED600038B500F1C005044601F0C2FD284616F092
:10ED7000D7FD00230022C4E92E230021182204F528
:10ED80009E70F4F7D5F9284616F00AFE204638BDE5
:10ED900010B500210446182200F59E70F4F7C8F95A
:10EDA0002046BDE8104001F043BD00BFAFF3008036
:10EDB00008B543F2E010C2F20000FFF7E9FF41F6A8
:10EDC000E803C2F200031868BDE80840FFF768BD19
:10EDD0002DE9F04741F6E804C2F200040646236834
:10EDE0000F46002B00F0AE8015F08AFF0246206827
:10EDF0000B46416AC6E92E23002900F0D480816ABF
:10EE0000002900F0A78006F0A3F9052F00F2828008
:10EE100006EB870341F2087ED3F83C210132C3F8A8
:10EE20003C21C2F2000ED6E92E45DEE9002364A1A2
:10EE3000D1E90001A21A65EB0303994208BF904291
:10EE40003CBF0023337122462B4630463946CEE97B
:10EE5000004502F065FA3379002B59D041F6F405EC
:10EE6000C2F2000530462B68D3F8E031012B59D0AF
:10EE700001F0D6FCDFF85091804644F2A814C2F2AB
:10EE80000004A01C414617F0D3F94BF67003C0F6FE
:10EE90000203DB5D002B65D14BF65003C0F6020385
:10EEA00044F2581053F827A022466423C2F200000F
:10EEB0005146237003F0B4FB2B6893F8DD355A06F6
:10EEC0000CD5752344F2581044F2A8125146C2F2F0
:10EED0000000C2F20002237003F0A2FBD9F8103048
:10EEE000F26C9A4255D2D6F8C030002BC4BF3546DA
:10EEF000002460DDD5F8C430384641469847D6F83E
:10EF0000C0300134A34205F10405F3DCBDE8F0870D
:10EF1000BDE8F0874BF2D870C0F60200BDE8F047BC
:10EF200019F04EBF01F09CFCDFF89C90044630467F
:10EF300001F076FCE10754BFD9F81030002300EB54
:10EF400003089AE742F6E070C0F60300BDE8F04718
:10EF500019F036BF4BF2C070C0F60200BDE8F047B2
:10EF600019F02EBF4BF65003C0F6020344F25810BE
:10EF700053F827A0C2F200007523514622462370A1
:10EF800003F04EFB2B6893F8DD355B06A6D56423B2
:10EF900098E74BF2E471C0F6020140F25E20BDE852
:10EFA000F04713F0B5BC4BF2AC70C0F60200BDE800
:10EFB000F04719F005BFBDE8F08700BFAFF3008050
:10EFC000007A030A00000000984A0120AFF3008095
:10EFD0004FF48051CEF20001F8B543F2D81244F25A
:10EFE000B81343F2DC154968C2F20003C2F2000212
:10EFF000C2F200051E68296011688E42C8BF166003
:10F0000040F2A852C1F2000241F24074C2F201047F
:10F010004FF0010E0136074690691E6084F800E04B
:10F020000DF00EFA44F2B8168028C2F2000620DD78
:10F0300043F2E0103946C2F20000FFF7C9FE4FF478
:10F040008052CEF2000244F2C413C2F200035768A9
:10F0500029681868356844F2BC12791AC2F20002B5
:10F06000013D0027814211603560277088BF19601B
:10F07000F8BD4BF60000C0F60200BDE8F84019F0FC
:10F080009FBE00BFAFF30080AFF30080AFF30080FE
:10F0900044F2C013C2F2000343F238311868C2F2DE
:10F0A000000117F015BA00BFAFF30080AFF3008086
:10F0B000014643F2E010C2F2000002F011B900BFB5
:10F0C00038B54BF60C0244F2C013C2F20003C0F68E
:10F0D00002021860126844F2A813C2F20003150C71
:10F0E00044F258101A809D70C2F200000C4603F0E2
:10F0F0003FFB4BF610004EF6A1012246C0F602007F
:10F10000C0F6000116F0CCFC4BF61C004EF6814117
:10F110002246C0F60200C0F6000116F0C1FC4BF614
:10F1200030004EF6B151C0F60200C0F60001BDE855
:10F13000384016F0C5BC00BFAFF30080AFF30080CD
:10F14000436AD3F8A031002B70B506460CDD074D9D
:10F150000024284606F03CFB736AD3F8A031013442
:10F16000A34205F11405F4DC70BD00BFD46E00208D
:10F17000436AD3F8A031002B70B506460CDD074D6D
:10F180000024284606F0D4FA736AD3F8A03101347B
:10F19000A34205F11405F4DC70BD00BFD46E00205D
:10F1A0002DE9F04F4AF26013C2F201032DED048BFA
:10F1B0001B7889B00D4623B109B0BDEC048BBDE8C6
:10F1C000F08F41F6E804C2F20004206800F52170D7
:10F1D00001F026FAB5EB400F24BF4BF68000C0F6D5
:10F1E000020080F0F68040F2A856C1F20006B06935
:10F1F0000DF026F9802840F3E8802068FFF780F9B9
:10F2000082460028D8D0B0F1FF3F00F01F8241F6BF
:10F21000F407C2F200073B68D3F8A831984200F324
:10F2200005812068FFF74CF900F0010B002D00F07C
:10F23000B6813B6893F8DD25D3F8F01541F6F40864
:10F240005006C2F2000802D5CA0700F10C828D42B6
:10F2500000F0B1812368002D40F08A804FF480587F
:10F26000CEF2000803F50E53D8F8042050469A60F9
:10F2700004F05EFB39682368D1F8DC21D8F80490EB
:10F28000069203F50E5CD1ED8A7ADCF80820C2EB19
:10F290000909CCF80C9006EE900AD8F804C00A6E62
:10F2A00003F50D5066EEA77A43F2B839C0F828C0CE
:10F2B0000698C2F20109C9ED9C7A002800F0AC81E1
:10F2C00002EBD272521006EE902AB8EEE68AD3ED27
:10F2D0009D7AF5EE407AF1EE10FA00F0DF81B4EE9F
:10F2E000E78AF1EE10FA00F1C9810022D3F8781212
:10F2F000C7F6C07291423FF45FAF41F6086E9A6A5A
:10F30000D3F87802D3F874120EFB0BFE0EF6C86326
:10F310001A4418F05DFF23684FF4805203F50D5333
:10F32000CEF20002996A5068411AD9625268BAF165
:10F33000000F1A633B6804DDB3F968209245C0F200
:10F34000C482D9F82800D3F8B0214DF6F02100F29C
:10F350004470C1F2000119F05BF823684FF480514A
:10F3600003F50D52CEF20001106B4968081A506384
:10F37000586A19F08DFA002840F05B8120680AF184
:10F38000FF3247F22E539A42866A3FF615AF3B682A
:10F3900093F8DC359B077FF50FAF44F2C817C2F234
:10F3A000000705973968002951D043F2B837C2F2F7
:10F3B0000107DDF814800694B9468B6C4F6D9D42B1
:10F3C0000ED0002F42D03946F7E74BF69400C0F636
:10F3D000020009B0BDEC048BBDE8F04F19F0F0BCA1
:10F3E000059C2268914208BFC8F8007003D105E06F
:10F3F000994229D01A46536D002BF9D1D1ED147AD8
:10F4000099ED027A67EE277A0C68FDEEE77A4BF603
:10F41000D01045F2D17317EE902A00942031C0F637
:10F420000200C0F6010306F0EBFECAE74BF6B0019E
:10F430000246C0F6020140F25E2009B0BDEC048B2A
:10F44000BDE8F04F13F064BA5765D7E7069C41F664
:10F45000086303FB0BF303F6C86306EB0309F358D9
:10F46000002B7FF7A9AE44F6F87BC2F2000B09F13E
:10F47000080809F15006002709E0D9F800300137E3
:10F480009F4208F1600806F16006BFF695AE56F897
:10F490000C3C9D42F1D1226802F5F3531868002319
:10F4A000C7F6C07398426DD006EE900AF5EEC06ABA
:10F4B000F1EE10FA66D492ED027ADBF80031DBF857
:10F4C0000821013356ED017ACBF80031DBF8001149
:10F4D00044F6F8739142C2F2000367EE277A04BF44
:10F4E0000022C3F80021F5EEC07ADBF80021F1EE2E
:10F4F00010FA54BF002301234BF82230DBF804211B
:10F500000132CBF80421002B40F0CB8156F8482C77
:10F51000FDEEE77A4BF6F41045F23173C0F60103C5
:10F520000092C0F60200A6F1400117EE902A06F004
:10F5300067FE304656F8101C18F0DAFDD8F848304F
:10F540009D4200F0E78105980168002900F0538290
:10F5500088451CBF0B464FF47A7206D1D1E1013ABF
:10F5600000F00A82984500F0CC815B6D002BF6D14B
:10F57000F3600A4600E01A46536D002BFBD1C2F837
:10F5800054807AE7F2F728FA02464BF6F4000B466D
:10F59000CDF800A0C0F6020019F012FC6DE744F2AD
:10F5A000D010C2F2000016F0EBFF00283FF441AE8D
:10F5B00019F04EF83DE6D3F85406B0F55E7F79D1E8
:10F5C00023684FF48052DFF8ACC3CEF20002DCF8BF
:10F5D0000000D2F804E0002103F50D52C7F6C07117
:10F5E0008842C2F820E000F07B8107EE100AB5EEF9
:10F5F000C07AF1EE10FA00F17381DCED017AF1EEE0
:10F60000677AC3ED9E7A70464FF48051CEF20001C6
:10F610004968091A51621EE6D1F8A01192FBF1F275
:10F6200007EE902AB8EEE77ADFEDCF7A87EE278AE9
:10F630004DE6B0690CF004FF80285CDC4BF6381016
:10F64000C0F6020019F0BCFB206898E64BF6A0015A
:10F65000C0F6020140F2551009B0BDEC048BBDE8C4
:10F66000F04F13F055B94BF6D000C0F6020019F078
:10F67000A7FBD8F80030D3F8F015E8E517EE900AAC
:10F68000F2F7AAF90B464BF61C110246C0F602012E
:10F6900040F25E2013F03CF9236826E64BF60C118D
:10F6A000C0F6020140F25E2013F032F92368D3ED78
:10F6B0009D7A14E60AF09CFF06EE900ADFEDAB7A25
:10F6C0003A682368B8EEE67A93F8801227EE277A34
:10F6D000D2ED6E7A27EE277AF0EE047AB4EEE77A6E
:10F6E000F1EE10FAD4BF00220122114383F87F22E9
:10F6F00083F8801265E7206800F5217001F038F981
:10F7000041F6E8068542C2F2000680F02381BAF194
:10F71000000F40F31A813B68B3F968309A4580F2D4
:10F72000148143F2B833C2F201033068D3F828C021
:10F730000CEB050393F84436002B3FF420AE00F5A4
:10F74000AE70CDF810C004F063FB2068483004F0C0
:10F750006FFB504604F0ECF83B68DDF810C0D3EDC9
:10F760008A7A06EE900ADCF8002041F6E80343F2BC
:10F77000B83966EEA77AC2F20003C2F20109002A84
:10F78000C9ED9C7AD8BF18687FF7F9AD0020C7F69D
:10F79000C070DFED778A059066464FF00008079746
:10F7A000CDF80CC006E008F10108904506F11406FA
:10F7B00080F2D88073689D42F5D199ED9C8A059FAF
:10F7C00018EE101AB94200F0E980B5EEC08AF1EEE9
:10F7D00010FA00F1EE80236803F5F4531B7E002B32
:10F7E000E1D143F2B832C2F2010292ED029AD6EDB3
:10F7F000037A337D29EE279A002B00F0EB80B5EEDB
:10F80000C08AF1EE10FA00F1F880D6F810C0BCF111
:10F81000000F00F00181CDF810C0FEF7A1FE01231A
:10F82000C8F200030340002BBEBF03F1FF3363F0B7
:10F83000010301331820DDF810C0226800FB03FE2D
:10F84000BDEEC99A0EF108014BF6BC100EF1380E50
:10F850004FF2711361440092F444C0F60200C0F606
:10F86000000319EE102ACDF810C006F0C9FCF8EE1E
:10F87000C97ADDF810C02768E8EE287A4BF6C41084
:10F88000FDEEE77A4FF2411317EE902AC0F6020020
:10F8900061460097C0F6000306F0B2FC03980268C8
:10F8A00081E744F2D413C2F2000317EE900A1B68FA
:10F8B0000693F2F791F80B464BF6DC110246C0F6C0
:10F8C0000201069815F0ECFED7E54CF6A001D9F838
:10F8D0002800D3F8AC21C1F2000118F099FD3CE5F5
:10F8E000F2F77AF802464BF6F4000B46C0F6020037
:10F8F000CDF800A019F064FA236803F50D52106AE0
:10F9000082E64BF61C21C0F6020140F25E2012F0A6
:10F91000FFFFB2E5236856F8481C93ED027AD6ED56
:10F92000027A67EE277A4BF60020FDEEE77A45F281
:10F93000D173009117EE902AC0F60200C0F60103C1
:10F94000A6F1280106F05CFC97E52068836A03F2C3
:10F95000447CEDE64BF64410C0F6020019F030FA94
:10F9600030680CE5079F09E5CDCC8C3F010C403A8F
:10F9700000007A44185201204BF60C20C0F6020019
:10F98000049219F01DFA0599049A0B68F260002B95
:10F990007FF4F1AD059AC2F800806EE54BF65C117C
:10F9A000C0F6020140F25E2012F0B2FF0398026836
:10F9B000F9E618EE100AF2F70FF80B464BF6701145
:10F9C0000246C0F6020140F25E2012F0A1FF039948
:10F9D0000A68E8E6376915F083F928EE288A0246B6
:10F9E0000B4638468DED018A8DED009A05F060FFDB
:10F9F00003990A68D7E6F160CCE718EE100AF1F730
:10FA0000EBFF02464BF68C100B46C0F6020019F0D5
:10FA1000D7F9039B1A68C6E64BF6AC10C0F6020095
:10FA200019F0CEF9039F3A68BDE600BFAFF300803E
:10FA3000F0B583B00746FEF763FD054618F068FA97
:10FA4000F1F7CAFF44F2D414CDE90001C2F2000478
:10FA50004BF640212A462068C0F6020115F020FE30
:10FA60002846266803F064FFF1F7B6FF07F5F35761
:10FA7000044678680D46F1F7AFFFCDE900014BF67B
:10FA80005821304622462B46C0F6020115F008FEEA
:10FA900003B0F0BDAFF30080AFF30080AFF30080A0
:10FAA00008B5FFF7F5FA44F2D413C2F2000344F2AA
:10FAB000D8111868C2F2000116F00AFDBDE808402E
:10FAC00002F04EBEAFF30080AFF30080AFF30080D2
:10FAD000F8B544F2D414C2F200040D4620600029A7
:10FAE0003ED044F2CC16C2F200064BF684204FF60C
:10FAF000A121C0F60200C0F60001356015F0E0FF5C
:10FB00004BF694204FF63121C0F600012A46C0F68C
:10FB1000020015F0C5FF276815F0FAF84BF6A02192
:10FB20000246C0F60201384615F082FD3368586A75
:10FB300018F0AEFE60B14FF2A1104BF6DC212A4660
:10FB4000C0F60000C0F60201BDE8F840FFF7F0B8CB
:10FB50004BF6B4212068C0F6020115F069FDEAE712
:10FB60004BF67820C0F60200BDE8F84019F028B93D
:10FB700070B444F6F875C2F20005D5F80431052BCF
:10FB80001EDCD5F80461D5F80011002ED8BF002086
:10FB900014DD0024D5F80821204600290B4601DA9F
:10FBA0009B18FDD455F823300130B0421C4401F1BC
:10FBB000FF31F2DB042CD4BF0020012070BC704761
:10FBC000D5F800110626E4E7AFF30080AFF300801C
:10FBD00038B502212DED068B0122044600F050FDC0
:10FBE00046F6C9112046C3F6BE710122002300F07B
:10FBF000BFFFDFED6B8A9FED6B9A1725012213463D
:10FC000018EE901A204600F0B3FF78EE898A20465D
:10FC100018EE901A0122002300F0AAFF013DDFED4B
:10FC2000619A78EE898AE9D19FED5F8A38EE88AAD9
:10FC3000012213461AEE101A204600F099FF3AEE00
:10FC4000088A2B4618EE101A2046012200F090FF79
:10FC500038EE298AF0EE698A24250122134618EE2F
:10FC6000101A204600F084FF38EE288A204618EE4D
:10FC7000101A0122002300F07BFF013D38EE288A94
:10FC8000EBD100212A462046C4F2BC31012300F00A
:10FC90006FFF9FED449A15250122134618EE101AA6
:10FCA000204600F065FF38EE098A204618EE101A4B
:10FCB0000122002300F05CFF013DDFED3A9A38EEAF
:10FCC000098AE9D1DFED397A9FED379A3AEE27AA12
:10FCD00038EE098A3AEE48AA1AEE100A16F0D8F958
:10FCE000DFED337A07EE100AB4EEE77AF1EE10FAA0
:10FCF0004CD50122134618EE101A204600F038FFAA
:10FD000038EE098A2B4618EE101A2046012200F020
:10FD10002FFF38EE298AF0EE698A21250122134649
:10FD200018EE101A204600F023FF38EE288A2046ED
:10FD300018EE101A0122002300F01AFF013D38EEE0
:10FD4000288AEBD1DFED1B7A77EEC87A17EE900A9E
:10FD500016F09EF9DFED167A07EE100AB4EEE77A98
:10FD6000F1EE10FA12D50122134618EE101A2046B1
:10FD700000F0FEFE00212046C4F234412A462B4604
:10FD800000F0F6FEBDEC068B257038BDBDEC068B91
:10FD90004BF6F020C0F60200BDE8384019F010B86C
:10FDA00057CF8E40C9693E4057CF0E410000B44343
:10FDB000CDCCCC3DCBA03344AFF30080AFF300807B
:10FDC00070B501220221044600F05AFC4FF4D551CF
:10FDD0002046C3F6BF710125002601F0A9F84DF2B7
:10FDE000747120462A462B4684F8646B2570C4F251
:10FDF000532100F0BDFE44F29C5120462A46334672
:10FE0000C4F2F52100F0B4FE4EF2A4512046324671
:10FE10002B46C4F2583100F0ABFE4AF2DB312046EB
:10FE20002A462B46C4F2683100F0A2FE46F6EC01E9
:10FE3000204632463346C4F2903100F099FE45F236
:10FE4000BB2120462A463346C4F2973100F090FE8B
:10FE500043F65A1120462A462B46C4F2CE3100F012
:10FE600087FE46F68A0120462A463346C4F2F1311F
:10FE700000F07EFE44F24621204632462B46C4F274
:10FE8000104100F075FE43F6330120462A462B460A
:10FE9000C4F2144100F06CFE4BF6951120462A4640
:10FEA0003346C4F2254100F063FE0021204632466D
:10FEB0003346C4F23441BDE8704000F059BE00BF83
:10FEC00070B544F2AE7104460025C3F6E15101F06D
:10FED0002FF8204684F8645B0221012200F0D0FB59
:10FEE000002120462A46C4F2A011012300F040FE62
:10FEF000002120462B46C4F28421012200F038FE66
:10FF00000122002120461346C4F28C2100F030FE6D
:10FF1000002120462B46C4F20831012200F028FEC1
:10FF20000122002120461346C4F20C3100F020FECD
:10FF3000002120462B46C4F27631012200F018FE43
:10FF40000122002120461346C4F27A3100F010FE4F
:10FF5000002120462B46C4F29E31012200F008FE0B
:10FF60000122002120461346C4F2A03100F000FE19
:10FF7000002120462A462B46C4F2AA3100F0F8FDA3
:10FF8000002120462A46C4F2B431012300F0F0FDDE
:10FF9000002120462A462B46C4F2BE3100F0E8FD7F
:10FFA000002120462A46C4F2C831012300F0E0FDBA
:10FFB000002120462B46C4F2D531012200F0D8FDA5
:10FFC0000122002120461346C4F2D73100F0D0FDB3
:10FFD000002120462B46C4F2F831012200F0C8FD72
:10FFE0000122002120461346C4F2FA3100F0C0FD80
:10FFF0004FF4004120462B46C4F21741012200F085
:020000040801F1
:10000000B7FD01224FF4004120461346C4F21841C7
:1000100000F0AEFD002120462B46C4F2294101220A
:1000200000F0A6FD0122002120461346C4F22A4119
:1000300000F09EFD002120462A462B46C4F23441A2
:10004000BDE8704000F094BDAFF30080AFF30080D6
:1000500010B502210022044600F012FB41F27B4160
:100060002046C4F2E2210022012300F081FD00229B
:10007000002113462046C4F2343100F079FD48F2E5
:100080001F512046C4F292310022012300F070FD7E
:100090000022002113462046C4F2B43100F068FD6E
:1000A00048F21F512046C4F2EC310022012300F037
:1000B0005FFD0022002113462046C4F2074100F0F4
:1000C00057FD44F28F212046C4F223410022012330
:1000D00000F04EFD0022002113462046C4F23441B8
:1000E00000F046FD0023237010BD00BFAFF3008079
:1000F00010B502210122044600F0C2FA4AF694012A
:100100002046C4F2BE210022012300F031FD01226D
:1001100046F6721113462046C4F2DC2100F028FD99
:1001200040F2D7512046C4F232310122002300F0C0
:100130001FFD002247F2CB2113462046C4F268314E
:1001400000F016FD01224DF6922113462046C4F21E
:100150008F3100F00DFD47F25E112046C4F2B2313E
:100160000122002300F004FD012243F2E7111346AF
:100170002046C4F2EA3100F0FBFC4BF24651204627
:10018000C4F206410122002300F0F2FC01224AF6EB
:10019000763113462046C4F2224100F0E9FC0021EA
:1001A000C4F2344101220023204600F0E1FC41F674
:1001B000816104F53662C4F20931002311602370B5
:1001C00010BD00BFAFF30080AFF30080AFF300803D
:1001D00070B502210446002200F052FA00250123E6
:1001E000002184F8643B20462A462570C4F207416A
:1001F00000F0BEFC002120462A462B46C4F23441C2
:10020000BDE8704000F0B4BCAFF30080AFF30080F5
:1002100070B5022104460022012500F031FA41F2B6
:10022000CB0144F69842204684F8645B84F8655B11
:10023000C3F6FF71C4F2BF0200F06AFE41F23D2135
:1002400020462B46C4F20F31002200F091FC002220
:100250004AF64E7120461346C4F2363100F088FC4F
:1002600046F6964120462B46C4F25731002200F054
:100270007FFC002241F6AB7120461346C4F2803168
:1002800000F076FC45F27B4120462B46C4F29031CB
:10029000002200F06DFC002246F29D3120461346FC
:1002A000C4F2A33100F064FC4CF2D42120462B466A
:1002B000C4F2B431002200F05BFC002247F6EF21CB
:1002C00020461346C4F2FE3100F052FC46F6A4016B
:1002D00020462B46C4F20841002200F049FC0022CF
:1002E0004BF6467120461346C4F2114100F040FC23
:1002F00044F6B76120462B46C4F21A41002200F0B2
:1003000037FC002245F6B80120461346C4F22341CB
:1003100000F02EFC40F2E96120462B46C4F22B414E
:10032000002200F025FC0022002120461346C4F2E2
:100330003441BDE8704000F01BBC00BFAFF300804B
:1003400070B501220221054600F09AF945F2EC1140
:100350002846C3F638710124002600F0E9FD00218B
:1003600028462246234685F8646BC5F8804BC4F2C4
:10037000202100F0FDFB0021284622463346C4F22E
:10038000302100F0F5FB0021284622462346C4F226
:10039000602100F0EDFB0021284622463346C4F2DE
:1003A000702100F0E5FB0021284622462346C4F2D6
:1003B000A62100F0DDFB0021284622463346C4F288
:1003C000B02100F0D5FB0021284622462346C4F286
:1003D000DE2100F0CDFB0021284622463346C4F240
:1003E000E82100F0C5FB0021284632463346C4F21E
:1003F000203100F0BDFB0021284622462346C4F2EE
:10040000343100F0B5FB0021284622463346C4F2C1
:100410005C3100F0ADFB0021284622462346C4F2A1
:100420006B3100F0A5FB0021284622463346C4F27A
:100430006F3100F09DFB4FF40041284622462346D1
:10044000C4F2823100F094FB002128462246334654
:10045000C4F2853100F08CFB002128462246234659
:10046000C4F2913100F084FB4FF40041284622464B
:100470003346C4F2933100F07BFB0021284632461C
:100480002346C4F2B43100F073FB00212846224613
:100490002346C4F2C63100F06BFB4FF400412846FE
:1004A00022463346C4F2C73100F062FB00212846E1
:1004B00022462346C4F2CD3100F05AFB4FF40041EE
:1004C000284622463346C4F2CF3100F051FB4FF4A8
:1004D0000041284622462346C4F2DA3100F048FBA8
:1004E0000021284622463346C4F2DD3100F040FBAD
:1004F0004FF40041284622462346C4F2E83100F07A
:1005000037FB0021284622463346C4F2EB3100F087
:100510002FFB4FF40041284622462346C4F20541F2
:1005200000F026FB4FF44041284632463346C4F2E1
:100530000A4100F01DFB4FF4004128462246334695
:10054000C4F2104100F014FB002128462246234645
:10055000C4F2154100F00CFB4FF4804128462246BE
:100560003346C4F2164100F003FB4FF440412846E5
:1005700022462346C4F21B4100F0FAFA0021284625
:1005800022463346C4F21D4100F0F2FA002128460B
:1005900022462346C4F2234100F0EAFA4FF4804198
:1005A000284622463346C4F2244100F0E1FA0021F5
:1005B000284632462346C4F23441BDE8704000F07C
:1005C000D7BA00BFAFF30080AFF30080AFF3008075
:1005D000F8B5044600F53D7704F53E76384615F04B
:1005E000DFFF04F53F75304615F0DAFF284615F0B9
:1005F000D7FF3846214615F0E3FF304604F1FC01F1
:1006000015F0DEFF284604F5FC7115F0D9FF2046F1
:10061000F8BD00BFAFF30080AFF30080AFF3008000
:1006200000F5A350C0687047AFF30080AFF30080BF
:100630002DE9F00100F5A35100F5366600F65835B6
:1006400000F65C3400274FF000080122C4F22007B6
:1006500000234FF07F5CC6F800800270C5F800C030
:10066000276080F8642BBDE8F0010B7280F8653BD1
:10067000704700BFAFF30080AFF30080AFF300809E
:10068000F8B5044600F5BB5300F5DB5600F5A3575B
:100690000025B16003F11400FD60294662701D6100
:1006A0004FF47C7284F8805B84F8815B84F8825B11
:1006B00084F8835B84F8845B84F8855B84F8865BCC
:1006C00084F8875B84F8885B84F8895B84F88A5BAC
:1006D00084F88B5BF2F72CFD84F8685B84F8695B27
:1006E00084F86A5B84F86B5B84F86C5B84F86D5B00
:1006F00084F86E5B84F86F5B84F8705B84F8715BE0
:1007000084F8725B84F8735B04F6743015F078FF3C
:1007100000237360F8BD00BFAFF30080AFF300802B
:10072000F8B5044600F5BB5505F11401002204F5A7
:10073000A35600F6743015F053FF06F11000FFF7D2
:1007400047FF002120460A46FFF79AFF04F65C3C6B
:1007500004F6583E04F536620023291D4FF47C77D9
:100760000025C4F8781B84F8645B84F8655B257009
:100770002946357204F68C3013606560A5603A46F0
:10078000CCF80030CEF80030F2F7D2FC04F58350FC
:100790003A4629461830F2F7CBFC294604F67C701D
:1007A000FC22F2F7C5FC294604F118004FF434622C
:1007B000F2F7BEFC2046F8BDAFF30080AFF3008037
:1007C000436853F821309856704700BFAFF300805C
:1007D000F8B5171E06460D46C8BF002403DC0DE021
:1007E0000134BC420AD0B36803EB8403294618687D
:1007F00015F02EFD0028F3D02046F8BD4FF0FF3055
:10080000F8BD00BFAFF30080AFF30080AFF300800E
:10081000836803EB81010A60704700BFAFF300807B
:10082000C06C7047AFF30080AFF30080AFF300807F
:100830000023036503648364704700BFAFF3008047
:1008400030B4D0E92623C06C141843F100052046CB
:10085000294630BC704700BFAFF30080AFF3008083
:10086000D0F8A000704700BFAFF30080AFF3008066
:1008700070B500251826044680F8545080F855506D
:1008800080F8565080F8575080F8585080F85950EA
:1008900080F85A5080F85B5080F85C5080F85D50CA
:1008A00080F85E5080F85F50294632466430F2F797
:1008B0003FFC324604F180002946F2F739FC2576E8
:1008C0006576A576E57625776577A577E57784F86B
:1008D000205084F8215084F8225084F82350E56495
:1008E00070BD00BFAFF30080AFF30080AFF30080B6
:1008F000F8B50027064600240025076007718760C9
:10090000C0F8A070C7634764C76080F8607080F863
:100910006170076507648764C0E90445C0E92A453A
:10092000C0E92C45FFF7A4FF012386F8307086F854
:10093000317086F8327086F8337086F8347086F835
:10094000357086F8367086F8377086F8387086F815
:10095000397086F83A7086F83B70C6E9264586F805
:10096000A4303046F8BD00BFAFF30080AFF3008085
:1009700000F5DB5300F5A3509B68C068022B18BF3D
:1009800040007047AFF30080AFF30080AFF300800A
:1009900000F5DB5208B59268022A1DD000F5A3527B
:1009A00000F67430D26891420BDB891A15F030FEE4
:1009B000DFED107A07EE100AE7EE277A17EE900ABD
:1009C00008BD15F025FEDFED0B7A07EE100A67EE85
:1009D000277A17EE900A08BD00F6743015F018FE5D
:1009E000DFED057A07EE100A67EE277A17EE900A18
:1009F00008BD00BF0000B44300003444AFF30080E2
:100A00002DE9F04F41F6F408C2F200082DED028BFB
:100A1000D8F8001085B001F50171064601F0F8F82C
:100A200041F6E80706F5DB52C2F20007014606F57B
:100A3000A35390683A6801930228D86802F5F452EB
:100A400006F5BB5A18BF4000CAF81010D0613046F6
:100A5000FFF79EFF3A6802F5F45208EE900AD0695B
:100A6000002823DD06F68C3346F2604BC1F2000B02
:100A7000029300241D469FED398A06F58353D9461B
:100A800022460393C346B4B9029B83ED008A039BBD
:100A900006F5396181ED008A9C61396801F5F451F0
:100AA0000134C869A04205F10405ECDC05B0BDECD9
:100AB000028BBDE8F08FDAF81010DDF804E0214475
:100AC000DEF80C30009291FBF0FE00FB1E11994203
:100AD0003046ACBFC3EB01088846FFF759FF06EE6E
:100AE000900A76EEE87AD9ED1A6AF5EEC07AF1EE60
:100AF00010FA009AB8EEE67A0DD577EE877AF5EE21
:100B0000C07AF1EE10FAF8D4B4EEE77AF1EE10FA0A
:100B100006D877EEC77AB4EEE77AF1EE10FAF8D994
:100B2000DBF8001091F8DD154B0658BFC5ED007AD3
:100B300010D5B04498F97C1F61B102F5397002F20A
:100B4000E52106EB800006EB8101C0ED017AC1EDE5
:100B5000017A0232C5F8EC249FE700BF00000000D4
:100B600000F5DB5080687047AFF30080AFF3008082
:100B70002DE9F04F00F5DB542DED028B0546A06802
:100B800089B01746984608EE101A002800F0E18058
:100B9000012A00F0D58005F5A356337A002B40F0EA
:100BA000B680CDF80C8000F0BBFD41F6F403C2F234
:100BB000000307EE900A1B6893F8DD355B0688EEAC
:100BC000278A40F1AA80B8F1010F00F0A680B5EEA7
:100BD000C08AF1EE10FADCBF4BF64430C0F60200DA
:100BE00040F3A780F268002A40F3BE80D4ED018A6A
:100BF000B4EEE88AF1EE10FA88BF84ED018A40F283
:100C0000DF8005F67433184618EE101A0293FFF7CA
:100C1000DFFD411C029B40F08880F168B1F1010AC0
:100C200000F10381D5F87C0B4FEA8A0C6044D0EDCB
:100C3000007AB4EEE78AF1EE10FAD8BF524608DD2A
:100C4000D7E070ED017AB4EEE78AF1EE10FA00F326
:100C5000D18012F1FF32F4D2002005900692834633
:100C600004900CF10409049C07965E46CB46994615
:100C70000AF101000023D5F8782BD2580433915D96
:100C80000C2B1154F7D15146484615F0C1FCD5F84C
:100C90007C3B0AF1FF3A5B44A2451860ABF1040BC0
:100CA000E6DAB346079EF168049BB8F101022B44D3
:100CB000D2F1000858EB020883F87C8F049B8B422A
:100CC00006D04BF6C430C0F6020018F079F8F1688F
:100CD00001310698F1600023D5F8782BD2580433FF
:100CE000115C0C2B02F80B10F6D1D5F8783BD5F837
:100CF0007C1B059A53F827300398114481ED008A34
:100D000003F80B0009B0BDEC028BBDE8F08FD8F101
:100D1000010338BF0023039345E705EB8703D3F8AE
:100D2000682B0132C3F8682B51E74BF6A830C0F6A8
:100D3000020009B0BDEC028BBDE8F04F18F040B8DE
:100D40006B78002B7FF427AF4BF62830C0F60200FB
:100D5000EFE74BF61030C0F6020009B0BDEC028B95
:100D6000BDE8F04F18F02CB884ED018A7FF449AF4C
:100D70000123F360D5F8783B9918A81800294AD0C8
:100D80009B580432002B4BD0D0F8801B0C2A1970D2
:100D9000F0D1B8F10100D0F10008D5F8783BD5F8D2
:100DA0007C2B58EB000885F87C8F53F8273003988C
:100DB00082ED008A187009B0BDEC028BBDE8F08F9F
:100DC00018EE100AF0F708FE044618EE900A0D46D9
:100DD000F0F702FECDE900014BF6603022462B46CB
:100DE000C0F6020017F0ECFF09B0BDEC028BBDE8C5
:100DF000F08F5246501C82450692B8BF8200049084
:100E0000BCBF83460592FFF64FAFDDF810B04FEA46
:100E10008B02059225E74BF68030C0F6020088E78A
:100E20004BF69030C0F6020083E700220592069050
:100E30009346049238E700BFAFF30080AFF3008021
:100E400007EE901A9DED007AF4EEC77AF1EE10FAF3
:100E5000DDED016A04DDF4EEE67AF1EE10FA00D47D
:100E60007047FFF785BE00BFAFF30080AFF300808F
:100E700010B52DED028BB1EE0E8A70EE088A0222BB
:100E800018EE901A01230446FFF772FE38EE888AA6
:100E9000204618EE101A02220023FFF769FEB2EE78
:100EA0000E0A38EE000ABDEC028B10BDAFF30080D5
:100EB00010B501222DED028B10EE101AF0EE408AD3
:100EC0001346B2EE0E8A0446FFF752FE78EE888A89
:100ED000204618EE901A01220023FFF749FE38EE53
:100EE000880ABDEC028B10BDAFF30080AFF3008029
:100EF00083680846194615F093BB00BFAFF3008026
:100F000010B4012480F8644B5DF8044B00F090BCF1
:100F100030B400F65C3300F65834012505702160CA
:100F20001A6030BC704700BFAFF30080AFF30080A1
:100F300007EE901AB6EE087AF7EE046A27EE877A83
:100F400067EEA67A012100F6583200F65C33017094
:100F500082ED007AC3ED007A704700BFAFF30080E6
:100F600070B50122044615460221FFF789FB204691
:100F7000C4F8845B9FED590AFFF77AFF00262046EC
:100F8000FFF776FFC4F2B4262046FFF771FF314623
:100F90002A4600232046FFF7EBFD204600EE106AAC
:100FA000FFF766FF00262046FFF762FFC4F23436E3
:100FB0002046FFF75DFF31462A462B462046FFF7C5
:100FC000D7FD204600EE106AFFF752FF00262046AC
:100FD000FFF74EFFC4F287362046FFF749FF314640
:100FE0002A4600232046FFF7C3FD204600EE106A84
:100FF000FFF73EFF2046FFF73BFF2046FFF738FF95
:1010000000264FF48041C4F2B43620462B46C4F289
:10101000B0310022FFF7ACFD31462A462B46204670
:10102000FFF7A6FD204600EE106AFFF721FF00261D
:101030002046FFF71DFFC4F2E1362046FFF718FFF8
:1010400031462A4600232046FFF792FD204600EE57
:10105000106AFFF70DFF00262046FFF709FFC4F2D4
:1010600007462046FFF704FF31462A462B46204616
:10107000FFF77EFD204600EE106AFFF7F9FE4FF401
:1010800000462046FFF7F4FEC4F21D462046FFF757
:10109000EFFE2A46314600232046FFF769FD204631
:1010A00000EE106AFFF7E4FE2046FFF7E1FE20465F
:1010B000FFF7DEFE00224FF4005113462046C4F233
:1010C0003241FFF755FD00212B4620462A46C4F247
:1010D0003441FFF74DFD0023237070BD0000000078
:1010E00070B504462DED048B01220E460025022129
:1010F000FFF7C6FA25702046B1EE040AFFF7D8FEC6
:10110000B0EE408A002E40F090802046FFF7D0FEDF
:101110002046FFF7CDFEB0EE408AB0EE480A2046EA
:10112000FFF7C6FE2046FFF7C3FE4AF2C501B0EE48
:10113000408AC4F21231002201232046FFF718FD35
:101140002046B0EE480AFFF7B3FE00220021134606
:10115000C4F23431B0EE408A2046FFF709FD204644
:10116000B0EE480AFFF7A4FE2046FFF7A1FE204696
:10117000FFF79EFE2046FFF79BFE2046FFF798FEF6
:1011800045F26201C4F2A33100220123B0EE408A8D
:101190002046FFF7EDFC2046B0EE480AFFF788FE38
:1011A0000022002120461346C4F2B431F0EE408AFA
:1011B000FFF7DEFCDFED2C9A9FED2C9A0325B0EEB5
:1011C000680A2046FFF774FE2046FFF771FE2046AE
:1011D000FFF76EFE2046FFF76BFE2046FFF768FE26
:1011E00007EE905AB8EEE78AF0EE408A28EE298A98
:1011F000002278EE497A012317EE901A2046FFF775
:10120000B7FC2046B0EE680AFFF752FE00222046E7
:1012100018EE101A01351346F0EE408AFFF7A8FCCD
:10122000052DCCD1BDEC048B70BDF1EE0E8A70EEB5
:10123000687A022217EE901A01232046FFF798FCE5
:101240002046B0EE480AFFF733FE2046FFF730FE97
:1012500070EE688A20462B4618EE901A0222B0EEF5
:10126000408AFFF785FC58E700003443ED7C0542D7
:1012700000F118010EC9016342638363704700BF28
:1012800070B445F21815C2F20005D5F80431052BEB
:101290001EDCD5F80461D5F80011002ED8BF00205F
:1012A00014DD0024D5F80821204600290B4601DA78
:1012B0009B18FDD455F823300130B0421C4401F195
:1012C000FF31F2DB042CD4BF0020012070BC70473A
:1012D000D5F800110626E4E7AFF30080AFF30080F5
:1012E00008B500EB81012DED028B91ED098ADFED50
:1012F000097AB8EE488AD0E92A0128EE278AF0F761
:101300009FFF07EE100A88EE077ABDEC028B17EEFE
:10131000100A08BD0000C842AFF30080AFF30080A0
:101320002DE9F04F05298BB00646CDE9062300F2E2
:10133000D18041F6F408C2F200084BF6E033D8F849
:10134000000090F8DD25C0F60203550613F801A051
:1013500096F8603006D496F861209A4202BF726C0B
:101360000132726406EB8A0986F8613086F86010F3
:10137000D9F8542006EB81030132C9F854205A6E83
:1013800001325A6696F8A4304FF0000C0024002B6E
:1013900036D043F2B837C2F20107C6F80CC097F84E
:1013A000E8CDBCF1000F3CD001293CD006EBCA0AC5
:1013B000DAE9202352EA030400F09580D9F81830C6
:1013C00006990B44991A00220023C9F81810CAE99B
:1013D000202390F8DD35F26C5C0648BF013297F8A7
:1013E000E93D0132F26443B1DDE90601F368C6E983
:1013F00004010022B36086F8A4200BB0BDE8F08F92
:10140000D6E90423DDE90645A41A65EB0305BFA36D
:10141000D3E90023AB4208BFA24238BF1446A4461A
:10142000B7E70029C2D197F884124FF0000B86F875
:10143000A4B000295CD096ED026AB34BF8EE467A70
:10144000D3ED006A06EE104A67EEA66AB8EEC67AD9
:10145000B4EEE67AF1EE10FA0CDDD3ED016A67EE38
:10146000A66AB4EEE67AF1EE10FA54BF4FF0000B24
:101470004FF0010B90F8DD35180700F1D980BBF172
:10148000000F40F0218106EBCA0ADAE9202352EA74
:10149000030100F0E980D9F81830069C23449A1A19
:1014A00000200021C9F81820CAE92001D8F800302E
:1014B00093F8DD3513F0400FF36C18BF013301339F
:1014C000F364DDE90601F368C6E90401B3600BB01B
:1014D000BDE8F08F4BF6F030C0F602000BB0BDE86F
:1014E000F04F17F06DBCDDE90623CAE9202370E751
:1014F00090F8DD253379DFF81CB212F0400F0CBFF5
:10150000012202222BB1DBF81010F36C8A1A9342ED
:10151000B9D3716DD7F8EC2D43F2B8339142C2F2D2
:10152000010300F0BC8045F20410C2F2000001216A
:1015300004F036FD13F0E4FBF36BD8F80020013320
:10154000F36392F8DD2541F21073C2F20003C3E9A0
:101550000001130700F1BB80012045F21813C2F20D
:101560000003D3F80011D3F808210131C3F80011AA
:10157000D3F80011914204BF0022C3F80021D3F830
:10158000002143F82200D3F804210132C3F80421DA
:10159000FFF776FE00286CD1012306EBCA0A3371EF
:1015A000DAE9202352EA030059D0D9F81830069915
:1015B0000B449A1A00200021C9F81820CAE920011A
:1015C000D8F80030F26C93F8DD35590648BF013287
:1015D00033680132F2640BB130469847334606F166
:1015E000240053F8187F59689A68776241608260D6
:1015F000D6E92C23DDE90601821A61EB0303C6E973
:101600002C01C6E92A233046FFF732F9D6E9262312
:10161000DBF81070D6F8A000316DD21943EBE773F8
:1016200001300131C6E92623C6F8A000316548E73C
:10163000C7EE276A45F21413C2F200031C6816EEC7
:10164000900AF0F7C9F9F56C0B464BF604410246D7
:1016500000952046C0F6020114F022F80FE7DDE9FC
:101660000623CAE92023ABE7DDE90601CAE9200128
:101670001CE7D7F8F41DD7F8EC2DD7F8F03D706DC6
:10168000B76DF56D00914BF65841019002970395A7
:10169000C0F6020140F25E2011F03AF97CE7B16D2C
:1016A000D3F8F02D91427FF43EAFD3F8F42DF36DD3
:1016B00093427FF438AF45F20410C2F200000021DB
:1016C00004F06EFC002048E7DFF848B021E745F25F
:1016D0001413D7F8F05D716DF26CC2F20003186854
:1016E000D7F8EC3D0095D7F8F44DD6F858E00194C2
:1016F000F56D02914BF61041CDF80CE00495C0F663
:10170000020113F0CDFF27E79441012000C42264B9
:1017100000000000984A0120AFF30080AFF3008082
:101720009FED057ADFED057A03280CBF17EE900ACE
:1017300017EE100A704700BF000034440000B443A5
:101740002DE9F0432DED068BD31A83B003F1FF3959
:10175000B9F1000F05460E46DDED108A9DED11AA88
:10176000129FDDF84C8058DD07EE102AF8EEC7AA6C
:101770009FED2C8A8AEE2A9A0024F6EE009A38EE23
:10178000298AF0EE687AE8EE097A013417EE901AA9
:1017900030462A4601230097CDF80480FFF750FB1E
:1017A00006EE904AB8EEE68AB0EE687AA8EE097ABC
:1017B0000097CDF8048017EE101A30462A46002311
:1017C000FFF73EFB4C45DAD1CAEE2A7A30462A466C
:1017D00001230097CDF8048007EE109AF8EEC76A4F
:1017E000B6EE007A36EE877AF0EE686AE7EE276AA0
:1017F00016EE901AFFF724FB38EE8AAA30461AEE4E
:10180000101A2A4600231097CDF8448003B0BDEC8F
:10181000068BBDE8F043FFF713BB06EE902AF8EE07
:10182000E6AAD1E700000000AFF30080AFF300802C
:10183000F0B50F1E85B015461E46044633DD511C1B
:1018400007EE901AF8EEE77A476017EE901AA2605A
:10185000FFF76EFB2B1C18BF012323702046314677
:101860000022FEF70DFF9FED147ADFED147A032EB0
:101870004FF000004FF000064FF0000E18BFF0EEE2
:10188000477AC4F27A46CBF68070029021463A46F7
:101890002B46CDED017ACDF800E003960020FFF74E
:1018A0004FFF05B0F0BD4BF69040C0F6020005B00A
:1018B000BDE8F04017F084BA000034440000B4439F
:1018C0002DE9F0430E464BF6A841C0F6020102F5A1
:1018D000217485B0154613F0E3FE2046FEF7A8FEFE
:1018E000D6F80412132900F2EE80DFE811F0E200CE
:1018F000DE00DA00D600D200CE00CA00C600BE006C
:10190000B600B100AD00A800A400A0009C007300C8
:101910002A00220014002046FEF75AFC2046FEF75B
:101920007FFE014605F6F85005B0BDE8F043FFF72D
:10193000DFBAD6F8E031204601210022FFF7E0FAB5
:10194000ECE7204602210122FEF79AFE00262046FF
:101950004FF08041002201230027FFF709F9C4F26C
:10196000B436C4F2A0174FF000094FF08043029341
:10197000012021463C220223CDF8009001960397D6
:10198000FFF7DEFE4FF000080022134620463946DE
:10199000C4F27A48FFF7ECF8012021463C220223EA
:1019A000CDF8009001960297CDF80C80FFF7C8FEA5
:1019B0000023CBF680730293009602230196CDF8A4
:1019C0000C80012021463C22FFF7BAFE002385F857
:1019D0008432A3E7204602210122FEF751FE0021B6
:1019E0002046C4F2343100220123FFF7C1F800225F
:1019F000002113462046C4F2B431FFF7B9F80122A2
:101A0000002113462046C4F20741FFF7B1F8002138
:101A100000232046C4F234410122FFF7A9F8002335
:101A200085F884327AE72046FEF762FB76E72046A7
:101A3000FEF7EEFB72E72046FFF792FA6EE72046CC
:101A40000021FFF74DFB69E7204600F001FA65E74A
:101A500020460121FFF744FB60E7D6F8E03120463D
:101A600024210122FFF74CFA58E7D6F8E03120464E
:101A70003C210222FFF744FA50E72046FEF7E8FA3D
:101A80004CE72046FEF7A4F848E7204600F058FA55
:101A900044E72046FEF714FA40E72046FEF790F9A7
:101AA0003CE72046FEF74CFC38E7204600F068F99A
:101AB00034E72046D6F80C12D6F81022D6F8E031DA
:101AC000FFF7B6FE2AE74BF6C440C0F6020005B0A9
:101AD000BDE8F04317F074B9AFF30080AFF30080B6
:101AE0002DE9F04F104681B0164698468946FEF71C
:101AF00097FD98FBF0F505FB10853046FEF790FD4D
:101B000007463046FEF78CFD2F44013F97FBF0F36C
:101B100003FB10773046FEF783FD06F67434294642
:101B20000646204614F074FD98FBF6F807EE908AFE
:101B300006EE900AF8EEE77A9FED337A77EEA67A12
:101B40003A4667EE877A2046FDEEE77A002117EEE7
:101B5000906AFEF735FE2A46834600212046FEF7AE
:101B60002FFE3A4610F1000A4FF00101204618BF3F
:101B70004FF0010AFEF724FE2A4610F100084FF04C
:101B80000101204618BF4FF00108FEF719FE3A4642
:101B90000221071C204618BF0127FEF711FE2A4626
:101BA0000221051C204618BF0125FEF709FE1BF186
:101BB000000B18BF4FF0010B041C18BF0124D345C4
:101BC00005D0514648463246F317FFF7A9FBB84502
:101BD00008D0002F0CBF0221032148463246F317DC
:101BE000FFF79EFBA5420BD04846002C0CBF0421FA
:101BF00005213246F31701B0BDE8F04FFFF790BB67
:101C000001B0BDE8F08F00BF0050C347AFF30080C4
